:020000040000fa
:100000000200d2021003000000000002100b0000ea
:10001000000000021013000000000002101b00008e
:10002000000000021023000000000002102b00005e
:10003000000000021033000000000002103b00002e
:10004000000000021043000000000002104b0000fe
:10005000000000021053000000000002105b0000ce
:10006000000000021063000000000002106b00009e
:10007000000000021073000000000002107b00006e
:10008000000000021083000000000002108b00003e
:100090000000000208a9e4900002781a79028002a8
:1000a000f0a3d8fcd9fa7a1b7b019000e478107990
:1000b000018015e493a3ad82ae838a828b83f0a383
:1000c000aa82ab838d828e83d8e9d9e712055512b7
:1000d00008c875d00075813f751c8075931e5392ba
:1000e000fe020096001000100000f800ffff001054
:1000f0000000ffe4936670130874019366700c08a7
:10010000740293667005087403936622c008c3e006
:1001100096f50808a3e096420808a3e0964208086e
:10012000a3e09645087001d3d00822c3e493960853
:100130007401939608740293960874039396226050
:1001400016080808c6c313c618c613c618c613c6b1
:1001500018c613c6d5e0ea22e026f008a3e036f080
:1001600008a3e036f008a3e036f022e056f608a334
:10017000e056f608a3e056f608a3e056f622e0f6ad
:1001800008a3e0f608a3e0f608a3e0f622c9c0e061
:10019000e7f20809e7f20809e7f20809e7f2d0e018
:1001a000f922e6f008a3e6f008a3e6f008a3e6f0db
:1001b00022cac0e0e6f30908dafad0e0fa22cac09f
:1001c000e0e2f30908dafad0e0fa22700422600dc6
:1001d00018c6c333c608c633c6d5e0f41822e47384
:1001e0005392fed083d082251cf8c51cc39824fbf3
:1001f000cef208e520f208e9c0e07908e709f20844
:10020000defad0e0f9eff208d0e0fed0e0f208ee3e
:10021000f208e473a81ce2fe08e208f520e9c0e059
:100220007908e208f709dffae208ffd0e0f9e2080e
:10023000c0e0e208c0e0881c5392fe22e584f20888
:10024000e585f222e208f584e2f585227402800059
:10025000c9c0e0e51cc399f51cc91201b1d0e0f991
:100260002274028000c9c0e0e51cc399f51cc912c4
:1002700001bed0e0f922d083d082ecc0e0edc0e036
:10028000eec0e0efc0e0e493a3fce493a3fde493ad
:10029000a3fee493a3ffef4e4d4c60151202f2ec67
:1002a00024fffced34fffdee34fffeef34ffff8052
:1002b000e5e493a3fce493a3fde493a3fee493a3fa
:1002c000ffef4e4d4c601512032fec24fffced3474
:1002d000fffdee34fffeef34ffff80e5d0e0ffd0fe
:1002e000e0fed0e0fdd0e0fce493a3c0e0e493c0e6
:1002f000e022c0e0c0f088f012012ba8f040071205
:1003000000f3a8f0701aa3a3a3a312012ba8f0a3d3
:10031000a3a3a34013d0f0d0e0d0e0d0e00202dcf1
:10032000a3a3a3a3a3a3a3a3a3a3d0f0d0e022c01d
:10033000e0c0f088f01200f3a8f0a3a3a3a3700b11
:10034000d0f0d0e0d0e0d0e00202dca3a3d0f0d027
:10035000e02275bc0075bc005392fe22800f8a8299
:100360008b835392fee0f5bda3aa82ab83ecf8ed3c
:10037000f9e824ff1ce934fffde84970e15392fedf
:1003800022e5bdf9e5bcfae9fb5392fe227400f5c3
:10039000d374022408f5d25392fe22a2afe433f8bc
:1003a000c2af5392fe906270e0a2e740f5e9c3331a
:1003b000906272f0906270e0d2e0f0e0a2e740fb61
:1003c000e8a2e092af2274fa1201e0a2af33f8c2c1
:1003d000afed900002f0eca3f0a37462f0a374738d
:1003e000f0a3e4f0e9a3f0a37412f0a37442f0ebdd
:1003f000906272f0ea906271f07400f5d575d402e3
:1004000075d601906270e0d2e1f0e0a2e740fbe82f
:10041000a2e092af7f010202145392fe906276e056
:1004200054706430700478038002780775c6807455
:1004300080659e70fa9062707408f088c790ff0a19
:10044000e0f5f1a3e0f5f3a3e0f5f4a3e0f5f59012
:10045000ff02e0f586a3e0f5c4a3e0f5c5a3e0f54f
:10046000c2a3e0f5f8a3e0f5fba3e0f5fca3e0f5fb
:10047000faa2fe500ee5f1a2e14008e5ff543f4428
:1004800040f5ff22c008c0098908750900740b787f
:10049000081201cbfae5094480fbd009d008539239
:1004a000fe2274f71201e0909093e064bf7063e560
:1004b000c7f50812035275c7007c937d007a007b54
:1004c0009012035c7c5d7d077aa37b9012035c90a5
:1004d0009094e014f5097f00801674032ffef91242
:1004e0000484eec4540ff5c77c007d0812035c0f32
:1004f000efc3950940e48508c71203818a088b0978
:10050000a808a909909095e0687003a3e069703e7f
:100510008038e5c7f5087fa57e02eef91204848acb
:10052000828b83eec4540ff5c778007908e02fff63
:10053000a3e824ff18e934fff9e84970f00eeec390
:10054000943040d68508c7ef7004790180027900a5
:100550007f04020214e51c24ecf51c5392fe90006b
:1005600001e090001af0e59d541864107005e0a2b7
:10057000e04035e5c7f8790075c700909000e06469
:100580000270010988c7e9a2e0501d1204a2e960c7
:10059000179000017403f0059290011be0f582a30f
:1005a000e0f58305921201de120419900001e4f0d7
:1005b00012038d12076c12075012018d7808120277
:1005c0004c12073b1205d0051c051c12087b80fb52
:1005d000eec0e0a81c12026112078b051c051cd09e
:1005e000e0fe2274f71201e0151c151ca81c120273
:1005f0003ce51c24ecf51ceafeebffee2404f5843c
:10060000e43ff5858e828f83780812017e90012168
:10061000780812016b7808120276000000000500cd
:100620000000000000001007000009001007000093
:1006300009014206000009029a06000009030907a1
:1006400075060592780812017e05929001257808ba
:1006500012010c4032120735f2087480f20874015e
:10066000f2e4f508f509780812024c12073b12056e
:10067000d0051c051ce51c2414f51ca81c12024402
:10068000051c051c02055090011d78081201a212dc
:100690000735f208e4f208f280c890011d780812cc
:1006a000017ee5095407f9e50849701490011d78a9
:1006b0000812017e740b780812013fa90812039bef
:1006c0000592e0f9ee2405fce43ffd059290011d42
:1006d000780812017e7402780812013faa08ab095b
:1006e0001203c60592e0f508e4f509f50af50b05d5
:1006f0009290011d78081201581207237402f20823
:10070000e4f208f2f50802066612072374038082f9
:100710000592e0600912075012018d02066675c944
:100720000880fe12072722e4a81cf2087402f208cf
:100730007409f208221207277401227c007d00e56b
:100740001c2402faab93e51c2403f8e22404f922ea
:10075000a81c7480f2087404f2087409f208e4f228
:10076000f508f509f50af50b087408225392fe9076
:10077000ff0ee0f87404687006900129e4f022741a
:10078000056870069001297401f02274fa1201e0e4
:10079000151c151ca81c12023ce9fe8a828b83e5fd
:1007a0001c2408f8e2fa08e2fb0592900129e060b7
:1007b00020e06401604ba81c120244051c051c7f4c
:1007c00001020214e586a2e040fa5392fee0f5c170
:1007d000a3eeff74ff2f1e0470ea12086c60d7e5c9
:1007e00086a2e040fa8a828b835392fee0f5c1a391
:1007f000aa82ab8380e4a2f840fc5392fee0f5f9b4
:10080000a374ff2e1e0470ee12086c60a9a2f840bb
:10081000fc8a828b835392fee0f5f9a3aa82ab8314
:1008200080e6c084c0858011e586a2e2500be5c158
:100830008a828b83f0aa84ab8512086c6026e586d9
:10084000a2e24004a2fa50f68a848b85439201a367
:100850000592900129e060d0640170dda2fa50d9c0
:10086000e5f980ccd085d0845392fe22ecf8edf9e6
:10087000e824ff1ce934fffde849227c047d007a6e
:100880001b7b0012082290001be05407f9a3e0fc38
:10089000e9fdec4d60077a1f7b001208227a1b7b72
:1008a000001205e3225392fe2274fa1201e0151c95
:1008b000151ceafeebffa81ceef208eff2aa1cab37
:1008c0009379011208a580ee12009322ffffffff2b
:1008d000ffffffffffffffffffffffffffffffff28
:1008e000ffffffffffffffffffffffffffffffff18
:1008f000ffffffffffffffffffffffffffffffff08
:10090000fffffffffffffffffffffffffffffffff7
:100f000012010002000000205824feff0000010230
:100f1000030109021b0001010480250904000000ef
:100f2000fe01020409210d03e84000010104030948
:100f300004120342006c00750065006700690067d9
:100f400000610016034c006f007700200045006e22
:100f50000065007200670079000a03310032003337
:100f6000003400080344004600550000ffffffff67
:100f7000ffffffffffffffffffffffffffffffff81
:100f8000ffffffffffffffffffffffffffffffff71
:100f9000ffffffffffffffffffffffffffffffff61
:100fa000ffffffffffffffffffffffffffffffff51
:100fb000ffffffffffffffffffffffffffffffff41
:100fc000ffffffffffffffffffffffffffffffff31
:100fd000ffffffffffffffffffffffffffffffff21
:100fe000ffffffffffffffffffffffffffffffff11
:100ff000ffffffffffffffffffffffffffffffff01
:10100000021108022fa1ffffffffff023b08ffffb5
:10101000ffffff023bb7ffffffffff023c6effff3a
:10102000ffffff02258cffffffffff0238ceffff0f
:10103000ffffffffffffffffffffff023c0effff71
:10104000ffffff023b92ffffffffffffffffffffde
:10105000ffffff022f87ffffffffffffffffffffe5
:10106000ffffffffffffffffffffff023a45ffff0c
:10107000ffffff023ce0ffffffffff023ac8ffff58
:10108000ffffff022facffffffffffffffffffff90
:10109000ffffffbf2a6e12000000000000000000ea
:1010a0000000b87582fd75837f7400121123e47906
:1010b000347802b800028004f709d8fce4900302f7
:1010c00078dd79058002f0a3d8fcd9fa7ade7b07b7
:1010d000901144786379028015e493a3ad82ae83c6
:1010e0008a828b83f0a3aa82ab838d828e83d8e918
:1010f000d9e77582fa7583da74021211237582f1c9
:101100007583de740212112375d00075813f75312d
:1011100000753202753303759f007593005392fe7c
:101120000210aec09ff59fe473d09f225392fed071
:1011300083d082c09fe493c0e0740193c0e0740246
:1011400093f59f220300000201020300000f00c379
:10115000a88ee8b19dcf7f5eb98b9f41efb055f46b
:1011600001fa00960064004b0032001e001400d605
:10117000be898e000106021213151429417671fff3
:10118000c1fbe84c90728be7b3518963ab23230218
:10119000841872aa612f3b51a8e53749fbc9ca0cd4
:1011a00018532cfd45e300400000fffffffffaff4e
:1011b000ffff00008000620000000500060007003d
:1011c0000000010001000001000102020300020012
:1011d00000000000020201000240420f001900005e
:1011e00000093d0000e4fffffffb349b5f8000002f
:1011f00080001000000000000000800100010000dd
:10120000000000010805000000ff000000000000d1
:1012100007030000008000010000800000040000bf
:1012200000000007090000000d0000010407000095
:101230000000000201000002020000070a0000088e
:1012400005b61abc1ac21ac81ace1ad41a3e1a48bf
:101250001c2a1cae1c961c9c1c800004050200006d
:1012600000800004060600000080000402800004e4
:1012700004800002000b000000800006000e17cc66
:101280001312193e14a81c4e1c7c1bb41c381a5097
:101290000601ffffff0000000080ffffffff0000ce
:1012a0000000c000000012112cc8ae0212112ce088
:1012b000ae0212112c0baf0212112c58af021211f8
:1012c0002c70af0212112c98af0212112ce8af0251
:1012d00012112c18b00212112c79b00212112c9597
:1012e000b00212112cb1b00212112cd6b0021211a0
:1012f0002c2fb10212112cbeb50212112c72b602a3
:1013000012112cd9db0212112cf1db0212112c620a
:10131000dc0212112ca5dc0212112cc3c602121120
:101320002c57c70212112ccdc70212112ce3c70291
:1013300012112c0fc80212112c24c80212112c7d7c
:10134000c80212112c9ec80212112cfcc8021211e4
:101350002c41c90212112cb2c90212112cddc90292
:1013600012112c61ca0212112c90ca0212112caf58
:10137000ca0212112cc3ca0212112c08cb0212117c
:101380002c56cb0212112c09c20212112c25c202ba
:1013900012112c5bc20212112c69c20212112c9a7a
:1013a000c20212112cc7c20212112cd0c202121199
:1013b0002c13c30212112c99c30212112c06c40261
:1013c00012112c57c40212112c86c40212112cdaed
:1013d000c40212112cacc50212112cb7c502121195
:1013e0002ceac50212112c1bc60212112c6cc6026b
:1013f00012112ca9c60212112c9f7f0012112cbfb2
:101400007f0012112ce87f0012112c56dd02121100
:101410002c6add0212112cc1dd0212112cdade025f
:1014200012112cd3dc0212112c00dd0212112c0f30
:101430009d0212112c769d0212112c8d9d0212110b
:101440002cd19d0212112c179e0212112c6b9e02a0
:1014500012112cbe9f0212112c97a00212112c3ec9
:10146000a10212112c62a10212112ca4a1021211cc
:101470002c3fa20212112c8da20212112ceba202ff
:1014800012112cfea20212112ceea30212112cf04a
:10149000a40212112c62a50212112cb93d001211e6
:1014a0002c5f3f0012112ce33f0012112c31410040
:1014b00012112ca0410012112cda410012112ca49f
:1014c000420012112c32430012112c11440012114f
:1014d0002c25450012112c17460012112c514700e3
:1014e00012112caa470012112c12480012112c8f35
:1014f000480012112c30490012112ca2490012117f
:101500002c3b4a0012112ca14a0012112c0f4b0047
:1015100012112c644b0012112cec4b0012112ca256
:101520004c0012112c584d0012112c1a4f001211a0
:101530002c4b510012112c90510012112c0c520006
:1015400012112c75520012112cc3520012112c6f63
:10155000540012112c0f550012112c9b5500121122
:101560002cdc550012112c5d570012112cbe5700b7
:1015700012112ce0580012112ce7590012112c16f0
:101580005b0012112c4a5c0012112c225e00121119
:101590002ce0600012112c78610012112c356200d1
:1015a00012112c26630012112c86630012112ce5f7
:1015b000670012112c606a0012112c2e6b001211a0
:1015c0002c6e6d0012112c846e0012112cad6f0068
:1015d00012112cc46f0012112c5ccb0212112c9b27
:1015e000cb0212112cc8cb0212112cf5cb02121116
:1015f0002ce2cc0212112cb9cd0212112ce5fe0105
:1016000012112c3eff0112112c9fff0112112c0010
:10161000800112112c1e800112112c3b800112112d
:101620002c58800112112cde800112112cf682013f
:1016300012112c5c830112112ccc830112112c0c81
:10164000840112112c40840112112c828401121188
:101650002cf0840112112c9e850112112cb68501eb
:1016600012112ced860112112c1b890112112ca1d3
:10167000890112112cd5890112112c138b01121121
:101680002c318c0112112c528c0112112c708c01f6
:1016900012112cac8c0112112cdf8c0112112cb305
:1016a000900112112cdb900112112c2791011211c3
:1016b0002ceb960112112c37970112112c789701ff
:1016c00012112c24980112112ce5980112112c7280
:1016d0009b0112112cc19c0112112c319d01121180
:1016e0002c7b9f0112112cf69f0112112c3aa001a4
:1016f00012112c86a00112112cdea00112112c7fd8
:10170000a10112112cc9a10112112c24a201121144
:101710002c2ea20112112c61a30112112cf4a30191
:1017200012112cb4a40112112c51a50112112ce795
:10173000a60112112c08a70112112c63a901121184
:101740002c7daa0112112c1dab0112112c91ab01a1
:1017500012112c2dac0112112c38ae0112112c4992
:10176000ae0112112c53ae0112112c3ab00112111c
:101770002ca1b00112112cd0b00112112c3eb101dc
:1017800012112c6db10112112c15b20112112c93f2
:10179000b20112112cfdb20112112c73b3011211fe
:1017a0002ca9b30112112cdeb30112112cfdb301cf
:1017b00012112c5cb40112112c6ab40112112ca963
:1017c000b40112112c18b50112112cafd60212114e
:1017d0002c6bd70212112c8dd70212112cd8d702e4
:1017e00012112c1bd80212112cbcde0212112cd2a9
:1017f0008f0212112cfe8f0212112c469002121130
:101800002c9b900212112cfc900212112c5d930261
:1018100012112c8f940212112c9c970212112ce0a1
:10182000970212112ceb980212112ced9902121151
:101830002c689b0212112cdd9b0212112cf09c02d1
:1018400012112cffcd0212112c2bce0212112c42a0
:10185000ce0212112c46ce0212112ce0ce02121131
:101860002c05d00212112c97de0112112cf8de018a
:1018700012112c15df0112112c42df0112112c6ef6
:10188000df0112112ca2df0112112cf1df01121164
:101890002c20e00112112c83e00112112ce0e00158
:1018a00012112caee10112112c28e20112112cc9e7
:1018b000e30112112c81e40112112c2fe701121106
:1018c0002cd5ea0112112c16eb0112112c6feb0131
:1018d00012112c1fec0112112cfded0112112c8d97
:1018e000ee0112112cceee0112112c24ef01121177
:1018f0002c7cef0112112ca2ef0112112cf5ef013b
:1019000012112c36f00112112ca7f10112112cc862
:10191000f20112112cd9f20112112c5df4011211f5
:101920002c73f40112112c9bf40112112c3bf501c4
:1019300012112c50f50112112c82f50112112c8874
:10194000f60112112c1ff70112112c55f70112117b
:101950002c9df70112112c91f80112112cecf801b9
:1019600012112cd3f90112112c46fa0112112c8af2
:10197000fa0112112c70fb0112112cccfd01121175
:101980002cfcfd0112112c7cfe0112112c6dd802d1
:1019900012112c7ad80212112c9dd80212112ce0af
:1019a000d90212112cedd90212112c1bda021211dc
:1019b0002c4dbd0212112c6cbd0212112c37be022f
:1019c00012112cddbf0212112c3bc00212112c6d22
:1019d000c10212112cd6c10212112c0a7f00121161
:1019e0002c387f0012112c627f0012112c9ed00225
:1019f00012112c27d10212112c59d10212112cc90b
:101a0000d10212112c6bd20212112c93d20212119c
:101a10002cdeb50112112c34b60112112c3ab8018a
:101a200012112cc5b90112112c8bba0112112c9b69
:101a3000bb0112112c39bc0112112cb6bc011211c0
:101a40002c68bd0112112cd0bf0112112c50c00105
:101a500012112cb4c00112112c5ec10112112c7094
:101a6000c20112112c75c30112112cf6c7011211fb
:101a70002c45ca0112112cf0cc0112112ca2cf015d
:101a800012112c82d20112112c65d40112112cd00a
:101a9000d60112112c68db0112112c19dd01121173
:101aa0002c96dd0112112c20de0112112c74de01a6
:101ab00012112cd1d40212112c4fd50212112c6507
:101ac000d50212112c7bd50212112c91d5021211c4
:101ad0002cb2d50212112cc8d50212112cded5025f
:101ae00012112c9a760012112c2a770012112cadab
:101af000770012112cd3770012112c9f780012114d
:101b00002c55790012112c95790012112c1b7a009a
:101b100012112c8d7a0012112cef7a0012112c6cfc
:101b20007b0012112c7f7b0012112c937b00121171
:101b30002cc87b0012112cfa7b0012112c2c7c007b
:101b400012112c727c0012112cb27c0012112c0686
:101b50007d0012112c157d0012112c1e7d0012111a
:101b60002cb17d0012112ce87e0012112c8eb602d1
:101b700012112c9db60212112c9bb70212112cad22
:101b8000b70212112c3bb90212112cf0b90212113a
:101b90002c59ba0212112c72ba0212112c88ba02f4
:101ba00012112cc2ba0212112c05bb0212112c4fb9
:101bb000bb0212112c98bb0212112c63bc02121131
:101bc0002c71bc0212112c79bc0212112ca1bc0286
:101bd00012112cbabc0212112cdfbc0212112cff04
:101be000bc0212112c0fbd0212112c1fbd021211ca
:101bf0002c31bd0212112c3fbd0212112c24da022d
:101c000012112c51da0212112c00800212112ca791
:101c1000800212112cff800212112c42810212113b
:101c20002c158d0212112c478d0212112c4a8f0295
:101c300012112ce4d20212112c46d30212112c6a7a
:101c4000d30212112cb9d30212112c0dd40212118d
:101c50002caed40212112cc7d40212112c98a60259
:101c600012112cb5a60212112cc5a70212112c2498
:101c7000a80212112ccca80212112c4baa0212118c
:101c80002cf7aa0212112c3eab0212112c9cab02b3
:101c900012112c02ac0212112c54ac0212112ce0c5
:101ca000ac0212112c5bad0212112c34ae021211d7
:101cb0002cffde0212112c03df0212112c05df02b1
:101cc00012112c0bdf0212112ca3100012112ccdbb
:101cd000dd0212112c3ade0212112c8dde02e766b3
:101ce00070100809e766700a0809e76670040809b9
:101cf000e76622e066701008a3e066700a08a3e0b9
:101d000066700408a3e06622c3e7960809e7960810
:101d100009e7960809e796a2d265d03322c3e09678
:101d200008a3e09608a3e09608a3e096a2d265d0a7
:101d30003322c021c3e096f52108a3e09642210892
:101d4000a3e096422108a3e0964221a2d265d033b7
:101d5000e5217001d3d02122c3e7960809e7960850
:101d600009e7960809e79622c3e09608a3e09608db
:101d7000a3e09608a3e09622c021c3e096f52108cf
:101d8000a3e096422108a3e096422108a3e09645ed
:101d9000217001d3d02122080808eac0e0ebc0e09e
:101da00086f0e7a4fa180986f0e7a42afa1809864b
:101db000f0e7a42afa180986f0e7a42afa1986f0af
:101dc000e7a4fbe5f02afa190886f0e7a42bfbe567
:101dd000f03afa190886f0e7a42bfbe5f03afa1876
:101de000180986f0e7a4c5f02bfbe43afa1908e7d6
:101df000c5f0c6a426f6e5f03bfbe43afa1886f0f7
:101e0000e7a4f6e5f00826f6e43b08f6e43a08f61f
:101e1000d0e0fbd0e0fa22e4cfc0e0e4cec0e0e4c2
:101e2000cdc0e0e4ccc0e075f020e626f608e6334d
:101e3000f608e633f608e633f6181818ec33fced2e
:101e400033fdee33feef33ffc3ec9709ed9709ee58
:101e50009709ef97191919400fffec97fc09ed97b7
:101e6000fd09ee97fe191906d5f0bfecf709edf75d
:101e700009eef709eff7191919d0e0fcd0e0fdd011
:101e8000e0fed0e0ff22121eee181818121e1712e4
:101e90001edd19191922121edd191919080808e684
:101ea00018181820e7e0121e17121eee1818182234
:101eb000090909e719191920e7dc080808e61818c4
:101ec0001820e703021e17121eee181818121e170c
:101ed000121eee181818121edd19191922e4c397e4
:101ee000f709e497f709e497f709e497f722e4c3c1
:101ef00096f608e496f608e496f608e496f622606c
:101f000017080808c6a2e713c618c613c618c613d2
:101f1000c618c613c6d5e0e9226016080808c6c36d
:101f200013c618c613c618c613c618c613c6d5e0fe
:101f3000ea227009080808226016181818c6c33368
:101f4000c608c633c608c633c608c633c6d5e0ead7
:101f500022e627f60809e637f60809e637f6080903
:101f6000e637f622e026f608a3e036f608a3e036c8
:101f7000f608a3e036f622e026f008a3e036f008e3
:101f8000a3e036f008a3e036f022c3e697f608098e
:101f9000e697f60809e697f60809e697f622c3e001
:101fa000c696f608a3e0c696f608a3e0c696f6081d
:101fb000a3e0c696f622e657f60809e657f60809a2
:101fc000e657f60809e657f622e056f608a3e0566b
:101fd000f608a3e056f608a3e056f622e647f60810
:101fe00009e647f60809e647f60809e647f622e05b
:101ff00046f608a3e046f608a3e046f608a3e04646
:10200000f622e046f008a3e046f008a3e046f00818
:10201000a3e046f022e667f60809e667f60809e657
:1020200067f60809e667f622e066f608a3e066f6ba
:1020300008a3e066f608a3e066f622e0f608a3e04f
:10204000f608a3e0f608a3e0f622e6f008a3e6f01f
:1020500008a3e6f008a3e6f022e0faa3e0fba3e081
:10206000fca3e0fd22eaf0a3ebf0a3ecf0a3edf07b
:1020700022e0fca3e0fda3e0fea3e0ff22ecf0a33e
:10208000edf0a3eef0a3eff022e0f8a3e0f9a3e077
:10209000faa3e0fb22e8f0a3e9f0a3eaf0a3ebf057
:1020a00022cac0e0e6f0a308dafad0e0fa22cac0f9
:1020b000e0e0a30592f0a30592daf6d0e0ca22533d
:1020c00092fefae9fb7921e7f0a309dafae8f0a336
:1020d000ebf9f0a3ecf0a3edf0a3eef0a3eff0a387
:1020e000e520f0a3e5f0f0a3e592f0a3e584f0a3ea
:1020f000e585f0a3e581f0a3e531f0a3e532f0a397
:10210000e533f0a3d0e0fad0e0f0a3caf0eac0e0f3
:10211000e0c0e07a007b00225392fecac0e0ebc030
:10212000e07921e0f7a309dafae0f8a3e0f9a3e007
:10213000fca3e0fda3e0fea3e0ffa3e0f520a3e005
:10214000f5f0a3e0c0e0a3e0f584a3e0f585a3d01b
:10215000e0f592d0e0fbd0e0fae0f581a3e0f531c4
:10216000a3e0f532a3e0f533a3d0e0d0e0e0c0e097
:10217000a3e0c0e0ea4b70027a0122b90010bb0074
:1021800008e88af084f8aaf022e4fbc8fa22eb708f
:10219000227b10c833c8c933c9335007c39ac3db85
:1021a000f280069a50012adbeac833f4c8c933f436
:1021b000c9fa2275f008e4c833c8c933c933c99acb
:1021c000c99b5004c92ac93bd5f0ecfbc833f4c8fd
:1021d000e4c9fa22600d08c6a2e713c618c613c6e2
:1021e000d5e0f322600c08c6c313c618c613c6d5c3
:1021f000e0f422700422600d18c6c333c608c6334b
:10220000c6d5e0f41822253210af08f532400c157f
:10221000338008f53240021533d2af2200c0d025fa
:102220003210af08f532500c05338008f5325002f9
:102230000533d2afd0d0222532f58210af08f53267
:10224000400c15338008f53240021533d2af853388
:102250008322c5822532c582c583353310af07f589
:10226000338582328007f533858232d2afc583222f
:102270002532f582e43533f583222532f584e435c1
:1022800033f585222532f8e43533f9222532fae494
:102290003533fb222532fce43533fd22e4735392bf
:1022a000fe2532c582c0e0e53334ffc583c0e0e5da
:1022b00032c3958224f810af08858333858232803b
:1022c00008858333858232d2afcef0a3e520f0a318
:1022d0007821e608f0a3defaeff0a3e58124faf80e
:1022e000e608f0a3e608f0a3e608f0a30808e6086d
:1022f000f0a3e608f0a315811581d0e0fed0e0f848
:10230000158115811581e8c0e0eec0e0225392fef0
:102310002532c582c0e0e53334ffc583c0e0e53235
:10232000c3958224f910af088583338582328008f3
:10233000858333858232d2afcef0a3e520f0a37837
:1023400021e608f0a3defaeff0a3e58124fbf8e62e
:1023500008f0a3e608f0a30808e608f0a3e608f0f2
:10236000a315811581d0e0fed0e0f815811581e834
:10237000c0e0eec0e0225392fe853383853282e0d6
:10238000a3fee0a3f5207821e0a3f608dffae0a39e
:10239000ffe0a3c0e0e0a3c0e0e0a3c0e0e0a3c092
:1023a000e0e0a3c0e010af08858232858333800867
:1023b000858232858333d2afd083d0825392fe029e
:1023c00011295392fe853383853282e0a3fee0a378
:1023d000f5207821e0a3f608dffae0a3ffe0a3c030
:1023e000e0e0a3c0e0e0a3c0e0e0a3c0e010af08dd
:1023f0008582328583338008858232858333d2afec
:10240000d083d0825392fe22c0925392fec0d02538
:1024100032c582c0e0e53334ffc583c0e0e532c396
:10242000958224f210af0885833385823280088537
:102430008333858232d2afc8f0a3e9f0a3eaf0a3d8
:10244000ebf0a37921e709f0a3d8faecf0a3edf0c3
:10245000a3eef0a3eff0a3d0e0f0a3d0e0f0a3d080
:10246000e0f0a3e520f0a3e5f0f0a3d0e0f02253e4
:1024700092fe853383853282e0c0e0a3e0f9a3e0d9
:10248000faa3e0fba37821e0f608a3dffae0fca3bf
:10249000e0fda3e0fea3e0ffa3e0c0e0a3e0c0e016
:1024a000a3e0f5d0a3e0f520a3e0a3f5f0e0a3c0fe
:1024b000e010af08858333858232800885833385b9
:1024c0008232d2afd0e0d082d083f592d0e0f8d083
:1024d000e032e584f0a3e585f022e0a3f584e0f5a1
:1024e000852274048006740280027401c0e0f40442
:1024f000122237d0e01220a12274048006740280d8
:10250000027401c0e0f404122237d0e01220ae229f
:10251000d083d082c5f0e493a3c5f0c395f0f5f065
:10252000e493a3c395f04005e5f0048001e475f061
:1025300002a42582f582e5f03583f583e493a3c0f8
:10254000e0e493c0e022d083d082e9c0e0e493a32a
:10255000c386f0c5f095f0f908e493a386f0c5f0c2
:1025600095f0700be493a3c3994005e9048002a39e
:10257000e475f002a42582f582e5f03583f583d079
:10258000e0f9e493a3c0e0e493c0e022c0e0c0d04f
:1025900075d008c092c082c083c0f0759800e5a8cd
:1025a000f8c2af5392fe9004d4e0d2e1f07534004b
:1025b000e8a2e7e433fee8a2e792af1212eed0f011
:1025c000d083d082d092d0d0d0e032c082c08353aa
:1025d00092fe9004a3e4f0a3f0a3f0a3f0d083d084
:1025e000822274f712230d790012198a9003ef12d8
:1025f0002e0aeac398f8eb99f9e82404fee439ffbf
:102600009003fce0fca3e0fdc3ee9cef9d402e9008
:1026100003fae0fca3e0fd9003fee02af8a3e03b10
:10262000f9e8c39cf8e99df99003ef122c28a3ec7c
:10263000f0a3edf09003fcecf0a3ed80239003ef0a
:10264000122ae19003fc122c069003fc122e0a9031
:1026500003f1122c289003f8e07004740280011436
:10266000f07aed7b03123713800ff08532828533c9
:10267000831224da740212221c7f020223c274f72e
:1026800012230de9fe9003f9e0f8ee600924fe60e4
:102690001d14601a80329003f6e0a2e35009e8604e
:1026a000279003f9148020c2e2f0d2e3801990034e
:1026b000f6e0a2e2500c740868600d9003f9e004a3
:1026c0008005c2e3f0d2e2f09003f7e070089003d7
:1026d000f574fff0804890600a122ad9703d90612d
:1026e0008fe0c0e09003f9e0f87408c398f8d0e0f8
:1026f000b800028004c313d8fcf52174ff65217073
:102700000990600ae4f0a3048010e5212401f8e4b4
:102710003400f990600ae8f0a3e9f01225e20226fd
:102720007974f712230de9fe24fc600624fe602a6a
:10273000800d9004bce06401705d1216d880589042
:102740000416e064017013900410e4f0ee700b7b4b
:10275000091238b4fa790012397d900410e070083b
:1027600090040e74fff0802f90618fe0ff790012cb
:10277000198a8b22a922900412e02af8a3e039f9e1
:10278000740f5ffae82af8e439f9900408122c284b
:102790007a067b0412371302267974f712230d741c
:1027a000fe1222371224d2900460122e0ae824125c
:1027b000fae439fb90605ce060088a828b83e0d2a7
:1027c000e1f0e82430fce439fde82432f584e43912
:1027d000f58590605ae0700690605ee060368a820f
:1027e0008b83e0a2e14019d2e1f0e82422f582e4f3
:1027f00039f583122ad11221f38c828d831231cfc5
:10280000e40592f0a3f079008532828533835392f8
:10281000fe022671e81231ad39f583123525858423
:1028200082858583e02ef0a3e03ff08c828d8305c6
:1028300092e0fca3e0fdc30592e09ca3e09d50c69e
:1028400088828983a3a3a3a3a3a3a3a3a38582842c
:102850008583858a828b83e0a2e15004740880021c
:10286000743e0592f07b02888289830592a3a3a31c
:10287000a3a3a3a3a3e0fa790012397d790180888c
:1028800074f512230d74fe1222371224d2122ac9b3
:10289000240af584e43ff5850592e0fc7003022ae2
:1028a000c4122dea0592122e0a8e828f83a3a3a34f
:1028b000a3a3a3a3a38582238583248e828f83a3ce
:1028c000a3a3a3a3a3a3a3a3aa82ab83ee2434123e
:1028d00034bf687003a3e069701a74026c7003025d
:1028e0002a5d74016c607a74096c60258a828b831e
:1028f00074228058ec146069147003022a5d24fa73
:10290000601c14600c146045147003022aa0022a93
:10291000c4906008e0a2e65003022ac4802fee248f
:1029200039f582e43ff583801388828983a3a3a3ca
:10293000e064037003022ac488828983122ad97052
:10294000e88a828b83e0641370037416f07b02853f
:102950002382852483e0fa790012397d7901022ae5
:10296000c6ee245512311fee244cfce43ffdea2450
:10297000fff521eb34fff522e521687003e52269bc
:102980007075ee244d122b678e828f83122adf8c96
:10299000828d83e025e0f8e433f9e82403f8500160
:1029a000098e828f83a3a3a3a3122c29900491e004
:1029b000a2e050098e828f83a3a3122c249004ab33
:1029c000e4f0a3f0a3f0a37402f0900491e0a2e07d
:1029d0004003022ac4906062e4f08c828d83e0f8a8
:1029e00075f0e2a4c8aaf075f004a42af9e8122d43
:1029f000fc122c28022ac4ea687002eb6960030208
:102a00002ac475210975220078211224e6ee241bc0
:102a1000fae43ffb121cd2740212221c900491e0d3
:102a2000a2e05007eefaeffb12312be40592f0ee34
:102a30002422f582e43ff5830592122ad11221f374
:102a4000ee2430f582e43ff5831231cfee2432f5e7
:102a500082e43ff583e4f0a3f07b08805ae8240188
:102a600008500109ee245c1234bf687003a3e069ca
:102a7000705275210575220078211224e6ee245744
:102a8000fce43ffdee2424fae43ffb121cd2740266
:102a900012221ceefaeffb1216d2e40592f080240b
:102aa000eefaeffb1212f4e40592f0059290049115
:102ab000e0a2e0500f7b07852382852483e0fa792a
:102ac0000012397d7900022efa900460123525ee4d
:102ad00022122c1c7403782122122e0ee84922a304
:102ae000a3e028f0a3e039f02274f812230d74fe5d
:102af0001222371224d2900460e0f584a3e0f58519
:102b0000122880e9704e12279ae97048e584242e35
:102b1000f582e43585f583e02401f0a3e03400f08c
:102b2000906008e0c0e0e5842436f582e43585f560
:102b300083d0e0f0e5841231ad3585122b6b059220
:102b4000a3a3e028f0a3e039f005929004601231cd
:102b5000251237138532828533831224da740212e8
:102b6000221c7f010223c2f582e43ff583122b7100
:102b700022e0f8a3e0f9e828f8e933f92274f71223
:102b8000230d74fe1222371224d28a828b83a3a3d0
:102b9000ac82ad839004b0ea241ef584e43bf58555
:102ba0000592e0f8a3e0f9e828f8e933f9900493f6
:102bb000e0f521a3e01231b30592e028f8a3e03953
:102bc000f98c828d83122c289004ab122c0f8c82ee
:102bd0008d83122c069004ad122c0f7a207b4e129e
:102be000217b882189228c828d83e09521f0a3e0ce
:102bf0009522f09004b2122c0fe828f8e933f9e896
:102c0000122df402266ac3e098f0a3e099f0221294
:102c10002e0e900493122c1c1231b922e0f521a340
:102c2000e0f52222a3a3a3a3e8f0a3e9f02274f71e
:102c300012230d74fe1222371224d2122ac9241232
:102c4000f584e43ff5850592e0a2e35008c2e3f085
:102c50000592022dde8e828f830592a3a3858221a9
:102c6000858322906062e06010791012198a8521b4
:102c700082852283eaf0a3ebf0122880e960030248
:102c80002de712279ae96003022de7906008e0c063
:102c9000e0ee2436f582e43ff583d0e0f09061d594
:102ca000e0f89061d7e06805926005e0d2e2800329
:102cb000e0c2e2f00592906062e09004ad6017e03f
:102cc00024c0faa3e03437fb1239529004b2123513
:102cd0002b122df4801512312512393c9004b212ba
:102ce0002b6d906064e028f0a3e039f085218285a7
:102cf0002283e024fff0a3e034fff0ee242b123413
:102d0000bf9004aff0ee2420f582e43ff583122a51
:102d1000d960498e828f83a3a3a3a3a3a3a3a3a354
:102d2000a3e07038ee243212311fea4b702eee24ed
:102d30003912311fea4b7024e82401500109900434
:102d400093122c29852182852283122e0a9004b0a9
:102d5000122c28eefaeffb122b7d8027900493743f
:102d600001f0a3e4f0ee241e122b67852182852258
:102d700083122ae19004ab122e0a852182852283d8
:102d8000122c068e848f850592a3a3a3a3a3a3056b
:102d900092906064122e0a7a717b0212217b892242
:102da000e82405f8e43522f9858482858583122c90
:102db000288e828f83a3a3a3a312312585848285c5
:102dc0008583e0f8c3ea98eb99a2d265d033500529
:102dd000eaf0a3ebf0122e07122dea122ae190047a
:102de0006012312512371302266bee242ef582e491
:102df0003ff58322122dfce8f0a3e92224eaf8e94a
:102e00003402f990606422900493122e0e22e0f8ae
:102e1000a3e0f92274f512230d74fe122237122456
:102e2000d28031c2e51238afc0e09004bae0122e71
:102e3000dfd0e0f09004bae004f0a3e004f0a3e0f7
:102e400004f09004bee0700c7401f07b007a00790d
:102e50000012397d90605ae0f521906002e0a2e016
:102e600050047800800590605de0f89004bbe0fac3
:102e7000e52128f8e43400f9e86a7001e960589027
:102e800004bae0f52374012523547ff521e52312cc
:102e90002edfe0f808089004bae028f074802521bd
:102ea000f582e43460f5830592900460e0f8a3e0d5
:102eb000c82408f584e438f585e0a2e70592e040ef
:102ec00003022e23d2e5f0122ef124db1238affae2
:102ed000122ef14a022e33853282853383802412ea
:102ee0002ee322547ff8748028f582e43460f58361
:102ef000229004bae0122ee3e022853282853383e9
:102f00005392fe1224da740212221c7f040223c29e
:102f100074f512230d74fe1222371224d289210572
:102f200092900460e0f582a3e0f583858284858336
:102f300085a3a3a3a3a3a3a3a3e0a2e74046900471
:102f4000bde0f8906054e0c398f5229004bde02500
:102f500022f0ae82af838011ee2439fae43ffb12f7
:102f600015faea4b60031217e085222374ff25232c
:102f7000f5220470e3e521a2e640097900eefaefbc
:102f8000fb121750022efac0e074f11224088535a6
:102f9000c675a70075a10079501219a87f010224f7
:102fa0006fc0d075d01875bf00d0d032c0e0c0d08f
:102fb00075d018c092c082c083c0f08535c6e59137
:102fc000fe759b00f4f5915392fe906002e0a2e042
:102fd00050047800800278087900e844015e6003bc
:102fe000122e14eea2e55004f9122f10eea2e750b3
:102ff00029e5a8f8c2af9004d4e0d2e0f07534001f
:10300000e8a2e7e433f9e8a2e792afe594a2e24050
:1030100009759403e594a2e250faeea2e640030299
:1030200030ec906061e0f99004bbe4f09004bdf0f6
:103030009004601231258a828b83a3a3a3a3a3a348
:10304000a3a3e02410601224fc600924fc700f127a
:10305000267e8066122721806112161e805c9004f5
:1030600090e060051460148023906060e0648060ec
:103070001be0c0e0123109d0e08010906058e0f809
:1030800090605ce028f8123109e028f0906060e080
:1030900064806016e0c0e0900460e0f8a3e0c8241b
:1030a00013f582e438f583d0e0f0900491e0a2e0db
:1030b0005005122c2e8003122ae9906059e0f890f6
:1030c00004a3e028f0906058e0f89004a4e028f011
:1030d00090605a12310090605e12310090605ce0a6
:1030e000f89004a6e028f012160c8004a2e7500322
:1030f000123758d0f0d083d082d092d0d0d0e032e6
:10310000e0f89004a5e028f022ea242cf582e43bc4
:10311000f583e0fa746b2af582e43404f58322f532
:1031200082e43ff583e0faa3e0fb2274f712230d5b
:10313000ea242af582e43bf583e025e0f8e433f95c
:1031400074f928f582740739f583e02432f8a3e096
:103150003400f9ea1231ad3bf583e0f521a3e0122a
:1031600031b3e8241ff8e93403f97a207b031221f4
:103170007b88218922ac21ad227a717b0212217bce
:103180008a218b22740578211221f39004ad12312b
:10319000cfecf8edf97a717b0212217b9004ab122f
:1031a0002c289004b2ecf0a3edf0022679241ef551
:1031b00082e422f5221231b922e88521f0a4c8aabe
:1031c000f08522f0a42afa8521f0e9a42af922e563
:1031d00021f0a3e522f02274f712230d74fe1222cf
:1031e000371224d2900460e0fca3e0fd122e07ec1d
:1031f0002429f582e43df583ec242bfae43dfb8a97
:10320000848b85740168497012e0f80592e028fa11
:10321000c39425402974db2afa8023e0f521e88550
:1032200021f0a4f8aaf08521f0e9a42af90592e09a
:10323000fae82af8e439f97a257b0012217beaf0d2
:10324000ea131313541ff8ec28f8e43df9e824249a
:10325000f582e439f5830592e0c0e074075af8d0ae
:10326000e0b800028004c313d8fca2e04028800527
:10327000e8cac39afaec24e5f582e43df583e0f868
:10328000eac39850ebec2af8e43df9e824c0f58253
:10329000e439f583e0faec242cf582e43df583ea89
:1032a00002266a74f612230d74fe1222371224d2fb
:1032b000900417e09060026004740e8002740ff0b6
:1032c000900411e0906001f090080912208990614b
:1032d0009512209512175c900416e0f52174016593
:1032e0002190040f7040e05402f97a187b04121602
:1032f0003c90040fe0a2e050097a9d7b04752140c8
:1033000080077a977b04752100a2e150047e8080bb
:10331000027e0075230678231224ea7c187d04e5da
:10332000214e44018068e0a2e050087a9d7b047839
:103330004080067a977b047800059290043d122520
:10334000017c1e7d04740d2521f582e43408f5838b
:103350000592e048f9121642740112221c900416dc
:10336000e0f86005740268702e90040fe0a2e0504f
:10337000087a9d7b04784080067a977b0478000564
:103380009290045d1225017c3e7d04e84404f9120c
:103390001642740112221c90040fe0a2e0e433f9fb
:1033a000121636759100900417e0906182600474e3
:1033b000c8800274c0f08532828533831224da74a7
:1033c0000212221c7f030223c2c082c0835392feda
:1033d000906002740ff09003f8e004f06403700250
:1033e000e4f0e02425906000f09008091220899014
:1033f00061951220959003f6e05420f912163612ca
:10340000175c9003f6e0a2e15004d2f08002c2f013
:10341000a2f0e43390600cf09003f6e0a2e15035a6
:1034200075d90da2e55004784080027800e8440385
:10343000f5d9e0a2e550067a9d7b0480047a977b5b
:10344000047906121612740675d9001470fae5e1b3
:1034500070fc75e19575910090618274c10225dc64
:1034600074f812230d74fe1222371224d21235186a
:1034700012175c12350e1220899061951220951258
:1034800035611231d7123548f584e43ff5858584de
:1034900082858583123530121750ee24121234bf04
:1034a000a2e250180592e0f8a3e0f5838882059225
:1034b000a3a3e02402f89061d5e028f0022b54f594
:1034c00082e43ff583e02274f812230d12351812be
:1034d000175c12350e1220899061951220951235d5
:1034e000611231d7123548f582e43ff58312353049
:1034f000121750ee1231ad3ff58312352b24fcf834
:10350000e934fff98e828f83122c24022b62ee2481
:1035100014f582e43ff58322900460123525906013
:1035200002740ff022e0fea3e0ff22122b71e822ca
:10353000122e0eee2437f582e43ff583e8f0a3e97e
:10354000f07900eefaeffb22ee242c1234bf9060eb
:1035500000f07591009004c8e0906182f0ee24398b
:1035600022ee24361234bf906008f0ee2418123494
:10357000bf906005f0ee24191234bf906006f0eea3
:10358000241a1234bf906007f02274f112230d74d4
:10359000fe1222371224d27521007522007c677d2d
:1035a00004801b888289831235258c828d83eef0fe
:1035b000a3eff0888289831231cf882189228c82ff
:1035c0008d83122acc4f70398c828d83eaf0a3eb65
:1035d000f08a828b83e4f0a3f0aa21ab22853282a9
:1035e0008533831224da740212221c7f080223c25c
:1035f000e5232527f8e5243528f98a828b83122aca
:10360000dfeef8eff988828983a3a38a848b85058e
:1036100092a3a3e0f523a3e0f5240592e0c395234c
:10362000f523a3e09524f5248a828b83a3a3a3a387
:10363000a3a3e0f525a3e0f526c3e5239525e5241e
:103640009526a2d265d033403e8a828b83122c28e5
:103650008a828b83a3a3a3a3858284858385122e6c
:103660000ac3e52398e52499a2d265d033500d858d
:103670008482858583e523f0a3e524f08c828d8305
:10368000eaf0a3eb0235d888828983a3a3a3a3a37e
:10369000a3e0f527a3e0f528c3e49527f525e495f5
:1036a00028f526c3e5259523e5269524a2d265d0e5
:1036b0003350288a828b83a3a3a3a3a3a3a3a3e04d
:1036c000a2e750030235f088828983a3a3a3a3a3b2
:1036d000a3a3a3e0a2e750030235a388828983a3b2
:1036e000a3a3a3858284858385c3e49523fce49505
:1036f00024fd123525c3ec9eed9fa2d265d0335038
:103700000b858482858583ecf0a3edf0e8fce9fd70
:103710000235be74f712230d74fe1222371224d222
:10372000ea4b6031a2afe433fec2af12358a8a821f
:103730008b838016aa82ab838582848583850592dc
:10374000e0f582a3e0f58312358ae582458370e4d3
:10375000eea2e092af02266b74f512230d790012ef
:10376000198a8a238b2479771219a89061b1e4f021
:10377000e070f87403f0e0640370f8900467122eb0
:103780000a900460122c28e8497012123898e594c7
:10379000a2e240030238927594000238928882892e
:1037a00083123125900467eaf0a3ebf088828983c5
:1037b000a3a3122c1c88828983a3a3a3a3e02521a1
:1037c000f8a3e03522f9e824fdfee934ffff90601c
:1037d0006074801238af2410601424fc600624fc4e
:1037e000600780451232a380501233c9804be52117
:1037f000c39523e5229524c39400a2d265d033500b
:1038000023e5232401f521e43524f522c3e5219e97
:10381000e5229f4009e5212401fee43522ff9003c3
:10382000ef1231cf1217628010900491e0a2e050a5
:103830000512346080031234c7aa21ab22793012fa
:10384000199ceefaeffb794012199c79541219a8d1
:10385000e521c39523f8e5229524f9c3e89401e90d
:103860009400a2d265d033500c121774e5e170fcbd
:1038700075e121801d900367e0a2e04012aa21ab10
:10388000221219969004a71220651238988003120c
:10389000177412185e022f0be5a8f8c2af9004d47b
:1038a000e0c2e0f0753400e8a2e7a2e792af22f0b0
:1038b0001238b422900460e0f8a3e0c82408f5822e
:1038c000e438f583e0220000853487c2af22c0e0ef
:1038d000c0d075d018c092c082c083c0f074fc12f2
:1038e00022065392fe9004d5e0601c12163090031d
:1038f00067e054117008e5c654384487f5c6900453
:10390000d5e4f0c2c78020c2c7aa32ab3312176e0b
:10391000e9640170129004d57401f0853282853318
:1039200083122059121852753400740412221cd0cc
:10393000f0d083d082d092d0d0d0e03275c3007462
:1039400020c39afa744e9bfbeaf5a2ebf5a35392bf
:10395000fe22c02175c301e5a2f521e5a375c300d0
:10396000f9e5212420f8e9344ef9e8c39af8e99bf7
:10397000f9e8f5a2e9f5a3d0215392fe2274f512dd
:10398000230de9feeaff8b21753400a2afe433f585
:1039900022c2af900576e0f52474012524540ff57a
:1039a00023900575e0652370057900121a02e5245d
:1039b00075f003a4f8a9f0740328f8740539f9e840
:1039c0002442f582e439f583eef0e82443f582e4fd
:1039d00039f583eff0e82444f582e439f583e521f5
:1039e000f0e523900576f0e522a2e092af7f040295
:1039f00023c2c082c08374fc122206e5a8f8c2afbd
:103a0000e5958532828533835392fef0e596c0e0da
:103a10007401122270d0e0f0e597c0e07402122227
:103a200070d0e0f0e8a2e7a2e792af740312227030
:103a3000e4f0853282853383122059740412221ceb
:103a4000d083d08222c0e0c0d075d018c092c0828e
:103a5000c083c0f0121b6a1239f290060a12206568
:103a6000e58955ab90060ef0e580900611f09006c2
:103a70000ee0f4f5899062d0e0f8a2e150279006bc
:103a80000ee0a2e5501f53abdf9062d0e0a2e0e46d
:103a900033900614f090060ee0c2e5f07b307a0019
:103aa000790612397d90060ee0600e7b007a00796f
:103ab0000612397d7900121b76c2c5d0f0d083d0b2
:103ac00082d092d0d0d0e032c0e0c0d075d008c053
:103ad00092c082c083c0f0121b6a1239f290060aab
:103ae000122065e58a558df890060ff0e590900656
:103af00012f0e8f4f58a7b017a00790612397d79b3
:103b000001121b76c2eb80b3c0e074f0122408905f
:103b100061a9e06017c2afe589f8e5abf975ab00c4
:103b2000e4f090624bf0888989abd2af900619e03f
:103b3000640f7012e5c7f8900368e0f5c790ff1caa
:103b4000e0f4f5ae88c7e5bbf8e5baf521e8fb90ef
:103b50000619e025e0f8e433f9741a28f5827406b2
:103b600039f583e521f0a3ebf0900619e02410fb72
:103b70007a00790612397de5a8f8c2af9004d4e046
:103b8000c2e2f0753400e8a2e7a2e792af7f02023a
:103b9000246fc0e0c0d075d018c092c0f0e5d1f855
:103ba00075d100c2c0a2e350097b037a00790412e8
:103bb000397dd0f0023ac1c0e0c0d075d010c092bb
:103bc000c021c022c082c083c0f05392fe90071073
:103bd000123cd2602a9006cbe0700c7401f07b009e
:103be0007a00790412397dee900710f0e5c1c0e04b
:103bf00074122521f582e43407f583d0e0800be5cb
:103c0000c4a2e650069006ca7401f0023cc1c0e0ae
:103c1000c0d075d010c092c021c022c082c083c065
:103c2000f0c2e95392fe9006cde0fa9006cce09afd
:103c3000543ff8602974ce2af582e43406f583e017
:103c4000f974012a543f9006cdf089c190070ee027
:103c50006870197b027a00790412397d800ee5a81c
:103c6000f8c2af9004d4e0c2e3123d408053c0e0fc
:103c7000c0d075d010c092c021c022c082c083c005
:103c8000f05392fe90079a123cd26029900755e0bb
:103c9000700b7401f07b00fa790412397dee900705
:103ca0009af0e5f9c0e0749c2521f582e43407f52b
:103cb00083d0e0800be5fba2e65006900754740128
:103cc000f0d0f0d083d082d022d021d092d0d0d0ea
:103cd000e032e0f52174012521543ffea3e06e227d
:103ce000c0e0c0d075d010c092c021c022c082c038
:103cf00083c0f0c2ea5392fe900757e0fa9007564d
:103d0000e09a543ff8602974582af582e43407f5a4
:103d100083e0f974012a543f900757f089f990071e
:103d200098e06870197b027a01790412397d800e5f
:103d3000e5a8f8c2af9004d4e0c2e4123d4080810f
:103d4000f0753400e8a2e7e433f9e8a2e792af2285
:103d50000306030202030302060203030105020233
:103d6000010001010101000003020000050002073b
:103d7000070002030101010806060503040401030c
:103d80000602020202010f000803050502070101f5
:103d90000901010201010200000003020201050500
:103da00002010103050001000301000000010104fc
:103db00004020302040104010074f012229e74f054
:103dc000122206e5c7f528900368e0f5c7752110b3
:103dd00075220078211224e67cdd7d037402122214
:103de0008c121cd2740212221c78211224e67c0050
:103df0007d007add7b03121cd8740212221c75210f
:103e000000805a852182a882e875f06fa4faabf091
:103e1000900365123f52246ef582e43bf583e0a2e5
:103e2000e050387f008f82ac82e875f037a4faab9f
:103e3000f09003d3123f522cfae43bfbea241af52c
:103e400082e43bf583e0fa74dd2cf582e43403f57b
:103e500083e04af00fefc3941040ca052190036439
:103e6000e0f8e521c398409b752100852182a88256
:103e700074dd1267253403f583e0fa8532828533d9
:103e800083e5821267253583f583e06af00521e535
:103e900021c3941040d5752100852182ae827f0018
:103ea000123f41a3a3a3a3a3a3a3a3e0f8123f41fe
:103eb000e048f52260778f27e522a2e0505c752369
:103ec000018f24e52778231221f3a82374dd2ef532
:103ed00082e43403f583e0586004790180027900bc
:103ee00074e52ef582e43403f583e0586004e9d2ea
:103ef000e1f98e238f24740378231221f38527257b
:103f0000e5232525fae43524fb74a02af58274f70d
:103f10003bf583e0fa7b00121b640527e522c313ff
:103f2000f522e527c394085004e522708b0521e5ae
:103f300021c394085003023e998528c77410024497
:103f400009853282853383e5822ef582e43583f557
:103f50008322123f5622e02afaa3e03bfbea2274b6
:103f6000f612229ee975f037a4faabf012130c900a
:103f700003d3126752e5c7ff900368e0f5c790f7d7
:103f80009e125c46e4c39af521741f9bf5227821aa
:103f90001224e67c007d00121cd8740212221c8fb1
:103fa000c779087cd57d037a007b0012182ee9645e
:103fb00008601b75210875220078211224e67c0018
:103fc0007d007ad57b03121cd8740212221c800e4d
:103fd0008532828533831224da740212221c7f0216
:103fe00002237674f012229e74fe1222371224d21b
:103ff0008a278b2812631e0592a38582218583223e
:10400000125c46ea4b60158e828f83a3a3a3858240
:1040100023858324c3e09aa3e09b500879011214fe
:10402000aa02410c05929007e51224f97b0705923c
:104030001263161219ba740412221c8e828f83a383
:10404000a3a3a3a38582258583268e828f83e01474
:10405000604a14606414602c14600d1470030240f4
:10406000f224fe607d02410c85238485248505921f
:104070001224fd8521828522830592124129121383
:104080006002410578251224e68523848524850570
:10409000921224fd12411612135480167825122410
:1040a000e685238485248505921224fd124116128b
:1040b000132a740412221c805a78251224e6ee2456
:1040c00017f584e43ff58505921224fd8523848548
:1040d00024851224fd124116121318740612221c94
:1040e0008031ee2417f582e43f127653e523452410
:1040f000700812412312135a801978231224e612f1
:104100004123121330740212221c8007aa27ab2805
:104110001217e00267dcee2415f582e43ff5830513
:1041200092e0f98521828522831259d7aa27ab28ec
:104130002274f612229e74fe1222371224d2eafe54
:10414000ebff89211263141219ae1247a4242a121c
:1041500052bbe060220592e024fd600c24fc701448
:10416000740765217011800c740a65216006740162
:1041700065217003752100e4439201f00592f090ef
:104180000363e0f522ac21eefaeffbe0f9121b2eff
:10419000900363e065226005a9221213f0023fd06c
:1041a00074f612229ee9ff8c218d22900363e0febb
:1041b00078211224e6740c122270e0fdeffc9003cb
:1041c00063e0f9121ae0740212221c900363e06e9d
:1041d0006005eef91213f0023fde74f212229e74b3
:1041e000fe1222371224d28a258b2612427b121904
:1041f000ae900363e0ff858482858583a385822357
:1042000085832478211224e6eefd7c0485238285b3
:104210002483124329121ae0740212221c900363b1
:10422000e06f6005eff91213f0e5842417f8e43528
:1042300085f988828983e02ef0a3e03400f07416bb
:104240006e701788828983c3e09416a3e0940040bf
:1042500009aa25ab261214a480197900852382852a
:104260002483125c461214aae40592f0aa25ab2618
:104270001217e0853282853383801c8c218d22e9e0
:10428000fe1258cc7b07900363e0fa790122853255
:10429000828533835392fe1224da740212221c7f29
:1042a0000602237674f412229e74fe122237122420
:1042b000d28a238b2412427b1219ae0592e0f87445
:1042c0000768700feef9ac21ad22aa23ab241214bb
:1042d000b6804d740a680592900363700fe0ffee9c
:1042e000fcaa21ab22e0f9121ae6801de0ff78213a
:1042f0001224e6eefd7c00858482858583a312432b
:1043000029121ae0740212221c900363e06f600508
:10431000eff91213f0e40592f0aa23ab241217e090
:104320008532828533830260bf127694900363e006
:10433000f92274f012229e74fe1222371224d274d3
:10434000fe1222068a278b288a828b83a3a3a3a32b
:10435000a3a3a3a3a3858225858326126314121920
:10436000ae852782852883a3a3e024faf52312478c
:10437000218525848526850592a385328285338310
:1043800005921246fb7e00804e900363e0ffe584b9
:104390002402f521e43585f52278211224e674fe05
:1043a00029fd7c03858482858583124329121ae0c6
:1043b000740212221c900363e06f6005eff9121380
:1043c000f0852582852683e0f5212efee5842521d2
:1043d000f584e43585f585852582852683e0f9ee2b
:1043e000c3952340a48921e523c395211246ec12ed
:1043f00047301214a40267d712221c8532828533fb
:10440000835392fe1224da740212221c7f080223c4
:104410007674f012229e74fe1222371224d274fe99
:104420001222068a238b24ea2409f8e43524126335
:10443000081219ae852382852483a3a3e024faf50c
:10444000221258c8858427858528e527242af582e5
:10445000e43528f5837401f0126784640170047eea
:104460000280027e107521008010e06f6005eff978
:104470001213f074022e2521f521e521c395225057
:104480005a5392fe900363e0ffa821853282853360
:104490008312622e3400f585eef52578251224ea84
:1044a000e5842403fce43585fd12451c0592900348
:1044b00063e0f9121af8740112221ce99003637088
:1044c000a9e06f6005eff91213f085278285288334
:1044d000e4f0aa23ab241217e0803e852221e521d7
:1044e00024fef8e434fff98e21e8c39521f8e9941d
:1044f00000f98532828533835392fe12616824016c
:10450000f8a3e03400f98527828528830592a31259
:104510005e02aa23ab241214a40267d70592a3e07b
:10452000faa3e0fb2274f012229e74fe12223712cc
:1045300024d274fe1222068a278b28ea2409f8e482
:1045400035281263081219ae852782852883a3a314
:10455000e024fbf52112526105929003d3125739e2
:10456000858225858326e525242af582e43526f5ee
:104570008374010592f07f00800de06e6005eef916
:104580001213f074042fffefc39521505beff885f1
:104590003284853385125deb85828485838505921f
:1045a000900363e0fe75220278221224eae52524b6
:1045b00017f523e43526f52478231224e612470a5a
:1045c000121af2740312221ce990036370ace06ebd
:1045d0006005eef91213f0852582852683e4f0aaa2
:1045e00027ab281217e0802ca821853282853383df
:1045f0001261623400f9e824fef582e934fff583a4
:10460000124747852582852683a3125e02aa27ab1f
:10461000281214a40267d774f012229e74fe12228c
:10462000371224d274fe1222068a278b288a828ba4
:1046300083a3a3a3a3a3a3a3a3a3858225858326e2
:104640008a828b83a3a3e024faf521126314121942
:10465000ae1247218532828533831246fb7f00806c
:1046600012e06e6005eef91213f08525828526832f
:10467000e02fff852582852683e0f8efc395215042
:1046800056e5252ffae43526fb8a828b83a38582a3
:1046900084858385900363e0fe74fc28f5227822ec
:1046a0001224eaea2405f523e43bf52478231224b6
:1046b000e612470a121af2740312221ce9900363ed
:1046c000709fe06e6005eef91213f0126d60aa277c
:1046d000ab281217e080128823e521c395231246e8
:1046e000eca3a31247301214a40267d7f895e0f99f
:1046f000e52528f582e52639f583221275f5242a69
:10470000f582e438f5837401f022858482858583ff
:10471000a3a3125745faa3e0fb0592900363e0f9c7
:1047200022125b04853282853383e8f0a3e9f0220c
:10473000a3124747853282853383126d56e8f0a372
:10474000e9f0aa27ab2822e02401f8a3e03400f91d
:104750002274f612229e74fe1222371224d21213f1
:10476000f0e970047a86801f1247a42416f584505d
:104770000205850592e0a2e040047a8180091217c3
:10478000daea4b70067a827b01800d0592e0c2e086
:10479000f012136c7a007b0085328285338353924a
:1047a000fe023fd61258cce5842274f212229e7487
:1047b000fe1222371224d2eafeebff8c258d261240
:1047c00013f0e970047a868012124b0860047a8133
:1047d00080091217daea4b70067a827b0180307406
:1047e00010122270e0f8c3941450048822800375dc
:1047f000221485252385262478231224e6a922ee77
:10480000fceffd12134e740212221c7a007b000290
:10481000428e74f012229e74fe1222371224d28a23
:10482000278b28ecff1213f0e970047a868025129a
:104830004b0860047a81801cefa2e04005c3940419
:1048400050047a80800e1217da8a258b26ea4526d4
:1048500070067a827b018034efc394165004effe19
:1048600080027e16740a1249961224f97b0705927b
:104870001263161219ba740412221ceef9ac27ad99
:1048800028aa25ab261213427a007b000243fb7450
:10489000f012229e74fe1222371224d28a258b2611
:1048a000ecfeedff7414122270e0f521c394135056
:1048b000191213f0e970047a868021124b08600403
:1048c0007a818018e525452670047a80800e1217bb
:1048d000da8a278b28ea452870067a827b01804d88
:1048e00074080592f0a3e525f0a3e526f09007e50e
:1048f0001224f97b0705921263161219ba74041276
:10490000221c741212227a05921224fd8e238f2407
:10491000059278231224e6a921ac25ad26aa27ab5f
:1049200028121336740412221c7a007b000243fb07
:1049300074f412229e74fe1222371224d28a22129a
:1049400013f0e970047a86801a124b0860047a81a9
:1049500080111217da8a238b24ae23af24ee4f7016
:10496000067a827b01802c74091249961224f97b05
:104970000705921263161219ba740412221ce5225a
:104980006004790180027900eefaeffb12133c7aa1
:10499000007b000260b60592f0a3e4f0a3f090075c
:1049a000e52274f012229e74fe1222371224d2eafb
:1049b000feebff8c278d281213f0e970047a8680b5
:1049c0001f124b0860047a818016ee4f70047a80c3
:1049d000800e1217da8a258b26ea452670067a821f
:1049e0007b0180547412122270e0f8c394145004b6
:1049f0008821800375211474060592f0a3eef0a3bc
:104a0000eff09007e51224f97b0705921263161266
:104a100019ba740412221c852723852824782312ae
:104a200024e6a921eefceffdaa25ab26121348745b
:104a30000212221c7a007b000243fb74f412229eb5
:104a400074fe1222371224d2eafeebff1213f0e9b1
:104a500070047a86801a124b0860047a818011ee05
:104a60004f70047a8080091217daea4b70067a8256
:104a70007b01802a7407124b03eef0a3eff08584cc
:104a800082858583a3a3a3eef0a3eff0e58424172a
:104a90001252bbe4f0a3f01214a47a007b0002606f
:104aa000b674f412229e74fe1222371224d2eafe49
:104ab000ebff1213f0e970047a86801a124b08603b
:104ac000047a818011ee4f70047a8080091217da1f
:104ad000ea4b70067a827b0180267405124b03a391
:104ae000a3a882a983eef0a3eff0888289831255f0
:104af000830592a3e8f0a3e9f01214a47a007b00e6
:104b00000260b6124c6ca3221258cc0592e02274bb
:104b1000f212229e74fe1222371224d28a218b2294
:104b2000ecfeedff1213f0e970047a868012124b4e
:104b30000860047a8180091217daea4b70067a82db
:104b40007b01801d7404124b03e521f0a3e522f0e4
:104b50000592a3a3a3eef0a3eff01214a47a007bb6
:104b60000002428e74f012229e74fe12223712242a
:104b7000d28a278b288c258d261213f0e970047aaf
:104b800086802e124b0860047a81802574141222cc
:104b9000700592e0ff74026f600974106f60047a10
:104ba00080800e1217da8a238b24ea452470067a55
:104bb000827b01803474030592f08f2175220005f9
:104bc0009278211224e67414122270124c95121c51
:104bd000d2740212221c124c78858482858583123d
:104be0004c861214a47a007b000243fb74f012225c
:104bf0009e74fe1222371224d28a278b288c258d90
:104c0000261213f0e970047a86802e124b08600495
:104c10007a81802574141222700592e0ff74026f6d
:104c2000600974106f60047a80800e1217da8a238c
:104c30008b24ea452470067a827b01802c8f2175b3
:104c4000220078211224e67414122270124c95125c
:104c50001cd2740212221c124c787401124c6c1279
:104c60004c861214a47a007b000243fb0592f08567
:104c70008482858583059222e5842415f582e435b6
:104c800085f583eff022124d4ae525f0a3e526f0e5
:104c9000aa23ab24221259d7e5842405fae43585ea
:104ca000fb2274f012229e74fe1222371224d28a42
:104cb000278b288c218d221213f0e970047a8680cc
:104cc00029124b0860047a81802074161222700524
:104cd00092e0ffc3941140047a80800e1217da8aa2
:104ce000258b26ea452670067a827b01805974124c
:104cf000122270125583e5842417f582e43585125b
:104d00005e0074020592f0e58424151252bbef0593
:104d100092f08f2375240078231224e67416122251
:104d200070124c95121cd2740212221c858482854a
:104d30008583124d4ae521f0a3e522f0aa25ab2692
:104d40001214a47a007b000243fba3e527f0a3e53d
:104d500028f00592a3a3a32274f112229e74fe12de
:104d600022371224d274fc1222067402122270120c
:104d70006752e5c7f527900368e0f5c77402122271
:104d800070127604853284853385e5820592f0a31e
:104d9000e583f0853282853383059212678afa743f
:104da000021222700592e02a124eee059290f79db3
:104db000e0f525ff741dc39af5268e228e2180080a
:104dc0000522efc313ff052190f79ce0fce521c30a
:104dd0009c5043eec39526503d124eff70e8efa263
:104de000e050dfa3a3a3a3a3e0640270d375230262
:104df00075240078231224e61259cce5842ef8e4b9
:104e00003585f9e82402fae439fb121cd274021247
:104e1000221c0e0e80acee6013858482858583a3f0
:104e2000ef6004740280027403124ed7e52270030f
:104e3000024ecf8532828533835392fe12678af801
:104e4000741dc398fa95e0fbc3ea9410eb9400a29a
:104e5000d265d033407974021222700592e0281294
:104e60004eeeaf258e218006efc313ff0521e5210d
:104e7000c39c5041e526603d5392fe124eff70ecfc
:104e8000efa2e050e3a3a3a3a3a3e0641070d9753d
:104e900023108e2478231224e61259cce5842402b0
:104ea000fae43585fb121cd2740212221c7e1074a7
:104eb000ff2522600e8584828585835392fea3742c
:104ec000068009858482858583a37407124ed78561
:104ed00027c77404026e6bf074012ef80592f00877
:104ee000853282853383059212678e28f022f584fd
:104ef000a3e03400f5850592a3a3a3a37e0022902e
:104f0000f796127640e52175f006a4faabf0e82a90
:104f1000fae93bfb8a828b83e02274f012229e74b2
:104f2000fe1222371224d274f912220685328285ab
:104f30003383ecf0a3edf08a278b28e9fe7522007d
:104f4000126d608a828b830592a3a3a3a38582231b
:104f500085832474026e600caa23ab241219eae93b
:104f600060027e02741912227012620f7410059290
:104f7000f074026e6003024ffe8523828524830550
:104f800092125583e8700374286970567f00741973
:104f900012227012620f740a0592f0e5c7c0e07425
:104fa00004122270d0e00592f0900368e0f5c71279
:104fb0006d60059290f79ce0f526f582ac8285271e
:104fc00082852883126e62500302513985278285bb
:104fd0002883a3a3125c46c3ec9ae49b50258c253e
:104fe0008024740168700374286970047f01809eb6
:104ff000740368700374286970047f0280907900dc
:10500000025146eaf525e814f521801274021222b5
:1050100070127601e521f0a3e4f015210521e521c8
:10502000c39525400302512a12558074051222703f
:10503000125e02852182a8827900e875f006a4fa42
:10504000abf0740512227a0592e02af582a3e03bc8
:10505000f583ac82ad830592e06f70c0852282aa91
:10506000828532848533850592e02a12572d740299
:1050700012227ae5820592f0a3e583126cf8e0240f
:1050800004f527126784f5236009e527652360038b
:1050900002512a852723ea126ce6400302512ae5d1
:1050a00027f0eaf522e824010850010974021222cf
:1050b00070059212620fe80592f0a3e9126cf812e3
:1050c00059c31224e68c828d83a3a3a31275fb120d
:1050d0002270126d20121cd2740212221c8029e54b
:1050e0002175f006a4f8a9f074051222705392feff
:1050f000125e08f8700302500c74016870030250cd
:105100000ce86f700302500c0521e521c395264081
:10511000cee5266521600302500c74021222701243
:10512000760174fff0a3f002501ce522600b7419a5
:105130001222705392fe126d667404122270539202
:10514000fee0f5c7a92274070243f874f712229e05
:1051500074fe1222371224d21242811219ae059225
:10516000e0f8740668600a7408686005740968707d
:105170001ce41252b27c0012451c0592e0f9121b8d
:105180002e900363e06e6005eef91213f00261e306
:1051900074f212229e74fe1222371224d28a258bb8
:1051a00026ecffedfeec24010ce43400fd12131e8e
:1051b0008a848b8574101222701259d3ec4d701da5
:1051c000eff9121594e9fec3941540027e147d0098
:1051d000eefceff9aa84ab851215ac801aeec394ed
:1051e0001540027e148e2175220078211224e612c9
:1051f0001cd2740212221ceef9aa25ab261213242b
:105200000242738532828533830261ec74f7122285
:105210009e74fe1222371224d28a848b8512524e3b
:1052200060237b081263161219ae12524efae4f094
:10523000900363e0fef9121aec900363e06e6005e0
:10524000eef91213f0aa84ab851217e080b5125262
:10525000619003d3e028f8a3e039f9e8126f88e001
:10526000221252652212526922900363e075f037d0
:10527000a4f8a9f02274f712229e74fe12223712ab
:1052800024d2124b08640b6026e58424191252bb09
:1052900074010592f01258c8740b05921252b2f9bb
:1052a000121b28900363e06e6005eef91213f00202
:1052b00061e3f00592900363e0fe22f582e4358518
:1052c000f5832274f012229e74fe1222371224d229
:1052d00074fd1222067401122270ecf0a3edf08925
:1052e000258a228b277a817b01e52275f006a4f8b6
:1052f000a9f090f796126b1af5850592a3a3a3e087
:10530000f582a3e0f583858284858385a3e08532d9
:1053100084853385f00592e0f52875210074ff65da
:1053200025600785252180020521900364e0f8e5ca
:1053300021c3984003025455852182a882e875f064
:105340006fa4fcadf0900365125591e584246e12b4
:1053500052bbe0a2e050d1e8900363f0900361e516
:1053600084f0a3e585f0853282853383e01313133f
:10537000541ffee05407f526e528a2e4503de8124c
:10538000545af8ed39f91260cca826b8000280040e
:10539000c313d8fca2e050231217daea4b60617401
:1053a0000112227a05921224fdad27ac22791b123c
:1053b0001534740212221c7a007b00e528a2e54015
:1053c0000302544c900363e012545afced39fdec97
:1053d0002422f582e43df583e0ac26bc0002800483
:1053e000c313dcfca2e0506412525160047a818045
:1053f000111217da8a238b24ae23af24ee4f7006e6
:105400007a827b01804f05929007e51224f97b0890
:1054100005921263161219ba740412221c74012523
:1054200022c0e01260d7126f88d0e0f0740112221f
:105430007a05921224fdad27ac22791deefaeffb1e
:10544000121534740212221c7a007b0074ff652549
:10545000700302532874030267d975f037a4f8a9c2
:10546000f09003d3e02efca3e03400fdec2822747e
:10547000f012229e74fe1222371224d289218c2728
:105480008d287522007412122270e0fea3e0ff8eb8
:10549000828f83e0f525e5c7f524125754f5269051
:1054a000f79ce0f8e526c39840097522018e828fab
:1054b000838023e526125c2670098524c77a887bc1
:1054c000018049a926121594e98e828f83f0c39535
:1054d000215007752207e4f08022a821e0c398f04c
:1054e000f8c39525500488238003852523e523f000
:1054f000ad21fca926aa27ab281215ac8524c7e547
:10550000226005fa7b0480047a007b000243fb746e
:10551000f612229e74fe1222371224d2eaf8ecfa16
:10552000edfb752100e5c7fe900368e0f5c7e814c0
:10553000fd740c12227012558390f79ce0fcedc3b1
:105540009c400b75210188828983e4f0801eed1256
:1055500055870592e0fca2e75004741080027402a3
:10556000888289830592f0ecf91219f68ec7e5213d
:10557000a2e05005fa7b0480047a007b00023fd051
:1055800090f7961276402275f006a4fcadf090f7e5
:1055900096e02cf584a3e03df5852274f612229e58
:1055a000e9ffeaf8ebf9e5c7fe900368e0f5c77498
:1055b0000a122270e0fbc3941540067a807b0180ba
:1055c0001690f79ce0c398e49950067a017b04801a
:1055d000061aeff91215468ec7023fde74f012224a
:1055e0009e74fe1222371224d274fe1222068532d5
:1055f00082853383ecf0a3edf089257e0012574eaf
:10560000f52290f79ce0c39522500302571ee52235
:1056100075f006a4f8a9f0059290f796125739850f
:1056200082278583280592a3a3e0fc24fa600a144c
:10563000600724fb600302571c7414122270e0f50b
:1056400021740c6c70030257028527848528850518
:1056500092a3a3a3e0f582a3e0f583852584aa8421
:10566000858284858385a3a3a3a3e0f8852123ea0b
:105670002523f523e43400f524e89523e49524c399
:1056800065d03350057e0d02571f0592a3a3858276
:1056900084858385852182a882790074066c88239d
:1056a00089247823701b1224e67402122270125788
:1056b00040faa3e03400fb121cd2740212221c80b8
:1056c000311224e6740212227012574012572daa8a
:1056d00082ab83121cd2740212221ce5212525c044
:1056e000e0852782852883a3a3a3126799d0e005cc
:1056f00092f08527828528835392fea3a3e0640c51
:10570000700b8532828533831259d380047c007def
:1057100000ab21aa2279ff12154680050e0e0e7fde
:10572000048526c7eefaeffb74020243f8f582a364
:10573000e03400f5830592a322125df539f583224a
:105740001257452a22e0fca3e0fd0592e0227f00eb
:10575000e5c7f526900368e0f5c7ea142274f41251
:10576000229e74fe1222371224d28c848d85e9ff8a
:10577000e5c7f521125754fe90f79ce0c39e5004f4
:1057800079018034740e122270e0f52260047a02ee
:1057900080027a80eef912158ee9701ce4f523f58b
:1057a0002478231224e6ad22effcaa84ab85eef91f
:1057b0001215a6740212221c8521c702432074f31d
:1057c00012229e74fe1222371224d28a218b2212b8
:1057d00058c88a828b83a3a3a3a3a3a3a3a3a3e0f4
:1057e000700f1259dd1215faea4b60781217e0803b
:1057f000f1e5c7fe900368e0f5c7e584242bf523a7
:10580000e43585f524852382852483126302605262
:1058100088828983a3a3a3a3a3a3a3a3a3aa82abe0
:1058200083e0ff8a848b850592a3a31224fd7d016a
:10583000888289830592a3a3e024f7fcea2404fa72
:1058400050010b74ff2ff91215a6740212221ce9e5
:10585000f525aa23ab241215fa1217e0e525702ec0
:1058600080a38ec7852182852283a3a37405f0853a
:105870002182852283a3a3a3a3a3a3a3a37419f0c6
:105880007900aa21ab22121324802a1217e01259a0
:10589000dd1215faea4b70f3e525f523782312247f
:1058a000ea8f23ac237d007918aa21ab221213784a
:1058b000740112221c8532828533831224da740229
:1058c00012221c7f050223761258cc2212526590b8
:1058d00003d31258d622e028f584a3e039f58522b7
:1058e00074f412229e74fe1222371224d28a848b00
:1058f00085858482858583a3a3a3a3a3a3a3a3a350
:10590000ae82af83e5c7f521900368e0f5c78e82cc
:105910008f83e014f990f79ce0c39950217401f54e
:105920002178211224ea8e828f831259d37916aa04
:1059300084ab85121378740112221c0243207a0270
:1059400012158ee970d91217da8a238b24ae23af91
:1059500024ee4f8521c7700c7a017b0090032e74d2
:1059600008022118ac84ad851259dd121600858419
:1059700082858583a3a38582218583221259c31240
:1059800024e6e5842404fce43585fdee2404fae4f1
:105990003ffb121cd2740212221c852182852283b5
:1059a000e08e828f83a3a3f08e828f83a3a3a3a311
:1059b000a3a3a3a37417f07900eefaeffb1213244c
:1059c00002593be0f5237524007823228a828b83d9
:1059d000a3a3a31259d722e0fca3e0fd221260dbaf
:1059e000242bfae439fb2274f112229e74fe122257
:1059f000371224d274fb122206740312227012672b
:105a0000528927ecfeed125aff7401122270125ec9
:105a100002e5c7f521900368e0f5c78e828f83a366
:105a2000a3e0f8ee1267253ff583a3a3a3a3858225
:105a300025858326741bc398f5228025e9c522c3da
:105a40009522f5228e828f83a3a3e029f0e52529f4
:105a5000f525e43526f5267401122270125afa044f
:105a6000f07401122270125afafac395275071e5a8
:105a700022606da832a9338823892478231224e672
:105a800085252385262478231224e6a9227c007dff
:105a900000ea2afae433fb7407122270125e11fa4c
:105aa000a3e0fb12157c740412221c85328285331c
:105ab00083e06088853284853385059212250174e0
:105ac00004122270059212678afca3e0fd790eeea3
:105ad000faeffb121378740112221c8521c7800c87
:105ae0008521c77900eefaeffb1213247405122208
:105af0001c853282853383026e7712761de022ff89
:105b0000125b0422125b08221252699003d3e02830
:105b1000f8a3e039f92274f012229e74fe122237a3
:105b20001224d28c218d22e9fe12574ef5257414d1
:105b3000122270e0f527a3e0f52890f79ce0c395ca
:105b400025500b8527828528837401025bfd7a012d
:105b5000a92512158ee9852782852883f060030226
:105b60005c1e852582aa827b00ea125c267077057e
:105b7000921258c8a884a985126734705e741212f4
:105b800022701259d3e82434f582e439f583ecf01d
:105b9000a3edf0e82436f582e439f583eef09003c6
:105ba00063e0ffeef52378231224eaac21ad22ea6c
:105bb00024010a50010b900363e0f9121afe7401ec
:105bc00012221c900363e06f6005eff91213f07a64
:105bd000017b009003a0740802211812673f8527fb
:105be000828528838017a925121594e9ffc3952182
:105bf000e49522500b8527828528837407f0801e48
:105c0000e521cfc39fffeec39f5002eeffad21ef12
:105c1000fca9257412122270125c461215ac85265e
:105c2000c7eff90267dc75f006a4f8a9f090f796c3
:105c300012616da3e0640c22858482858583e02453
:105c4000f9f98e828f831276942274f112229e7457
:105c5000fe1222371224d274f812220612674c74f4
:105c600006122270ecf0a3edf089277f00e5c7f55e
:105c700026126d05f522126d2a5003025de1126da8
:105c80004150048c218003eaf521e814fe8532821c
:105c9000853383127613740412227ae5820592f01a
:105ca000a3e583f08013888489850592e0f8a3e05a
:105cb000f9e80592f0a3e9f00eeec3952140030246
:105cc0005de15392fe1255807402122270125e0240
:105cd000ee75f006a4f8a9f07402122270125e08a4
:105ce000f525a2e7500b126aff1221f3126b1f80f9
:105cf00003126b0df585eaf52378231224eaac84b0
:105d0000ad8579027405122270125c461219f07486
:105d10000112221ce960a17a01eef912158ee970d8
:105d200097ac27853282853383e02406faa3e034da
:105d300000fbeef9121588e97003025cb8eff87405
:105d40000612227a125deba882a983efc394124057
:105d500003025de174042fff8e23e5232401fae49e
:105d60003400fbea05921267538017ee75f006a423
:105d7000faabf074021222705392fe125e11652586
:105d8000601c0eeec3952240e2e5226e7010888200
:105d900089835392fea3a374fff0a3025cb71e7421
:105da000041222705392fe12678afaa3e0fb8882e3
:105db00089830592a3a3ea700374286b60177401aa
:105dc0006a700374286b600d74036a700374286b27
:105dd0006003025ca6ee2401f8e43400f9e8025cfa
:105de000b48526c7eff97408026e6b0592125df553
:105df0003400f58322e028f582a3e022f582e43a1c
:105e0000f583e8f0a3e9f022125e0c22126172e041
:105e100022125e180592e022e02af584a3e03bf509
:105e2000852274f412229e74fe1222371224d2e9c3
:105e3000ffecfeef126214fc8e82a88279006039ba
:105e400014603614603314603014606214700302fe
:105e50005eec147003025f4d147003025f9b1470bc
:105e600003025fe914700302605714700302609c20
:105e7000147003025f4d0260b6ec6e60030260b600
:105e80008821892278211224e6eafcebfde58424ae
:105e900003fae43585fb121ccc740212221c8b22ff
:105ea000ea452270047901800279000260b6858497
:105eb00082858583a3a3a3a3a3e06e60030260b6db
:105ec0008821892278211224e6eafcebfd0592a3c1
:105ed000a312451e121ccc740212221c8b22ea450e
:105ee0002270047901800279000260b60592a3a3b2
:105ef000a3e0fca2e75004781080027802e86e600c
:105f0000030260b6eca2e7501b547ff5218922748e
:105f10000478211221f390f798e02521f582a3e07f
:105f20003522800c2cf8e433f990f79a125df5399c
:105f3000f583ac82ad83eef521059278211224ea37
:105f4000eef91219f0740112221c0260b60592a338
:105f5000a3a3e0f523a3e0f524852382f58305922e
:105f6000a3a3a3a3e06e60030260b6882189227810
:105f7000211224e6eafcebfd852382852483a3a37a
:105f8000125c46121ccc740212221c8b22ea45229f
:105f900070047901800279000260b60592a3a3a380
:105fa000e0f523a3e0852382f5830592a3a312677e
:105fb0008a6e60030260b6882189220592782112d8
:105fc00024e6eafcebfd858482858583a3aa82ab67
:105fd00083121ccc740212221c8b22ea452270040c
:105fe0007901800279000260b674026e600302607b
:105ff000b60592a3a3a3a3e0fc131313541ff5212a
:1060000005921260d72521f8e439f974075cf5216f
:106010001260ccac21bc00028004c313dcfca2e003
:106020005004d2f08002c2f0a2f0e433fc12672ade
:10603000e0a821b800028004c313d8fca2e05004f9
:106040007802800278008a828b83ec48f8e06870de
:1060500002a3e0705f805974026e705a0592a3a388
:10606000a3a3e0fc8a828b83131313541ff874d507
:1060700028f584e43403f585e0c0e074075cf8d0cb
:10608000e0b800028004c313d8fca2e0e433f805b2
:1060900092e0687002a3e0701d09801a74016e70ae
:1060a000158a828b83e0f521121432e96521700490
:1060b0007901800279008532828533835392fe1202
:1060c00024da740212221c7f04022376e8241af5d3
:1060d00082e439f583e0221260db22125b08e822b9
:1060e00074f712229e74fe1222371224d2e975f040
:1060f00006a4f8a9f090f796126168f874016a7026
:1061000009e8a2e040507902805274026a7039e8ce
:10611000a2e1503ea2e450420592900363e075f084
:10612000e6a4f8a9f090045e12616239f9e824113e
:10613000f582e439f583e0a2e75009900361126724
:106140008af470167905801474806a700de8a2e7ed
:1061500040c279038006a2e340be79000261e39069
:106160000365e028f8a3e02212616de0221261725b
:10617000a3221258d605922274f712229e74fe12a0
:1061800022371224d2126213f96058146055146039
:106190005214604f14601714601d14602814602d91
:1061a000146036146033146034146019803305921f
:1061b000a3a3a3a3a3801e0592a3a3a3e0a2e750d9
:1061c000187910801e1261f9a3a3e080091261f909
:1061d00012620f0592e0f9800a7902800679018047
:1061e0000279008532828533835392fe1224da7459
:1061f0000212221c7f010223761261fea322059265
:10620000a3a3a3e0f8a3e0f58388820592a322125a
:1062100067a022e975f006a4f8a9f090f79612623b
:106220002e39f585858482858583a3a3e022e02825
:10623000f584a3e02274f012229e74fe122237121b
:1062400024d28a228c278d288b251213f0e970071f
:106250007a867b010262ff12631eee2431f584e42c
:106260003ff5858584828585830592e0600302621f
:10627000fbee242df582e43ff583126302607c85fa
:1062800084828585837401f0ee2432f582e43ff543
:1062900083e522f0705dee2436f584e43ff5850554
:1062a00092e0f8e525c398500585252180028821d4
:1062b000e521f0f523752400059278231224e6ac3d
:1062c00027ad28ee2434f582e43ff583125c4612b4
:1062d0001cd2740212221c0592e0f8ee242ff582e3
:1062e000e43ff5830592e0f9a3e0f5838982a3a357
:1062f000e028f07b0912631612397d7a007b0002d8
:1063000067dc127640e84922f9853282853383e8da
:10631000f0a3e9f07b07900363e0fa7901221267aa
:10632000c5ae82af832274f712229e74fe1222370a
:106330001224d2eaff1213f0e970067a867b0180fc
:10634000421267bc2431f8e43bf9888289830592c4
:10635000e0702cea242df584e43bf5850592e0f805
:10636000a3e0f9e849601874010592f0ea2432f5d7
:1063700082e43bf583eff07b0912631612397d7ad4
:10638000007b000261e374f012229e74fe12223739
:106390001224d274fb1222067404122270e9f074e3
:1063a00001122270126752ec853282853383f074b9
:1063b00003122270edf01267bcf8ebf9740412229c
:1063c000700592e0fc2401f525e43400f526ec127a
:1063d0005587858427858528853282853383e0fe2d
:1063e0007f007417122270127655ee2523f521e4f2
:1063f0003524f522852782852883a3a3e024fa701b
:106400000302648d1470030264d61470030265489d
:106410001470030266161470030266991460651402
:1064200060030266d37403122270e070030266e216
:106430001267347048900363e0fe740112227a05fb
:10644000921224fd059278231224e674041222701d
:10645000e0fd7c02aa25ab26900363e0f9121b0441
:10646000740412221c900363e06e6005eef91213af
:10647000f07a017b009003a0740802211812673f94
:10648000f9026720121432e970030266ba85278286
:10649000852883a3a3a31267a8600dc3e52398e50d
:1064a0002494004003026633c3e89521e49522500a
:1064b000030266a48e218f2278211224e67403122f
:1064c0002270126779faa3e03524fb121cd2740201
:1064d00012221c0266d3852782852883a3a3a38565
:1064e00082278583281267a8600dc3e52398e524d9
:1064f00094004003026633c3e89521e495225003db
:106500000266a48e218f2278211224e674031222bf
:1065100070126779f582a3e03524f5830592a3aa6a
:1065200082ab83121cd2740212221c853282853304
:1065300083e0a82328c0e0852782852883126799f5
:10654000d0e00592f00266d3853282853383e07015
:106550000302671ee5234524600ec3e5239402e58c
:106560002494004003026633c3e5219403e522949a
:106570000040030266a4740165234524700b740176
:1065800012227012676fe080087401122270126785
:106590008a126758ea28f8e43bf9e8241af584e4fb
:1065a00039f58574075df87401b800028004c333bf
:1065b000d8fcf8eca2e050060592e0488007e8f429
:1065c000f80592e058f00592e0fe131313541ffaf9
:1065d0001260d72af8e439f912672a74075ef87452
:1065e00001b800028004c333d8fcf8eca2e15004e7
:1065f000e0488005e8f4f8e058f090036112678afb
:10660000fe74ff6e600a126f91eefb7a8812181604
:1066100012149802671e853282853383e07003026c
:10662000671ee52345246010c3e5239402e5249406
:106630000040057907026720c3e5219403e5229411
:10664000005061740165234524700b74011222709f
:1066500012676fe08008740112227012678a126755
:106660005874d51267253403f58374075df87401f7
:10667000b800028004c333d8fcf8eca2e05004e078
:10668000488005e8f4f8e058f079087cd57d037a75
:10669000007b0012181602671ec3e5219402e52252
:1066a00094004004790d8078853282853383e060e0
:1066b0006d12186ae9c39402400479038062740180
:1066c00012227012678a60047901800279007affd1
:1066d00012146e74031222705392fee060047c0068
:1066e00080027c01900363e0fe740112227a05921d
:1066f0001224fd059278231224e67404122270e01d
:10670000fdaa25ab26900363e0f9121b0474041262
:10671000221c900363e06e6005eef91213f079001d
:1067200074050267d928f582e422e82422f582e480
:1067300039f58322e82431f582e439f583e022e457
:10674000f0e82432f582e439f583e022853282854f
:106750003383eaf0a3ebf022fc852782852883535c
:1067600092fea3a3a3a3e0fd131313541ff822e08a
:10677000f8a3e0f5838882a3221259d70592a3a338
:10678000e025232285328285338312678e22e0f54d
:1067900084a3e0f5850592e0221276081267a02214
:1067a000e0f584a3e0f585221267a08584828585c3
:1067b00083a3a3a3a3e0f8e5234524221267c5aa77
:1067c00082ab83ea2212526505929003d3e028f54a
:1067d00082a3e039f58322740212221c853282855d
:1067e000338302440474f112229e74fe1222371283
:1067f00024d274fe1222068a238b24ecfe8d2512ed
:106800006213ff8d82aa82ea2dfce433fd8e82a8fa
:1068100082ef603314603014602d14602a14604ecf
:106820001460741470030268aa1470030268d5140b
:1068300070030268fe1470030269bc147003026adc
:1068400034146066026a3fef9e50068f82ac8280ed
:1068500002e8fc7d008c218d2278211224e6e5845b
:106860002af8e43585f9e82403fce439806485845a
:1068700082858583a3a3a3a3a3e0fc9e4002e8fc3a
:106880007d008c218d2278211224e60592a3a3a3fa
:10689000e02afca3e08039ad25eefc0592a3a3a37a
:1068a000e0f9aa231219fc026a3f126a44a3a3e08a
:1068b000ff9e50078f8285822180028821752200e9
:1068c00078211224e68c828d83a3a3e02afca3e026
:1068d0003400fd8024126a4412678afc9e4002e85c
:1068e000fc7d008c218d22059278211224e6e5841e
:1068f0002a1252bba3ac82ad83aa23026a2a059254
:10690000a3a3a3a3aa84ab858a828b830592e0ff0d
:10691000900363e075f037a4f52185f027e527f5ae
:10692000229003d3e02521f584a3e03522f585effd
:10693000131313541ff521e5842521f521e4358532
:10694000f522e521241af582e43522f583e0c0e042
:1069500074075fffd0e0bf00028004c313dffca216
:10696000e05004d2f08002c2f0a2f0e4338532821b
:10697000853383f0a3e4f08a828b83126a57e5841f
:106980002afae43585fbea2422f582e43bf583e02c
:10699000c0e074075ffad0e0ba00028004c313dae3
:1069a000fca2e050047a0280027a008532828533ac
:1069b00083e04af0eec394034052804c0592a3a3b7
:1069c000a3a3aa84ab858a828b830592126a57742b
:1069d000d52af582e43403f583e0c0e074075ffa5a
:1069e000d0e0ba00028004c313dafca2e05004d263
:1069f000f08002c2f0a2f0e433853282853383f066
:106a0000a3e4f0ee940340047a028002e8fa7b00eb
:106a10008a218b2278211224e67402122270e582e8
:106a20002cfce5833dfdaa23ab24121cd274021278
:106a3000221c800b121432e9852382852483f07492
:106a400002025aee0592a3a3a3e0fca3e0fd8c8210
:106a50008d830592a3a322e0ff131313541ffa2280
:106a600074f212229e74fe1222371224d274fe1285
:106a7000220612674c8c258d26e9ff752100e5c79b
:106a8000f522900368e0f5c77e0080010e90f79c28
:106a9000e0f8eec398505bee126d10500b126affd7
:106aa0001221f3126b1f8003126b0df585eaf5239b
:106ab00078231224eaac84ad857902740112228c09
:106ac0001219f0740112221ce960c1eef91215943a
:106ad000e9f8efc39850048f23800288237d00ac2f
:106ae00023eef9aa25ab261215aceef9121594e99e
:106af000f5218522c7a921740212221c0242737a51
:106b000010547ff52375240074047823227a02251b
:106b1000e0f8e433f9059290f79a12622e392205d3
:106b20009290f798e02523f584a3e035242274f0b1
:106b300012229e74fe1222371224d274fb122206f5
:106b400012674ce9125aff7403122270125e028c13
:106b5000848d850592a3a37405126cf8a3a3a37476
:106b600009f00592e0f8ec1267253df5830592a344
:106b7000a3a3a3858225858326858482858583e0da
:106b800004f075210074026f6022eff9853282856e
:106b90003383126d201219eae960117f0274031227
:106ba0002270127629127604e024f2f0e5c7c0e0e4
:106bb0007402122270d0e0f0126d05126d2a50039b
:106bc000026ccc126d4150048c228003eaf52274d1
:106bd00003122270e0faa3e0ca2433f582e43af506
:106be00083e0fe7052e814fe852582852683e4f05a
:106bf0008045eaf0c3941640037415f0e52528faa1
:106c0000e43526fbe5272401f8e43400f98a828b79
:106c100083a3125e027d00852582852683e0fcee3b
:106c2000f9ea2403fa50010b1215ac85258285265a
:106c300083e02521f5210eeec395224003026ccca2
:106c40008e82858227e527126d10500b126aff1283
:106c500021f3126b1f8003126b0df585eaf5237883
:106c6000231224eaac84ad85eff97401122270126c
:106c70006d201219f0740112221ce960b97a01ee3c
:106c8000f912158e741712227012620fe90592f034
:106c90006010e521603674171222700592126d663d
:106ca000802aeef9121594e9fa0a0a852182a8824f
:106cb000852582852683e0f5237003026bf2ea6561
:106cc000237009e8126ce65003026bfc7402122276
:106cd000705392fee0f5c77403122270127619ee1b
:106ce000f0a9210267202523fae43400fbea941678
:106cf000eb9400c365d03322f08c828d830592a380
:106d0000a3a3a3a322900368e0f5c790f79ce02219
:106d100075f006a4f8a9f090f796125e0ca2e7228f
:106d2000e02404faa3e03400fb22f582ac82853231
:106d30008285338312678ef8a3e0f9c3ec98e49957
:106d4000228532828533830592126d56a312769482
:106d5000c3ec9ae49b22e0faa3e0f5838a82a322a3
:106d60008532828533831267a0e40592f02274f1a4
:106d700012229e74fe1222371224d28a848b858cb2
:106d8000258d267e008c828d83e4f0e5c7f52712e1
:106d90006d05ff8f82ac82858482858583126e6249
:106da0005003026e5b0592a312451ec3ec9ae49b4e
:106db00050048f238003eaf523e814ff8029e5259a
:106dc0002afae43526fbe824015001098a828b83e4
:106dd000a3125e03ecf9ea2403fa50010b1219f630
:106de000740225242efe0fefc39523506e8f82a8c8
:106df000827900e875f006a4faabf05392fe90f7a2
:106e000096125e11fc8525828526830592e0faecb8
:106e1000a2e7500f752410ea600574026a703c7492
:106e200002800d752402ea600574016a702d7401f8
:106e3000f08e82aa82852421ea2521f521e43400fe
:106e4000f522e521240250020522c39416e522947e
:106e500000a2d265d0335003026dbe8527c7eef97c
:106e6000800c127640c3ec98e4992212221c8532e1
:106e7000828533835392fe1224da740212221c7f1d
:106e80000702237674f212229e74fe122237122415
:106e9000d289218982a882e875f037a4feaff0ea92
:106ea00024fe605a24fe6003026f61126f6488231f
:106eb000892412615f3524f9900361125e02752501
:106ec0003775260078251224e67c007d009003d3d8
:106ed000e02efaa3e03ffb121cd8740212221c9091
:106ee0000365126b24f5850592e0f46074126f91ce
:106ef00090036112678afb7a8812182e8060126fe5
:106f00006412615f39f9900361125e027b07aa2166
:106f100079011219ae126f81e060137b08aa217902
:106f2000011219ae126f81e4f080031217e0126fa4
:106f300071242bfae439fb1215faea4b70ed752334
:106f40001075240078231224e67c007d00126f71f6
:106f5000241afae439fb121cd8740212221c1214ef
:106f60009802428ee8900363f075f06fa4f8a9f0e0
:106f700022126f75229003d3e02ef8a3e03ff9e8c8
:106f800022126f75126f88222419f582e439f58375
:106f90002279100592900363e075f037a4faabf004
:106fa0009003d3123f56241afce43bfd22c3ec9a13
:106fb000ed9b4004ea4b7004790180027900539202
:106fc000fe02112974f012229e74fe12223712243e
:106fd000d274f71222067401122270126752125be9
:106fe000007405122270125e027a0074011222707f
:106ff00012630270100a7405122270127639ea12b6
:107000002270125e02752300752400740112227032
:107010001275f12408f584e438f5857403122270a2
:10702000e584f0a3e585f07403122270e0f5840591
:1070300092e0c0e07407122270d0e00592f0544153
:10704000c0e07408122270d0e0f0eaa2e05003021f
:1070500070ede060030270f57407122270e0641ea8
:1070600070030270f57405122270127639e84960d7
:107070000e7401122270125c461217e00275bc12e7
:1070800017da8a218b22a821a9227405122270e026
:10709000faa3e0ca242f125dfce849700c7a017b48
:1070a0000090032e740802211888828983a3a3e428
:1070b000f0041222701255837405122270e0faa3b4
:1070c000e0ca242d125dfc740512227012764674fb
:1070d00005122270127619e4f074051222701275ee
:1070e000f12431f582e438f583e4f0800874051268
:1070f00022701276469003a074081220bf8b22eaf9
:10710000452260030275bc852382852483a3a38561
:1071100082258583267403122270127604a3ac8222
:10712000ad837403122270126771ae82af83740153
:107130001222701276048582848583857407122258
:1071400070e0547f14700302753014700302754ba5
:1071500024fe70030272b11470030272ea14700309
:107160000271e8147003027314147003027267143e
:1071700070030272f81470030273b914700302757d
:10718000101470030273b914700302752014700395
:1071900002738714700302751014700302722d14a9
:1071a00070030273061470030273331470030273c6
:1071b0008124fd70030275581470030273811470ea
:1071c0000302756514700302738124fe7003027458
:1071d0007d24fe700302749c14700302750324cc9a
:1071e00070030273220275721276851215cae96065
:1071f000030272ba852382852483a3a3a3a3a3a336
:10720000a3a37407f08525828526837405f0e52302
:107210002409fce43524fd0592e024f5f9eefaefab
:10722000fb121582e970030272d00272df127685ba
:107230001215cae960030272ba1275d97411127676
:107240005da832a9338821892278211224e612759b
:10725000c1121528740212221c853282853383e004
:10726000600302744280781276851215cae9704a6a
:10727000853282853383e4f0a832a93388218922bc
:1072800078211224e6ac23ad241275c11215b8740e
:107290000212221ce9700e853282853383e070056c
:1072a000740af08009853282853383e0603102748c
:1072b000421276851215cae9600675210102734be8
:1072c0001275d912765deefaeffb1215bee9700f5a
:1072d00075210a78211224ea8e828f8302745385e5
:1072e0002582852683e02902746f740112227012b0
:1072f0005c461214c802758a7401122270125c4630
:107300001214c202758a7401122270125c461214a1
:10731000d402758a7401122270125c461214ce02d5
:10732000758a75210078211224ea125c38121564de
:1073300002749575210178211224ea125c38121525
:1073400064740112221ce9602af52178211224ead2
:107350008e828f831275fb12227012678af9740273
:107360001222700592125c46121378740112221ccc
:107370000275837401122270125c46121366027544
:107380008312152e0274ea852582852683e0700615
:107390001275df740ff0ac23ad240592e024fbf5e9
:1073a00021e434fff522740178211221d4a921eec1
:1073b000faeffb1215760274ea7a007b00852382cd
:1073c000852483a3a3a3a3a3a3a3a3a38582278523
:1073d0008328852582852683e0700a1275df740b69
:1073e00012767c04f0740312227012678a640c70a7
:1073f0001a8523828524830592a3a3a3a3a3a3a311
:10740000a3740df08c828d83125c46a832a9338858
:107410002189225392fe78211224e685272185288e
:107420002278211224e67916eafcebfd125c421266
:10743000157c740412221ce9f8853282853383e0be
:10744000602485328485338505921225018e828fd2
:107450008305921275fb12227012678af9aa23ab78
:1074600024121378802f18852582852683e028f042
:107470007c047d00aa23ab241215d6806d858482fe
:10748000858583e024f9f52178211224ea79011217
:107490005c421214b0740112221c804ee5c7f890b1
:1074a0000368e0f5c790f7f4e05404f52188c7605d
:1074b0001874051222701275f12416f582e438f55d
:1074c00083e0d2e0f07905800279028584828585a7
:1074d00083e024f9f52278221224ea125c42121485
:1074e000b0740112221ce521600b7401122270128b
:1074f0005c460275877401122270125c4612136c8e
:1075000002758a7401122270125c4612153a807a52
:107510001275cc1222700592125c461214bc806a5d
:107520001275cc1222700592125c461214b6805a63
:107530007403122270127613e0f97403122270128f
:107540006771a3125c461214aa809f740112227004
:10755000125c46121372802b7401122270125c4668
:10756000121570801e7401122270125c4612156a88
:1075700080117401122270125c461217e0e5234557
:10758000246007aa23ab241217e07408122270e0cb
:10759000702a7407122270e0641e602074051222a3
:1075a00070127629e4f0a3f074051222701275f1be
:1075b000242ff582e438f583e4f0a3f07409026720
:1075c000d90592e024f7f9eefaeffb220592e024c8
:1075d000fbf91c1ceffd740122852582852683742e
:1075e00005f0852382852483a3a3a3a3a3a3a3a338
:1075f000221275f522e0f8a3e0c8221259d77404cc
:10760000225392fe12760822e0f8a3e0f5838882e6
:10761000a3a322127608a3a32212761d221275f5c7
:107620002433f582e438f5832212762d221275f583
:10763000242df582e438f5832212762d127640222d
:10764000e0f8a3e0f9221275f5242ff582e4381250
:10765000765322f583e0f523a3e0f5242212767c0d
:10766000f8e5231267253524f583a3a3a3a3ac82f1
:10767000ad83852582852683e004f022f08525826e
:10768000852683e0228c828d831259d78e828f8348
:1076900012769422e0faa3e0fb2274ef12229e7489
:1076a000fe1222371224d2ecffedfee9127715ef1d
:1076b000a312771d2405127a0190089f7825121fc6
:1076c000649008a37825121fc974087825121f3208
:1076d00078217925121fdc9008f37821121fef9092
:1076e000063a782112204a741312227a0592122443
:1076f000fd7a3a7b067909127a8012229c74021272
:10770000221c8532828533831224da740212221cf1
:107710007f0902237690063e127bf3f022f0eea35f
:10772000f0f525f582ac827d002274ec12229e7465
:10773000fe1222371224d2e9ff8a258b26ecfeefb7
:1077400090063ef0eea3f0f5297d002402127a0b9c
:10775000f52af52bf52c9008f77829121f6490086c
:10776000a37829121fc974087829121f3278217949
:1077700029121fdc9008fb7821121fef90063a783f
:107780002112204a78251224e67a3a7b06790612dd
:107790007a7e12229c740212221c853282853383e7
:1077a0001224da740212221c7f0c02237674f61261
:1077b000229e74fe1222371224d2e9feeaffee90d6
:1077c000063ef0efa3f0a3e4127c2604f0a3e4f05d
:1077d000027a4d74ec12229e74fe1222371224d2c9
:1077e000e9fe7416122270e0f525a3e0f526e525e2
:1077f00045266066ee12798a7418122270e09006af
:1078000043f0f529752200240650020522e4c52222
:10781000f521e4f523f524f52af52bf52c9008ff46
:107820007829121f649008a37829121fc974087858
:1078300029121f3278217929121fdc90090378213f
:10784000121fef90063a782112204a78251224e67a
:1078500090064312794c790a801012787a1224e645
:107860007c007d007a3a7b067909127a7e12229c8e
:10787000740212221c790102779aee90063ef0a360
:10788000e4f0a3127bf3f012789314f0a3740112c6
:107890007ae62290063a7480f0a37405f0a322746d
:1078a000f012229e74fe1222371224d2e9feec4d11
:1078b000606aee1277157412122270e0900641f0a1
:1078c000f525752200240450020522e4c522f52185
:1078d000e4f523f524f526f527f5289008b7782553
:1078e000121f649008a37825121fc9740878251206
:1078f0001f3278217925121fdc9009077821121f89
:10790000ef90063a782112204a8c218d227821129c
:1079100024e690064112794c7908801012787a1288
:1079200024e67c007d007a3a7b067909127a7e1281
:10793000229c740212221c790185328285338312c3
:1079400024da740212221c7f08022376e0fc7d00f8
:107950007a3a7b062274f612229e74fe12223712a5
:1079600024d2e912798a740c122270e09006431234
:107970007c6a7402f0a314127ae21224e67c007d81
:10798000007a3a7b06790a027a60127bf0f0a3ec67
:10799000f0a3edf02274ef12229e74fe1222371231
:1079a00024d2ecffedfee990063ef0efa31277182b
:1079b0007413122270127c5f12771d2407127a0151
:1079c0009008c77825121f649008a37825121fc954
:1079d00074087825121f3278217925121fdc90094e
:1079e0000b7821121fef90063a782112204a741565
:1079f00012227a05921224fd7a3a7b06790b0276de
:107a0000f7127a0bf526f527f52822e43400f52243
:107a1000e4c522f521e4f523f5242274f612229e12
:107a200074fe1222371224d2e990063e127b5b7458
:107a3000011278987403127ae21224e67c007d0029
:107a40007a3a7b0679058018127cf7f0e4f521f587
:107a50002278211224e67c007d007a3a7b067907a1
:107a6000127a7e12229c740212221c853282853385
:107a7000831224da740212221c7f020223760592fa
:107a800090064ee0f582a3e0f58305922274f4128d
:107a9000229e74fe1222371224d2e98a218b228c74
:107aa000238d2490063ef0a3782112204a12789369
:107ab000f0a37402127ae21224e67c007d007a3a86
:107ac0007b067909127a7e12229c740212221c858e
:107ad00032828533831224da740212221c7f04025c
:107ae0002376127ae622f0e4f521f5227821227439
:107af000f612229e74fe1222371224d274fc122235
:107b000006eafeaa32ab33f9121978ee90063ef07f
:107b1000853282853383e090063ff0740112227033
:107b2000e05401900640f07403122270e090064188
:107b3000127b5b7404f0a304f0a314127ae2122403
:107b4000e67c007d007a3a7b067908127a7e122262
:107b50009c740212221c7404027a68127b5f221247
:107b60007b6322f090063a7480f0a32274f612220e
:107b70009e74fe1222371224d2127bbb027a487402
:107b8000f612229e74fe1222371224d2e9127bf0e2
:107b9000027a4874f612229e74fe1222371224d200
:107ba000127bbbf0a3e4f0a31278861224e67c00db
:107bb0007d007a3a7b067909027a60e990063ef008
:107bc000a37485f0a374012274f612229e74fe122f
:107bd00022371224d2e9feecffee90063ef0efa32e
:107be0006006f0a374048003e4f0a3127bf380b872
:107bf00090063ef0a3eaf0a3eb2274f612229e74e4
:107c0000fe1222371224d2e9feeaffee90063ef081
:107c1000efa36006f0a374028003e4f0a3127c26b5
:107c2000f0a304027a4b127d00f0a32274f6122214
:107c30009e74fe1222371224d2e9feeaffee90066d
:107c40003ef0efa3f0a3ecf0a3edf0740c12227061
:107c5000127c5f127c6a7403f0a3740102797712bc
:107c60007ee2900642e8f0a3e922127b5f7406f000
:107c7000a32274f412229e74fe1222371224d2e937
:107c800090063ef0a37408f075218075220a7523d2
:107c90000375240290063a782112204a8a218b2209
:107ca00078211224e67c087d007a3a7b0679060268
:107cb0007ac474f612229e74fe1222371224d2e97c
:107cc000feea70077a00121b5e8029ee90063ef0f5
:107cd000eaa3f0a37402127cf7127ae21224e67c83
:107ce000007d007a3a7b067907127a7e12229c7414
:107cf0000212221c027a6b127d0012789874012203
:107d0000127b6374032274f712229e7a04121b5ea4
:107d10007f0102237674f712229e7a0880ef74efb7
:107d200012229e74fe1222371224d2eaffebfe7456
:107d3000992990063ef0efa3f07521067522007890
:107d4000211224e67a407b06121cd2740212221cf5
:107d5000ee900646f07413122270e0900647f0741d
:107d600014122270e0900648127720240b127a0138
:107d700090090f7825121f649008a37825121fc957
:107d800074087825121f3278217925121fdc90099a
:107d9000137821121fef90063a782112204a7415a9
:107da00012227a05921224fd7a3a7b06790f027626
:107db000f774f412229e74fe1222371224d274f049
:107dc000122206e9feeaff1213dee9f5226022ac78
:107dd00032ad33740a12228ceef91213d8740112e8
:107de000228ceef91213e4eef91213eae9f5218080
:107df0004075230675240078231224e67c007d005c
:107e0000740c12228c121cd8740212221c752309c5
:107e100078231224e67c007d00740312228c121c4d
:107e2000d8740212221c853282853383e4f07521d6
:107e3000ffee90063ef0e522a2e55004d2f080026b
:107e4000c2f0a2f0e433f8e522a2e750047a0280ff
:107e5000027a00e84a4fa3f07523067524007823c0
:107e60001224e6740c1222947a407b06121cd274ff
:107e70000212221c853282853383e0900646f0741c
:107e800004122270127ee2900647e8f0a3e9f07433
:107e900008122270127ee2900649e8f0a3e9f0741d
:107ea00006122270127ee290064be8f0a3e9f0e59c
:107eb00021a3127b5b7410f0a37403f0a3e4f0f52c
:107ec00021f52278211224e67c007d007a3a7b0697
:107ed0007914127a7e12229c740212221c741002ef
:107ee0007acce0f8a3e0f92274f612229e74fe1216
:107ef00022371224d2e9fe90063eeaf0a3ebf0ee20
:107f0000a3127c2614f0a3027a4bc082c08375347e
:107f1000015392fe900367e0a2e05004788080064f
:107f20007800800288c6e59e6870f99062707408d7
:107f3000f0d083d082021129c082c08374fe122245
:107f4000067902aa32ab3312178c853282853383cd
:107f5000e0f5bc7401122270e0f5bc740212221c20
:107f600080cf74f712229e74fe1222371224d28a16
:107f7000848b85800b5392fe90618fe00592f0a375
:107f8000e9f874ff28190470ec8532828533835335
:107f900092fe1224da740212221c7f01022376c0a0
:107fa00082c083121402e9900368f079017c007d9d
:107fb000ff7a677b031213fcd083d08202112974ed
:107fc000f612229ee9ffe5c7fe900368e0f5c78f31
:107fd0002175220078211224e6121cd2740212228a
:107fe0001c8ec77f02022376c082c083790353921e
:107ff000fe906276e0a2e65002790780bb80feff29
:1080000074f612229e75210c75220078211224e646
:108010007c007d007a547b60121cd802b39fc08222
:10802000c0838a828b8380075392fee0f5d9a3e94f
:10803000f874ff28190470f00285acc082c0838aee
:10804000828b838007e5d95392fef0a3e9f874ff91
:1080500028190470f00285ac74f612229e74fe1288
:1080600022371224d2e970159004bce06401700d2f
:108070009003f7e0640170051216cc804f9003f76f
:10808000e070231280cf60160592a3a3a3a3a3a33d
:10809000a3a3e0f9121780900404e4f0a3f0900386
:1080a000f574fff08026790012198a8b22ea2402e7
:1080b000f8e43522f99003efe8f0a3e912ac1f9041
:1080c00003f1128b0e7aed7b0312371302b39690f5
:1080d0000404e0f584a3e0f585e58445852274f485
:1080e00012229e74fe1222371224d274fc1222062f
:1080f0008a848b85853282853383e412b512a3f09e
:1081000090618fe0c0e08532828533837821122030
:108110003be5842521f582e58512a6bfd0e0f090ed
:108120000897782112203b8532828533837821128b
:108130001f779008b7782112203b853282853383e0
:108140007821121d6840b985848285858312208933
:108150008532828533831220957a00853282853379
:1081600083782112203be521543ff8743f68601f5b
:10817000e8601c853282853383782112203b7401ac
:108180007821121f191282e00aeac3941b40ccea3c
:10819000c3941b50030280f48584828585837821f3
:1081a00012203b90080978211220288532828533dd
:1081b00083782112204a79007a00853282853383c0
:1081c000752101752200ea78211221f3e522339509
:1081d000e0f523f5247821121fc9e5214522452326
:1081e00045246001090aeac3942040cee9c3940201
:1081f00050030280f40592e0f8858482858583052a
:1082000092a3e068701c858482858583a3a3e068bf
:108210007010858482858583a3a3a3e06870030220
:1082200080f4858482858583122089853282853316
:108230008312209579007a1f8532828533837821d5
:1082400012203be5215403f874026860057401684c
:10825000700109853282853383782112203b7401b5
:108260007821121f191282e01aea70cce9c394191e
:1082700040030280f4858482858583782112203b27
:10828000741a7821121f198532828533837821125e
:10829000204a79007a05853282853383782112203d
:1082a0003be5215403f874026860057401687001ad
:1082b00009853282853383782112203b740178212d
:1082c000121f19853282853383782112204a1aead7
:1082d00070c4e9c3940250030280f4740402b1ff35
:1082e000853282853383e521f0a3e522f0a3e523df
:1082f000f0a3e524f02274f612229e74fe122237b7
:108300001224d28a848b85e9701e7521087522009b
:1083100078211224e67c007d00121cd874021222ff
:108320001c74010592f080280592e0a2e0e433f08d
:10833000752107752200059278211224e67c007dc4
:10834000000592a3aa84ab85121cd8740212221cc9
:108350008532828533835392fe02b39c74f61222d7
:108360009e9004d4e0a2e04060793012198a8a21fc
:108370008b22ae21af229061b1e4f0e070f874037b
:10838000f0e0640370f81217749004d4e0d2e0f0c7
:10839000753400e59ea2e640fae594a2e240097534
:1083a0009403e594a2e250fa790012198a8a218b8b
:1083b00022c3ee9521feef9522ff54807004ee4f0c
:1083c0007007e5e170fc75e12102b3a474f6122296
:1083d0009ee9fe60067c9d7d0480047c977d04758b
:1083e000210675220078211224e67a167b60121c81
:1083f000d2740212221c906015e0c2e0f0ee60041c
:10840000780180027800e048f002b3a474f61222ea
:108410009ee9fe75210675220078211224e6eafc09
:10842000ebfd7a1c7b60121cd2740212221c90603d
:1084300015e0c2e1f0ee600478028002780080c6a8
:1084400074f712229e74fe1222371224d2e9fe8c97
:10845000848d85740b122270e0ff74072ff5d98e7e
:10846000d979061216128007439201e0f5d9a3efdd
:10847000f874ff281f0470f0e5e170fc75e19502c7
:10848000ab7b74f612229ee9fe90046012ab75601d
:1084900004793a8058906022e0f874ff687004799b
:1084a00007804a7f0080040fc313f8e8a2e040f77a
:1084b00075210675220078211224e6eafcebfdef17
:1084c00012858e121cd2740212221c752101ef78c3
:1084d000211221f3af21eff4f8906023e058f0ee81
:1084e0006003e04ff0906022e04ff0790002b3a407
:1084f00074f312229e74fe1222371224d289258a26
:10850000848b8590046012ab756004793a80669024
:108510006022e0f522a3e0ff7521017e00e52255ef
:10852000216043e5256007852182a88280027800ca
:10853000ef552168703075230675240078231224c6
:10854000e6ac84ad85ee12858e121ccc740212222c
:108550001c8b24ea4524700ee521f4f8906022e09b
:1085600058f07900800f0ee521c333f521eec39456
:108570000840aa79128532828533831224da740284
:1085800012221c7f050223767cbf7d04e52275f054
:1085900006a4f8a9f0742428fa746039fb22c0827a
:1085a000c0835392fe906022e402b2f5d083d08261
:1085b0005392fe02112974f012229e74fe12223789
:1085c0001224d28c278d28eafcebfdea24faf8eb82
:1085d0001286e440030286c3e52724faf8e5281250
:1085e00086e440030286c3c3e5279ae5289b50032f
:1085f0000286c3741612227012b27dc3ee94f5ef98
:10860000940140030286c37414122270e0f521a382
:10861000e0f522e52124f6f8e52212899b9477e91a
:10862000940c40030286c39004c6e0f8c394024051
:1086300037e8c333f88882858225ecf8edf9aa255e
:108640007b0012217b8a238b24a823a924e849607c
:1086500017ec2525fae43dfbeac398fceb99fdc332
:10866000e5279ce5289d405b740378211221f3c027
:1086700021c022ee2401f525e43ff526e4f527f597
:10868000288c218d22f523f52478257921121d9738
:10869000d022d02178217925121f8a852125852293
:1086a000268523278524289009307825121fc9e5bf
:1086b00025452645274528700ae5214522452345bd
:1086c000247004791280117412122270128913ec32
:1086d0000592f0a3edf079008532828533835392c1
:1086e000fe02a95612899b947be9940c2274f01225
:1086f000229e74fe1222371224d274fb122206e943
:10870000853282853383f07403122270ecf0a3ed7e
:10871000f08a278b28900491e0a2e040079003f5af
:10872000e0f46005790c028910741c122270e0f5e7
:1087300023a3e0f524741e122270e0f521a3e0f5d6
:108740002278211224e678231224e674051222846a
:108750008825892678251224e6742012227012a614
:10876000d4741e12227012a3ee12165a740612222c
:108770001ce960030289101217868a258b26ae2514
:10878000af26ee4f700579090289108e828f83a380
:10879000a3a3a3a3a3a3a3e0c0e0740312227012b7
:1087a0008913d0e00592f0e5274528604475250639
:1087b000752600059278251224e6ac27ad28ee2414
:1087c0000bfae43ffb121cd2740212221cee24129c
:1087d000129b5b853282853383e005926005e0d28f
:1087e000e08003e0c2e0f00592906014e0c2e38014
:1087f000080592906014e0d2e3f07417122270e042
:1088000060047a0180027a00900495e054fef8a397
:10881000e0f9e84a900495f0a3e9129cbaee24141a
:10882000fae43ffb1216247a0090618fe0c0e01258
:108830009ca82418f582e439f583d0e0f00aeac355
:10884000940340e512b097ee12a4ae3ff585740193
:1088500012227012ab5bee2422f582e43ff583e531
:1088600023f0a3e524f0129f551296e2e521f0a330
:10887000e522f0129f2d7405f0ee241bf582e43ff3
:10888000f5837402f00592e0f8a3e0f9129f23e863
:108890000592128b0f9004b9e0c0e0ee24e5f5825a
:1088a000e43ff583d0e0f0752105752200782112b0
:1088b00024e67cb47d04ee2424fae43ffb121cd2af
:1088c000740212221ceefaeffb1216d290618fe0b6
:1088d00054072405c0e0ee2429f582e43ff583d057
:1088e000e0f0e5a8f8c2af9003fa12a3eea312a637
:1088f000c49003f1eaf0a3eb12a33a900404eef063
:10890000a3eff09003f574f0128c2012174a79004f
:1089100002a94be0f584a3e0f5852274f712229eac
:10892000e9feec4d602cea4b6028ea24e0f8eb12fb
:108930008992500aec24e0f8ed1289924004790003
:10894000804dec2af8ed3bc313f9e81390041212a2
:108950008b0fee6004900411f07409122270e09005
:108960000416f0740b122270e090040f6005e0d240
:10897000e08003e0c2e0f0906014e054fcf0740a80
:10898000122270e0f86006906014e048f07901026d
:10899000ab8c12899b94e1e9943f2234fff9c3e840
:1089a0002274f612229ee990040f6005e0d2e18065
:1089b00003e0c2e1f075210675220078211224e659
:1089c000eafcebfd7a187b04121cd2740212221c02
:1089d000790002b3a474f612229e74fe122237129a
:1089e00024d274ff122206e9fe9004107077e06032
:1089f0006fa2afe433f521c2af900460e06406706b
:108a000004a3e06404701712ae254009759403e5d1
:108a100094a2e250fae5e170fc75e142800d900409
:108a20000e74fff07a067b04121744900410e4f0f1
:108a3000e521a2e092af90040e128c2c64f460f653
:108a40009004141280d260180592a3a3a3a3a3a339
:108a5000a3a3e0f9121780900414e4f0a312a33149
:108a6000790002b391e06004793a80f6eec3940293
:108a7000900417400474018001e4f0900416e0f8bb
:108a8000740368604c74026860479004c7e0600437
:108a9000790c80ce1217868a218b22a821a92290d8
:108aa0000414128b0ee8497004790980b590049182
:108ab000e04401f0900495e054fef8a3e0f990043e
:108ac0000fe0a2e0e433fae84a900495f0a3e980cd
:108ad00006900414e4f0a3f074016e90040a700789
:108ae000e4f0a374088005740af0a3e4f090041085
:108af0007401f090040e74f4f07a067b0412174aa5
:108b0000028a60e5212434f582e43522f583e812f7
:108b1000b28e2274f512229e74fe1222371224d2d3
:108b200074ff122206e9feeaffee7073a2afe4338f
:108b3000f523c2af900460e064ed7004a3e0640329
:108b4000701712ae254009759403e594a2e250fa1d
:108b5000e5e170fc75e14280309003f7e06401705c
:108b6000281280cf60160592a3a3a3a3a3a3a3a357
:108b7000e0f9121780900404e4f0a3f09003f57478
:108b8000fff07aed7b031217449003f7e4f0e5233e
:108b9000a2e092af9003f5128c2cf4600c80f5905b
:108ba00003f5e0f874f868701a7900740112221c59
:108bb0008532828533831224da740212221c7f03e9
:108bc00002237674ff686004793a80df9003f8e44a
:108bd000f0906009f0eb9003f66005e0d2e48003ca
:108be000e0c2e4f0906014e0c2e2f0ef6004e0d292
:108bf000e2f09003f9e4f09003f6e054b3f09060f3
:108c00000a7401f0a3e412ac1fa3128b0e9003f1bf
:108c1000128b0e9003f574f8128c2012174a80897b
:108c2000f09003f77401f07aed7b032212962fe0a7
:108c300022c082c083e95392fe90619a700e743311
:108c4000f0a37455f09061a0743a800312908c02e6
:108c5000b2f5c082c083e9c3940f4002790ee9c423
:108c600054f0f85392fe906186e0540f4802b2f53a
:108c700074f612229ee9ffc3942040027f1fe5a8ec
:108c8000fec2af8f2175220078211224e6eafceba8
:108c9000fd7a1e7b04121cd2740212221cef900477
:108ca0003df0eea2e7a2e792af02b3a474f612225f
:108cb0009ee9ffc3942040027f1fe5a8fec2af8f4c
:108cc0002175220078211224e6eafcebfd7a3e7b36
:108cd00004121cd2740212221cef90045d80c27434
:108ce000f412229e74fe1222371224d2749f122292
:108cf00006e9fee5c7f521900368e0f5c790036734
:108d0000e0a2e0401ae0d2e0f00592900840122480
:108d1000f97b0a7a0079001219ba740412221c74c1
:108d2000ff6e70069004c6e08001ee8532828533c6
:108d300083f07523dc75240078231224e67c007d03
:108d4000007aed7b03121cd8740212221c85328239
:108d5000853383e09004c6f075236678231224e6f9
:108d60007c007d007a007b60121cd8740212221ce9
:108d7000900412e4f0a37402f09004117407f090d0
:108d8000040e74fff09003fe744b12b09c9003f13c
:108d9000743212b09c9003f6f09003f3740412b096
:108da0009c90040c740512b09c7523257823122422
:108db000e67c007d007a6b7b04121cd874021222c0
:108dc0001c75230478231224e67cff7d007ab47b93
:108dd00004121cd8740212221c9004b8741ff09064
:108de0000467e4f0a3f0900404f0a3f074ff6e6055
:108df00011ee75f0e6a4faabf012130c90045e12bb
:108e0000a6c490045e12b2839004c7e41290ab80b3
:108e100018e58424e6f8e43585f985848285858320
:108e2000e8f0a3e9129099e004f0e0fa12a167eeed
:108e300024fff8e434fff9c3ea98e499a2d265d09c
:108e40003340ce858482858583e4f0a31290999087
:108e50000406e4f0a3f090040e74f4f09003ede443
:108e6000129cb079107cc7fd740112228c1213fc85
:108e700075230678231224e67c0e7d787403122273
:108e80008c121cd2740212221c7523107823122417
:108e9000e67ce97d077413122270aa82ab83121c50
:108ea000d2740212221c78107401122270e5821210
:108eb0009b6d3583f583e064bff008e8c3942040e0
:108ec000e774011222848823892478231224e6740b
:108ed000031222947413122270aa82ab831212d648
:108ee000740212221c79107cd77dff74111222703b
:108ef000aa82ab831213fc75231075240078231209
:108f000024e67413122270ac82ad83740312228c97
:108f1000121ccc740212221c8b24ea45247005809a
:108f20000c121786eeff74ff2f1e0470f41219a2a4
:108f30001217e69061c67401f09061807440f09061
:108f400061917448f09061bc7407f090619a12903e
:108f50008cf090618674e1f0a37419f09061bce428
:108f6000f0900367e0a2e7403879017c017dffaa19
:108f700032ab331213fc853282853383e0c4540f45
:108f8000f0c3940f4003740ef0e0c454f0f090610d
:108f900086e0540ff8853282853383e048906186fd
:108fa000f074ff6e7007906192e0d2e7f09060225b
:108fb000e4f0906009f043a90143b901759b007585
:108fc0009100439a01c2a890f7f4e0a2e350047420
:108fd000e1800274c09004c8f0906181e4f0a37451
:108fe0008012b09c794074211222947a037b001283
:108ff000182ee9fb74ff6b60367a00802d74211205
:109000002270e5822af584e43583f585858482859e
:109010008583a3e0c0e00592e0f87480129b6d3474
:1090200061f583d0e00592f00a0aeac39b40ce12b4
:1090300025cb12160c1217569004bae4f09004bc1b
:10904000f09004bbf09004bdf0906002740ff090bb
:10905000f7f4e0a2e4500474058002740290600307
:10906000f0900460e4f0a3f0900495e054fef090da
:10907000040fe4f079067cea7dff7a977b041213f3
:10908000fc1219de8521c7746102b1ff743ff0a3a1
:10909000745af09061a0747f221290abe00592a305
:1090a000a3a3a3a3a3a3a3f0059222f085328285f4
:1090b00033832274f612229ee5a8fec2af75210604
:1090c00075220078211224e6eafcebfd7a9d7b04f0
:1090d000121cd2740212221c028ca274f712229e5d
:1090e00074fe1222371224d2e975f0e6a4fcadf02a
:1090f00090045ee02cf584a3e03df585ea8584824a
:10910000858583a3a3a3a3a3a3a3a3a3f00592a3ed
:10911000a3a3a3a3a3a3a3a3a3740af08532828568
:109120003383059202ab8474f012229e74fe1222e5
:10913000371224d274ff1222068a278b281296280f
:109140003528f583e0547f12a343ae82af838a8231
:109150008b830592a3a3a3a312962f12a5478a82fd
:109160008b83a3a3a3a3a3ac82ad83ee240af5252e
:10917000e43ff526ee2411f521e43ff52285328205
:10918000853383e070030292e71470030292b014f7
:1091900070030292a814700302944a14700302959b
:1091a000511470030295ae1470030295b514700348
:1091b00002935f14700302925d14606614700302e0
:1091c00093691470030293a5146009147003029349
:1091d000360295fb75230575240078231224e6eeec
:1091e000243ffae43ffb121cd2740212221c852594
:1091f00082852683e064077002e4f085218285225f
:1092000083e0d2e1f0a2e0400dac27ad28eefaef0a
:10921000fb1217688007aa27ab281217e07b03020e
:1092200095e6852582852683e064066003029363c4
:10923000852182852283e0d2e212aafce4f0752126
:1092400008f52278211224e6aa23ab24121cd2743a
:109250000212221caa27ab281217e0804685218221
:10926000852283e0d2e2f075210875220078211270
:1092700024e6aa23ab24121cd2740212221c790108
:10928000aa23ab2412162a78211224ea7823122466
:10929000e67909ac27ad28eefaeffb1216c074038d
:1092a00012221c7b040295e61296a874090293bc54
:1092b0008525828526837402f07521077522007842
:1092c000211224e6ee2457fae43ffb121cd274026a
:1092d00012221caa27ab281217e0ee245c1296bebd
:1092e000603a12969280358525828526837401f036
:1092f00075210b75220078211224e6ee244cfae445
:109300003ffb121cd2740212221caa27ab28121790
:10931000e0ee24551296be6003129692e5a8f52160
:10932000c2af7901eefaeffb121750e521a2e7a2d6
:10933000e792af0296231296a8e064037021e4f04e
:10934000852182852283e054e7f07b078e828f831c
:10935000a3a3a3a3a3a3a3a3e0fa790012397daa30
:1093600027ab281217e0029623852182852283e00d
:10937000d2e4f075230078231224eae4f52478235c
:109380001224e6790bac27ad28eefaeffb1216c0db
:10939000740312221c852182852283e0c2e6f0d26a
:1093a000e3f0029623852182852283e0d2e4129f96
:1093b000ee852182852283e05005c2e7f080a0542b
:1093c0003ff075210078211224eae4f52278211279
:1093d00024e6790bac27ad28eefaeffb1216c07429
:1093e0000312221c75210878211224e6129683129a
:1093f0001cd2740212221c75210478211224e61258
:109400009674121cd2740212221c78211224e612c5
:109410009665121cd2740212221c85258285268331
:109420007403f075211678211224eaee245ef521ea
:10943000e43ff52278211224e67403c0e01217da23
:10944000eafcebfdd0e0f90296178525828526839c
:109450007404f0ee242ef584e43ff5857800797de0
:1094600012b03012a3ee12217b89240592e028f875
:10947000a3e03524f9e824010850010912aae4e820
:109480000592128b0f75231675240078231224e69b
:10949000ee245efae43ffb121cd2740212221c7905
:1094a00008ee2474fae43ffb1219e47904ee247cfc
:1094b000fae43ffb1219e475230878231224e6121c
:1094c0009683121cd2740212221c78231224e612f4
:1094d0009656121cd2740212221c75230478231291
:1094e00024e6129674121cd2740212221c782312e3
:1094f00024e6129665121cd2740212221c782312e2
:1095000024e6129647121cd2740212221c782312ef
:1095100024e6129638121cd2740212221c85218273
:10952000852283e04418f075210c78211224eaee9c
:109530002474f521e43ff52278211224e67904ac65
:1095400027ad28eefaeffb1216c0740312221c801e
:1095500060852182852283e0d2e4f075210c75229a
:109560000078211224e6ee2474fae43ffb121cd2a8
:10957000740212221c75210878211224e6129656d4
:10958000121cd2740212221c75210478211224e6c6
:10959000129647121cd2740212221c78211224e661
:1095a000129638121cd2740212221c02935f1217f8
:1095b000e07b0680311217e0900491e0a2e05011a8
:1095c0008e828f83a3a3a3a3a3a3a3a3e0f9121660
:1095d000e4852182852283e054e712aafc740b12f1
:1095e0009fee403f7b078e828f83a3a3a3a3a3a3f9
:1095f000a3a3e0fa790012397d8028752101782132
:109600001224ea74011222848821892278211224ea
:10961000e67907ac27ad28eefaeffb1216c074030b
:1096200012221c740102a94dea2424f582e422e0ee
:10963000853282853383f022ee247cfce43ffdee0c
:1096400024aafae43ffb22ee247cfce43ffdee2456
:10965000bafae43ffb22ee2474fce43ffdee2498ca
:10966000fae43ffb22ee2470fce43ffdee24a6fa70
:10967000e43ffb22ee2470fce43ffdee24b6fae466
:109680003ffb22ee2468fce43ffdee2490fae43f29
:10969000fb228e828f83a3a3a3a3a3a3a3a3a3745c
:1096a0002812aafc740af0228c828d83e08e828fad
:1096b00083a3a3a3a3a3a3a3a3a312aafc22f58419
:1096c000e43ff58512ae1412ac270592e0c398f87a
:1096d000a3e099f9ee1296e20592e028a3e039544e
:1096e00080222420f582e43ff5832274f712229e23
:1096f00074fe1222371224d2eafeebffa2afe4334b
:10970000f521c2af12981aeefceffd1297fb12166c
:1097100000129805700988828983eef0a3eff07932
:1097200001aa84ab85121750e521a2e092af8532e1
:109730008285338302ab8474f712229e1296283bf3
:10974000f583e0547ffe12975e243dfae439fb1264
:1097500016007b05eefa790012397d02ab8ceafc2b
:10976000ebfdee75f0e6a4f8a9f090045e12977197
:109770002212a90b39f9e82274f712229e74fe1204
:1097800022371224d2eafeebffee4f60618e828f09
:1097900083a3a3e070051217e0805312981aa2afba
:1097a000e433f521c2af1297f11298df402ca2e307
:1097b000eefceffd401f1297fb1216001298057089
:1097c0000988828983eef0a3eff07901aa84ab8542
:1097d0001217508013121600800eeefceffd1216c9
:1097e00000aa84ab851212f4e521a2e092af0297a1
:1097f0002ee584243bfae43585fb22e5842439fafe
:10980000e43585fb22e5842437f8e43585f9888240
:109810008983e0faa3e0fbea4b22129b53e0547fda
:1098200012a16b2274f412229e74fe1222371224ab
:10983000d28a848b85ecfeedffee4f70030298dc3c
:10984000858482858583a3a3a3a3a3a3a3a3e0c048
:10985000e0129b4fd0e0129b647403f0741012224c
:1098600070e0f523740125238e828f83a3a3129bbe
:1098700064a3e9f0e523601f75240078231224e631
:10988000741012227012a6d4ee2405fae43ffb12e3
:109890001cd2740212221ca2afe433f521c2af1213
:1098a00098dfeefceffde584500f1297f3121606d9
:1098b000aa84ab851212f4801d1297fd12160012b5
:1098c0009805700988828983eef0a3eff07901aae8
:1098d00084ab85121750e521a2e092af02b20212ca
:1098e000a0d1a2e72274f012229e74fe1222371237
:1098f00024d2eafeebff8e848f850592a3a3e5d9df
:1099000014f0e5d98e828f830592a3a3a3f0a2e57c
:10991000502a0592e0c3940640227800e5d9c0e0c1
:1099200074bf129b6d3404f583d0e05392fef008af
:10993000e8c3940640e60592e024faf07800800e31
:10994000129b6d3ff583a3a3a3a3d0e0f008858409
:10995000828585835392fee0f9e8c399e5d9c0e09a
:10996000ee40dd2425f582e43ff583d0e0f0ee24df
:1099700026129b5be5d90592f0f8a2e74003029a14
:10998000f0740358242505929004c5f00592e05424
:10999000fcf0240c7003029b4824fc600a1217e0c0
:1099a0007a007b00029b4c05929003f6e0a2e44013
:1099b00003029b48906009e0f8906022e048f52699
:1099c0007522007521018e828f83a3a3a3e0f87412
:1099d0004058f528906023e0f527740f58f525745a
:1099e000046525600ee5a8f8c2af9003f6e0c2e674
:1099f00012a33ae52655216031e5286007852182ca
:109a0000a88280027800e527552168701d7523061d
:109a100075240078231224e6128588121ccc740267
:109a200012221c8b24ea4524600fe521c333f52163
:109a30000522e522c3940840ba906014e0a2e274c3
:109a4000086522500f7003029b48906009e0452191
:109a5000f0029b486036906009e055217013e045a4
:109a600021f0e525607a740665256003029b488035
:109a70006f7404652570129003f6e0a2e6500ae5c3
:109a8000a8f8c2afe0c2e68062029b2b74ff652695
:109a90007003029b487521017522008008e521c3ef
:109aa00033f5210522e526552170f275230675242c
:109ab0000078231224e6128588121cd27402122226
:109ac0001ce521f4f8906023e058129b64e0a2e6c4
:109ad0005007906023e04521f0906009e04521f0b7
:109ae000e5a8f8c2af9003f6e0d2e612a33a805898
:109af000748048fb129b4feb0592f0547f12a167d4
:109b0000e5842411f8e43585f9888489858e828f6f
:109b100083a3a3a3e05403640360190592e0a2e4c5
:109b200050127a3d747f5bf91216a2eefaeffb1227
:109b300017e08010439201e0a2e6500cc2e4f0ef7f
:109b4000fb1212fa7e007f00eefaeffb0286d812bb
:109b50009b5322ee1296293ff58322f8e43ff988c1
:109b600084898522f08e828f83a3a3a32228f58285
:109b7000e42274f212229e74fe1222371224d212b0
:109b8000b27a9004bce014f0906060e0c0e0129ff4
:109b900019d0e0f0e5d9fb129f37e5d9a2e6e050f5
:109ba00004d2e08002c2e0f07a00e5d9c0e0129c65
:109bb000a8240bf582e439f583d0e0f00aeac394d7
:109bc0000640e774fb2bf88002e5d974ff281804df
:109bd00070f790600ee0f525a3e0f5268e848f8562
:109be0000592a3a3791012198aea2525f8eb3526e8
:109bf000f9e82404500109858482858583128b0f3e
:109c000090046780048882898312ab7560478882dc
:109c10008983a3a3a3a3a3a3a3a3e0a2e740e6850c
:109c20008482858583e0a2e092f088828983a3a361
:109c3000e0a2e020f001b3401c900367e0a2e00541
:109c400092e0400924fff0a3e034ff80072401f0f4
:109c5000a3e03400f08e828f835392fea3a3a3a3cc
:109c6000a3a3740412b09c900404129cb09003f758
:109c7000e4f0ee129f107403129cba8e828f83a3bd
:109c8000a3a3a3a3a3a3a3a3129f4112397deefa1a
:109c9000effb1237138532828533831224da740284
:109ca00012221c7f06022376ee2af8e43ff9e8220e
:109cb000f0a3f09003f574fff022f012adf9e4f098
:109cc0002274f712229e74fe1222371224d2ea2442
:109cd000e5f8e43bf988828983e4f0fcec13131384
:109ce000541ff8ea28f8e43bf9e82424f584e43921
:109cf000f585439201e0c0e074075cf8d0e0b8005d
:109d0000028004c313d8fca2e0501c0592e0f8eadc
:109d100028f8e43bf9e824c0f584e439f585ec053e
:109d200092f00592e004f00cecc3942540ae02ab37
:109d30007b74f212229e74fe1222371224d29004f7
:109d4000bce014f090041412b27de5d9f8e5d9f91d
:109d500018740f5964057005742268601008088033
:109d600002e5d974ff28180470f7029f0490606020
:109d7000e0c0e0129f19d0e0f012b097129f37e9cf
:109d8000a2e6e05004d2e08002c2e0f07906ee24c0
:109d90000bfae43ffb121618ee2414f584e43ff5a9
:109da000857906aa84ab851216187916aa84ab8524
:109db000121618e5d9e5d9ee2429129b5b0592e02d
:109dc000c4135407c0e0129f2dd0e00592f0059215
:109dd000e0541ff08e828f830592a3a3a3a3a3a3b5
:109de000a3a3a3e4f0ee241e129b5b129f55129fc7
:109df00010740bf0c30592e09406a3e094005003a6
:109e0000029f047a00129ca812962939f583539276
:109e1000fee070070aeac3940440ea74046a700d15
:109e2000ee2428129fe6541f7003029f04eefaefff
:109e3000fb12312bee241bf584e43ff5850592e0ff
:109e4000700474018007c3940940037408f0e0f8bb
:109e500075f0e2a4c8aaf075f004a42af9e824a0d9
:109e6000f8e93406f90592906064128b0eeefaef71
:109e7000fb1216d28e828f83a3a38582258583262b
:109e8000791012198a129f2312ac23e828f8e933bb
:109e9000f9ea28f8eb39f9e824025001098525820e
:109ea000852683128b0f0592e025e0f8e433f9e86c
:109eb0002403f85001098e828f830592a3a3a3a3e4
:109ec00085828485838512aa5112aaf4e024fef0cb
:109ed000a3e034fff00592e02402f0a3e03400f0a8
:109ee0007a007b00123952900414e4f0a3f090043d
:109ef00010f090040e74ff129f4112397deefaefbc
:109f0000fb1237138532828533835392fe029c9b6a
:109f10002436f582e43ff58322ee2413f582e43ff4
:109f2000f58322ee241cf582e43ff58322ee242af9
:109f3000f582e43ff58322ee2412f582e43ff583b7
:109f400022f07b018e828f83a3a3a3a3a3a3a3a349
:109f5000e0fa79002285848285858312ac27e87532
:109f6000f005a4f8aaf075f005e9a42af9ee24306a
:109f7000f582e43ff58312b28dee2274f612229e32
:109f8000eafeebff75210575220078211224e67c9c
:109f9000007d00ee24b1fae43ffb121cd8740212db
:109fa000221c78211224e67c007d00ee24a1fae434
:109fb0003ffb121cd8740212221c900491e0a2e014
:109fc0005004788080027800ee24b5129fe6481293
:109fd0009fee5004780080027880ee24a5f582e49c
:109fe0003ff583028406f582e43ff583e022f0909a
:109ff0000491e0a2e02274f612229e74fe1222372f
:10a000001224d212a0c944c0129fee4007aa84ab0a
:10a01000851216de75210078211224eae4f52278f3
:10a02000211224e61217daeafcebfd7406f9aa8481
:10a03000ab851216c0740302b39374f612229e7499
:10a04000fe1222371224d274ff122206ea853282cf
:10a05000853383f012a16675210178211224ea74f8
:10a06000011222848821892278211224e61217da2b
:10a07000eafcebfd740df9aa84ab851216c07403db
:10a0800012221c02b39174f612229e74fe12223721
:10a090001224d212a0c9d2e6f07521007821122430
:10a0a000eae4f52278211224e61217daeafcebfd45
:10a0b0007405f9aa84ab851216c0740312221caa77
:10a0c00084ab851216de02b396e912a16b12a0d101
:10a0d00022e5842411f582e43585f583e02274f6c7
:10a0e00012229e74fe1222371224d2e9feeaffeefb
:10a0f00012a167ef7036e5a8f521c2af7a06eef936
:10a100001216ea858482858583a3a3a3a3a3a3a3b0
:10a11000a3a3a3e4f0e58412aaee3585f583e05409
:10a12000e7f0e521a2e7a2e792af8037e58424803b
:10a13000f521e43585f52278211224e6e584249082
:10a14000fce43585fdaa21ab221212d6740212223c
:10a150001c900491e0a2e0eef950051216f0800385
:10a160001216e402b396e912a16b2275f0e6a4f888
:10a17000a9f090045ee028f584a3e039f58522c0bb
:10a1800082c083ea4b603fea2426f582e43bf583f4
:10a190005392fee0a2e7500e9004c5e0f97cbf7d2b
:10a1a0000412149280208a828b83a3a3a3e0540319
:10a1b00024fe6005146007800a1213b4800812168a
:10a1c000a880031217e00285ac74f412229ea2af9d
:10a1d000e433fec2af9004bce0700ceea2e092af9c
:10a1e0009004bee4f0803aeea2e092af1217daeaf1
:10a1f0004b602e1216c6ea4b60031216fca2afe4a7
:10a2000033fec2af9004bce014f070079004bee4cb
:10a21000f080097b007a00790012397deea2e0928d
:10a22000af02b210c082c08312170202b2f674f6f7
:10a2300012229e74fe1222371224d2e9feeaffeea9
:10a2400012a343e5822411f8e43583f988848985d3
:10a25000ef604614604914605214606914606d1414
:10a26000601e14606e14700302a2f214700302a246
:10a27000f914700302a30014700302a31e02a32e9c
:10a28000e582243dfae43583fb1215faea4b7003ac
:10a2900002a32e1216fc02a32e12170202a32ee016
:10a2a000d2e5f0eef91213a802a32e0592900491c4
:10a2b000e0a2e0500354fef00592e0c2e5f0eef9b2
:10a2c0001213ae8069eef91213ba8062eef912131e
:10a2d000c0805be582245efce43583fde582246674
:10a2e000f58250020583059212a3eeeef91218d002
:10a2f000803ceef91213c68035eef91213d2802e8f
:10a30000059290041412b12ff9121780900414e4ee
:10a31000f0a3f090041012a3311213a28010e5a84c
:10a32000f8c2af0592900367e0c2e012a33a02833d
:10a3300050f0900491e054fef022f0e8a2e7a2e78a
:10a3400092af2212a3472212a34b2275f0e6a4f883
:10a35000a9f0059290045ee028f582a3e039f58328
:10a360002274f712229ee9feea4b600aea24fcf806
:10a37000eb12a3df500eec4d600eec24fcf8ed1256
:10a38000a3df400479008054ee9003f66005e0d22c
:10a39000e18003e0c2e1f0ea4b60069003fe12a602
:10a3a000c4ec4d60089003faecf0a3edf09003fece
:10a3b00012a3ee9003f112ac23c3ea98eb99500676
:10a3c0009003f112a6c47409122270e09003f660a3
:10a3d00005e0d2e58003e0c2e5f0790102ab8c1222
:10a3e000899b94fde9943f22853282853383e0fa8c
:10a3f000a3e0fb2274f112229e74fe122237122473
:10a40000d2eaffe912a6cae521240afce43522fdbe
:10a410008c828d830592e0f8740868607c7409680a
:10a4200070028075e5a8fec2af852182852283a3d4
:10a43000a3a3a3a3a3a3a3a3858225858326eff0cb
:10a4400012a6b8e5212430f584e43522f58505927d
:10a45000e0f8a3e0f912a4ac3522f58512a93b126d
:10a46000217b12ab14128b038c828d837408f0ee67
:10a47000a2e7a2e792af75240178241224ea782596
:10a480001224e61217daeafcebfd7402f9aa21abfa
:10a49000221216c0740312221c8532828533831265
:10a4a00024da740212221c7f07022376e521241e7f
:10a4b000f584e42274f012229e74fe1222371224d4
:10a4c000d274fe12220612ab0412a9190592e07092
:10a4d00008900491e0a2e05004793a80651217dafe
:10a4e00012ab68700479078059e5a8f523c2af79eb
:10a4f00000ee2444fae43ffb12162a12a925122189
:10a500007b12a6da50010912a911128b0c85278241
:10a510008528837406f0e523a2e7a2e792af7523ae
:10a520000878231224ea12a54778231224e6790832
:10a53000740312227012a9411216c0740312221c55
:10a540007900740202a94dee2444f523e43ff5247a
:10a550002274f012229e74fe1222371224d274fb4f
:10a56000122206e9853282853383f012a6ca05924b
:10a57000a3a3a3a3a3a3a3a3a3a3e06005793a0283
:10a58000a6b57417122270e0f523a3e0f524741920
:10a5900012227012b27d78231224e68e258f26783f
:10a5a000251224e67407122284882589267825122c
:10a5b00024e612165a740612221ce9600302a6b59c
:10a5c0001217da740112227012a6c47401122270da
:10a5d00012ab757005790702a6b512a6b878007996
:10a5e0007d12a4ac352212a93712217b12a6da50b3
:10a5f0000109128b03e521244cf527e43522f528c7
:10a6000075250975260078251224e6e521241bfc12
:10a61000e43522fdaa27ab28121cd2740212221c98
:10a62000740312227012ac23e521244f128b07e52c
:10a6300021245312a6bceef0a3eff0e52124511221
:10a64000a6bce523f0a3e524f0e521244d12a6bc29
:10a65000e4f0a3f08527828528837402f0e5a8fa48
:10a66000c2af12a6b8e5212420f584e4352212aa4f
:10a6700065500109e5212455128b07852182852229
:10a6800083a3a3a3a3a3a3a3a3a3a3740112aa4870
:10a6900075230b78231224ea78271224e6790074b4
:10a6a0000412227012a6d4aa21ab221216c074037f
:10a6b00012221c790002a94be521242ef582e435f3
:10a6c00022f58322eaf0a3ebf02212a34785822130
:10a6d00085832222e0fca3e0fd22892612a9093508
:10a6e00026f9e82401082274f612229ee9fe75215b
:10a6f0001075220078211224e612975e2480fae475
:10a7000039fb121cd202b39f74f012229e74fe1207
:10a7100022371224d274fd122206853282853383b9
:10a7200012a6c47402122270e9f08c238d2412aa9e
:10a730005f900491e0a2e0500b12a3e81217e079b9
:10a740000c02a9058e828f83a3a3a3a3a3a3a3a313
:10a75000a3a3e0600b12a3e81217e0793a02a9055f
:10a76000ee241112a919e0c2e4f0d2e312ae0f12e6
:10a77000a92e12217b892212a9093522f9e8240188
:10a780000850010912a911128b0cee2466f584e41d
:10a790003ff585ee245ef525e43ff526ec45247073
:10a7a0003075210875220078211224e67c007d0096
:10a7b000aa25ab26121cd8740212221c752102781d
:10a7c000211224e67c007d00aa84ab85121cd8806f
:10a7d0002f75210275220078211224e6aa84ab8508
:10a7e000121cd2740212221c75210878211224e650
:10a7f000e5232402fce43524fdaa25ab26121cd255
:10a80000740212221cee2470f584e43ff58579046d
:10a81000aa84ab851219e4ee2468f521e43ff52201
:10a820007908aa21fb1219e4852782852883e0a2f2
:10a83000e7503fe5a8f8c2af8e828f83a3a3a3a3fe
:10a84000a3a3a3a3a3a3740512a33a75220078229d
:10a850001224eae4f523f52478231224e6790a7415
:10a860000312227012a9411216c0740312221c0294
:10a87000a90375230875240078231224e6ac21adc2
:10a8800022ee2490fae43ffb121cd2740212221c26
:10a8900075210475220078211224e6ac84ad85ee82
:10a8a00024b6fae43ffb121cd2740212221c782157
:10a8b0001224e6ac84ad85ee24a6fae43ffb121c1c
:10a8c000d2740212221ce5a8f521c2af8e828f83ba
:10a8d000a3a3a3a3a3a3a3a3a3a37403f075221606
:10a8e00078221224ea78251224e67903e9122270ec
:10a8f00012a9411216c0740312221ce521a2e7a27c
:10a90000e792af7900740380440592e028f8a3e051
:10a9100022ee2434f582e43f22f527e43ff5288532
:10a920002782f58322ee242ef582e43ff58378001a
:10a93000797dee12a4ae3ff5850592e0faa3e0fb27
:10a9400022e0fca3e0fdeefaeffb22740512221ccc
:10a950008532828533831224da740212221c7f0826
:10a9600002237674f012229e74fe1222371224d231
:10a9700074fc122206740212227012a6c4892112db
:10a9800017da12ab687005790702aa43e52112aa0b
:10a990005fa3a3a3a3a3a3a3a3a3a3e060108532f3
:10a9a00082853383e0fa1217e0793a02aa43ee2453
:10a9b0002ef523e43ff52485238212a92c12217b56
:10a9c00012a6da50010912a911128b0cee2457f5c8
:10a9d00027e43ff52875250575260078251224e61d
:10a9e000740412227012a6d4aa27ab28121cd274a7
:10a9f0000212221ce5a8fac2af852382852483eec9
:10aa00002420f584e43f12aa65500109ee245cf588
:10aa100082e43ff583e812aa51a3a3a3a374021210
:10aa2000aa4875230778231224ea78271224e679a6
:10aa300001740312227012a9411216c0740312226b
:10aa40001c7900740402a94df0eaa2e7a2e792afd4
:10aa50002212b28e8e828f83a3a3a3a3a3a322125a
:10aa6000ab0c059222f5850592e0f8a3e0f9e82801
:10aa7000f8e933f905921297712407f82274f2125b
:10aa8000229e74fe1222371224d212ab04f525e462
:10aa90003ff526852582f5830592e0700bee12aa1c
:10aaa000ee129fe9a2e05004793a80351217da8a53
:10aab000238b24ac23ad24ec4d7004790780221243
:10aac000a92512217b12ab14e824010850010912b8
:10aad000aae412aaf47407f0eefaeffb12176879f1
:10aae00000029c95ee2434f582e43ff58322241184
:10aaf000f582e422e8f0a3e912aafc22f08525827f
:10ab000085268322e912ab0cee240a2212a34bae57
:10ab100082af8322892412a9093524f92274f712fd
:10ab2000229e74fe1222371224d275846775850422
:10ab300080048884898585848285858312ab7560cd
:10ab400017ea687002eb6970e98a828b8312ab5b4b
:10ab50008a828b83e4f0a3f002972e12ac278584bf
:10ab60008285858312b28d22853282853383eaf015
:10ab7000a3eb1290ab12ac27e849228532828533d1
:10ab8000835392fe1224da740212221c7f010223e4
:10ab90007674f412229e74fe1222371224d28a8412
:10aba0008b85a2afe433f521c2af90046012ac23d1
:10abb000858482858583a3a3ae82af83e849702c08
:10abc000e594a2e24009759403e594a2e250fa7973
:10abd0000012198a8b24ea2404f8e4352412ac12fa
:10abe000123713e5e170fc75e106801d88828983c8
:10abf000a3a312a3ee88828983a3a3a3a3e02af8c8
:10ac0000a3e03b12ac12123713e521a2e092af028f
:10ac1000b202f98e828f8312b28daa84ab8522f0a4
:10ac20009003fa12ac2722e0f8a3e0f92274f312a1
:10ac3000229e74fe1222371224d2eafeebff8925ef
:10ac4000ee2437fce43ffd8c848d850592e0f5828f
:10ac5000a3e0f5839061d0e0f87480c398fae582b0
:10ac600045836023e5822424f584e43583f585e07b
:10ac7000547ff9900460e0f8a3e0c82408f584e468
:10ac800038f585e069600302aded858284858385b2
:10ac9000a3a3a884a985e0fb8a217524002402f5da
:10aca0002350020524c3e5219523e49524a2d2650f
:10acb000d033404ceac39b24fefa74012bf5d985ae
:10acc0008284858385a3a3a3e0f5d97b008012e568
:10acd000822bf584e43583f585a3a3a3a3e0f5d9fe
:10ace0000b88848985e0f521ebc3952140e1e5e1fe
:10acf00070fc75e19585828485838512ae03708a28
:10ad0000a882a9838c828d83e80592128b0fe5259a
:10ad1000700302aded900491e0a2e0400302adedbe
:10ad2000900493c3e09402a3e09400500302adedbd
:10ad3000e5945404f521700e12ae25400975940374
:10ad4000e594a2e250fa1219908a238b24a823a931
:10ad500024c3e89401e99400a2d265d03340731271
:10ad6000b021ecfaedfb12217be89402e99400405b
:10ad700061e8fae9fb8c21ea8cf0a4caacf08df012
:10ad8000a42cfc8521f0eba42cfb8e828f83a3a343
:10ad9000c3e09af0a3e09bf0900493c3e098f0a383
:10ada000e09912ae0fc3e098f0a3e099f09004afe1
:10adb000e0c0e012adf9d0e0f0eefaeffb122b7d2f
:10adc000ee2412129fe6d2e3f0e5e170fc75e14259
:10add000801be5217017e5a8f8c2af12b493e59483
:10ade000a2e25003759402e594a2e240fa85328211
:10adf0008533835392fe02857bee242bf582e43f5c
:10ae0000f58322e0f582a3e0f583e582458322f015
:10ae100012ae1422ee242ef582e43ff583229061d7
:10ae200082e4f0a3f0e5a8f8c2af9004d4e0d2e049
:10ae300012b49de594a2e222e5e170fc75e191e592
:10ae4000e170fc75e1810285b0e5e170fc75e1918e
:10ae50000285b074f612229e74fe1222371224d29a
:10ae6000906002740ff012b27aee242b129fe60467
:10ae7000f064037002e4f0e02425906000f0900894
:10ae800009122089906195122095900495e0540153
:10ae9000f9121636ee240bf521e43ff522ee2412ca
:10aea000f584e43ff5850592e0a2e0e433f9aa21b8
:10aeb000ab2212163c12175c75d923900495e0f86a
:10aec000a2e050047a4080027a000592e0a2e050ad
:10aed000047c8080027c00ea4c4405f5d9e8a2e0bd
:10aee00050067a9d7b0480047a977b0479061216bb
:10aef000127906aa21ab221216127904ee2414fa52
:10af0000e43ffb1216127903ee2418fae43ffb1219
:10af100016127909ee241bfae43ffb12161279058a
:10af2000ee2424fae43ffb121612ee2429129fe6c7
:10af300044a0f5d9e5e170fc75e19590600d74c110
:10af4000f090046780068584828585831289138545
:10af50008482858583a3a3a3a3a3a3a3a3a882a973
:10af600083e58445856005e0a2e740da12b021e57b
:10af700084458560710592a3a3858482858583902d
:10af800003ef12a93b0592e0c39afaa3e09bfbea08
:10af90002cfaeb3dfb8882898312b0161221f3ea6a
:10afa000c39521faeb9522fb8e828f83a3a3a3a3e3
:10afb000a3a3a3a312b0161221f3ea2521f8eb35bf
:10afc00022f9ecfaedfb12217b8a218b22a821a920
:10afd00022e89404e994005006e82cf8e93df9e8e9
:10afe00024fcf8e98005ec24fff8ed34fff9900427
:10aff00000128b0e90600e128b0ea3ecf0a3edf0fe
:10b0000075910090618274c0f075a100c2c275a7ed
:10b0100002d2ba02b396e0f52175220074027821bb
:10b020002212b030e0fca3e0fdec2cfced33fd225d
:10b03000ee241ef582e43ff5832274f612229e74fc
:10b04000fb122206ec4d604a8532828533837406fa
:10b05000f07401122270744712b09c7403122270b3
:10b060007403f0a37401f0ea12aaee3bf583e0d278
:10b07000e0f075210578211224ea740112228488f7
:10b0800021892278211224e6790c1216c074031249
:10b09000221c740502b3a19004937401f0a3e4f0a0
:10b0a0002274f712229e90046012ab75700479002e
:10b0b000801b9004d4e0a2e050047902800f900439
:10b0c000a71220718a828b8312207d790102ab8cba
:10b0d000c082c0835392fe90046012b12f2410608e
:10b0e0002a24fc600624fc60198029e5e170fc90ac
:10b0f0000416e0f87411129b6d3408f583e0f5e155
:10b10000802ae5e170fc75e1168021e5e170fc75af
:10b11000e1178018900491e0a2e05009e5e170fc8d
:10b1200075e1108007e5e170fc75e11102b2f6e00f
:10b13000f8a3e0c82408f582e438f583e02274f629
:10b1400012229ee9fec394035020ee900490f07505
:10b15000212575220078211224e67c007d007a6b7f
:10b160007b04121cd8740212221c02b3a474f412c1
:10b17000229e74fe1222371224d212a1668003127c
:10b1800017e0e584243dfae43585fb1215faea4b15
:10b1900070ed1297fb1215faea4b60081217e08067
:10b1a000f11217e01297f11215faea4b70f3858449
:10b1b00082858583a3a3a3a3a3a3a3a385822385b9
:10b1c0008324e0ff7521e675220078211224e67cb5
:10b1d000007d00aa84ab85121cd8740212221cefd9
:10b1e000852382852483f090046912ab5b90046907
:10b1f000e584f0a3e585f09004c7e014f080031225
:10b20000221c8532828533831224da740212221cb6
:10b210007f0402237674f412229e74fe12223712e7
:10b2200024d290046912b27dee4f60488e828f83e3
:10b2300012b2838e848f850592a3a3a3a3a3a3a395
:10b24000a3e0f5217523e6752400059278231224e6
:10b25000e67c007d00eefaeffb121cd8740212228d
:10b260001ce5210592f0129f1974800592f090045c
:10b27000c7e004f0eefaeffb8088900404e0fea340
:10b28000e0ff2212ac2790046912b28d22e8f0a3ed
:10b29000e9f022c082c0835392fe906184e4f09072
:10b2a00061a0e0f8e4f0e5e170fc75e1029061bfb7
:10b2b000e060fae0f5bce0f5bc80159061bf12b229
:10b2c000e612b2e6e5bc8a828b83f0a3aa82ab8346
:10b2d000e9fc74ff2c190470e2e5e170fc75e101f2
:10b2e000e89061a0800fe0f5bde0f5bde0f5bde0c0
:10b2f000f5bd22f0a3f0d083d08202112974f6129a
:10b30000229e900490e06402703c78008007740be9
:10b31000687002780ce8c333241a906184f0e5e188
:10b3200070fc75e10290618ee0f974806960f6e965
:10b330008a828b83f0a3aa82ab8375e10108e8c3fc
:10b340009426501980c87521257522007821122471
:10b35000e67c6b7d04121cd2740212221c7521251e
:10b3600075220078211224e67c007d007a6b7b0434
:10b3700002801874f612229ee9fe752105752200de
:10b3800078211224e61297622424fce439fd02a7f6
:10b3900002740112221c8532828533831224da74ee
:10b3a0000212221c7f02022376c082c0835392fec7
:10b3b0009004a3e08a828b83f09004a412b3d7f0a8
:10b3c0009004a512b3d7a3f09004a612b3d7a3a3f9
:10b3d000f01225cb02b2f6e08a828b83a322c082d0
:10b3e000c083e975f0e6a4f8a9f05392fe12976abb
:10b3f0002413f582e439f583e0f902b2f674f4120d
:10b40000229e74fe1222371224d28c848d85e97517
:10b41000f0e6a4feaff0752306752400782312240d
:10b42000e612b450240bfce439fd121cd274021253
:10b43000221c12b4502412f582e439f583e0a2e014
:10b44000e4330592f0853282853383059202b20897
:10b4500090045ee02ef8a3e03ff9e822c082c083aa
:10b460005392fe90605ae402b2f3c082c083e5e1d9
:10b4700070fc75e101e5a8f8c2af5392fe12b493d7
:10b4800090605a12a3ee906058e412b512a3f0a394
:10b4900002b2f39004d4e0c2e012b49d22f07534fd
:10b4a00000e8a2e7a2e792af2274f712229e12ae42
:10b4b0001e40037594019060517401f0a37484f0f0
:10b4c00090605fe4f0906053f090605e7403f090e1
:10b4d00061e9e4f090081512207190619512207dc9
:10b4e00012b50ae9c333f8e9c394149061a6500772
:10b4f0007420f074188004e4f0741628906184f0cd
:10b50000e5e170fc75e11802ab8c906054e4f0a3a7
:10b510007455f0a3f0a3f02274f412229e8921ea5c
:10b52000ffebfe12ae1e4003759401906051740350
:10b53000f0a37493f090605e7403f0906053e4f0b5
:10b540009061e9f09008151220899061951220957c
:10b5500012b50ae521c333f8e521c394149061a61e
:10b5600050077405f074188005740ff07416289055
:10b570006184f0e5e170fc75e1f174022ff5d98e7c
:10b58000d98fd978008004e4f5d908e8c39f501f0b
:10b59000ee600814601114601280ec7419129b6d37
:10b5a0003408f583e080e1740f80dd745580d9e5bf
:10b5b000e170fc75e19574036e906190700de0d2be
:10b5c000e5f0e5e170fc75e104800be0c2e5f0e533
:10b5d000e170fc75e11979701219a802b21074f5c6
:10b5e00012229eeafeebff8923e9c3941140037502
:10b5f000231085232175220078211224e6121cd203
:10b60000740212221c741065236026852382aa828c
:10b610007410c39af52195e0f52278211224e67c76
:10b62000007d00ee2afae43ffb121cd874021222bd
:10b630001c02ba7874e812229e74fe122237122479
:10b64000d274fb1222068a298b2a752b00752c00d6
:10b650008a828b83782112203be5c7c0e0740412f4
:10b660002270d0e0f0900368e0f5c78a828b83a354
:10b67000a3a3a3e0fa8529828b838a25e4f526f526
:10b6800027f5287825121f6490f7e8e0f52de4f5fa
:10b690002ef52ff530740b782d121f327825792d69
:10b6a000121d58500302b7ea8529848b850592a3a1
:10b6b000a3a3a3a305929008937821121f64eafe26
:10b6c000e5215403fc700302b75574031222707411
:10b6d000fff0740212227074fff0740112227012d3
:10b6e000b82f8c82aa82740412bfb750057404c3a9
:10b6f0009cfe8e2575260078251224e6ac84ad8547
:10b700007402122270e5822afae43583fb121cd2fd
:10b71000740212221c7904ac32ad338521258522b6
:10b720002685232785242874027825121f19aa2527
:10b73000ab26121426e5842ef584e43585f585853f
:10b740002982852a83a3a3a3a3e0c39efe90089722
:10b750007821121f64eec394044031eef9ac84ad3d
:10b76000858521258522268523278524287402782e
:10b7700025121f19aa25ab261214268e25e525545d
:10b78000fcf8e58428f584e43585f58574035efcd2
:10b79000605e740312227074fff0740212227074df
:10b7a000fff0740112227012b82f8c2575260078d4
:10b7b000251224e6ac84ad85740212228c121cd2b0
:10b7c000740212221cac32ad338e25e4f527f52825
:10b7d00078217925121f5174027821121f19aa218c
:10b7e000ab227404f91214268006752b80752c0187
:10b7f0007404122270e0f5c790063ee52bf0a3e535
:10b800002c12ca3e740712cf731224e612ccd11246
:10b81000229c740212221c740512221c853282851d
:10b8200033831224da740212221c7f1002237674ee
:10b83000fff0853282853383f02274e812229e74f1
:10b84000fe1222371224d274c01222068a828b83ff
:10b850008582848583850592a3a3a3a3e0fee5c723
:10b86000ff900368e0f5c790f7e8e0f525e4f526da
:10b87000f527f528740b7825121f32eec39441404a
:10b88000027e400592782912203b78257929121de5
:10b8900058400302b962852921852a22852b2385f8
:10b8a0002c248e2de4f52ef52ff5307821792d12ec
:10b8b0001f5178217925121d585005e529f404fe01
:10b8c0009008937829121f64852921852a22852bc7
:10b8d00023852c24740f7821121f19e521f5238567
:10b8e00023c7ac29e52a4480fd8e828582257526f2
:10b8f00000ec2ef521e43df522c3e5259521e495e4
:10b9000022500c78251224e6740212228c8049e51c
:10b9100025c39521f525e49522f52678251224e600
:10b92000740212228c121cd2740212221c74012581
:10b9300023f5c778211224e67c007d80c3e495219d
:10b94000fae49522fb7402122270e5822ef8e435a7
:10b9500083f9e82afae93bfb121cd2740212221c7a
:10b9600080027e008fc7ee90063ef0f525f582ac92
:10b97000827d00240112bca6f526f5279008977851
:10b9800025121f6474087825121f32782179251238
:10b990001fdc90089b7821121fef90063a78211245
:10b9a000204aa832a9338821892278211224e67af4
:10b9b0003a7b06790512ccdb12229c740212221cff
:10b9c000744002b81974f512229e74fe12223712c6
:10b9d00024d2eafeebff7523008e828f83a3e0fb67
:10b9e00074ff6b601e7c007d007a0479008e828f6c
:10b9f00083e025e012c78a12cce012229ce9700392
:10ba00007523018e828f83a3a3e0fb74ff6b6034e8
:10ba10007c007d007a0379008e828f83e025e0fe32
:10ba2000e433ff74e72ef58474083ff58505921220
:10ba3000cce012229ce97004d2f08002c2f0a2f0a5
:10ba4000e4334223e523a2e05006788079018004a4
:10ba50007800790012ba7d740e12cf731224e612a8
:10ba6000ccd112229c740212221c8532828533832f
:10ba70001224da740212221c7f0302237690063eff
:10ba8000e8f0a3e912d45de4f0a32274ec12229e44
:10ba900074fe1222371224d274c01222068a848bba
:10baa00085858482858583a3a3a3a3e0f8c39440fe
:10bab000500488218003752140e5c7f522858482e2
:10bac000858583782512203b740f7825121f19e590
:10bad00025f5c7852182ae828e2375240078231236
:10bae00024e6858482858583782512203bac25e574
:10baf000264480fd740212228c121cd2740212227f
:10bb00001c8522c785848285858312208990063e04
:10bb1000122095ee900642f02405e43400f526e468
:10bb2000c526f525e4f527f528e0f529e4f52af5fd
:10bb30002bf52c90089f7829121f649008a3782970
:10bb4000121fc974087829121f3278257929121f0b
:10bb5000dc9008a77825121fef90063a782512206e
:10bb60004aa832a9338823892478231224e6eefcdc
:10bb70007d007a3a7b06790912ccdb12229c740292
:10bb800012221c744012221c8532828533831224b7
:10bb9000da740212221c7f0c02237674f612229ea3
:10bba00074fe1222371224d274f91222061216548d
:10bbb0007f007e00ac32ad33740112228ceef9129c
:10bbc000197ee9601c740112228c853282853383d0
:10bbd000e0f9121648e9600890063e12d40c800e77
:10bbe0000f0eeec3940840cc90063ee4f0a3f0efb5
:10bbf000a312d435740712cf731224e67c007d00a3
:10bc00007a3a7b06790712ccdb12229c740212224c
:10bc10001c7407800e12cf731224e612ccd11222ac
:10bc20009c740212221c8532828533831224da74ba
:10bc30000212221c7f0202237674ec12229e74fef2
:10bc40001222371224d2e9fe8c258d2690063eea78
:10bc5000f0a3ebf0eea3f0f529f582ac827d002491
:10bc60000312bca6f52af52bf52c9008ab78291207
:10bc70001f6474087829121f3278217929121fdc79
:10bc80009008af7821121fef90063a782112204acf
:10bc900078251224e67a3a7b06790712ccdb122249
:10bca0009c740202bb85e43400f522e4c522f52130
:10bcb000e4f523f5242274f612229e74fe12223734
:10bcc0001224d274fc122206ea14600614603b02ad
:10bcd000bd63900607e024026005146009800e90a1
:10bce000063e7484800c90063e748a800590063e61
:10bcf000748512cf661224e612ccd112229c7402f3
:10bd000012221c900607e4f080597e00aa32ab3361
:10bd1000eef9121978e96044ee90063e12c7e990f8
:10bd2000063ff07401122270e05401900640f07456
:10bd300003122270e090064112cf7c740412ca38bc
:10bd40001412cf731224e67c007d007a3a7b0679c8
:10bd50000812ccdb12229c740212221c0eeec39439
:10bd60000840a9740402bc2374f212229e74fe12cd
:10bd700022371224d28922ebfeea600d24fb6029cf
:10bd800014700302bf5e02bf7a900607e0fa7440a7
:10bd900012bfb7400302bebee0f87440c398f5245a
:10bda00002bec090060774fef0ee700302bf7a90e8
:10bdb0000607e0a2e75027eec3944140047f40808d
:10bdc00002eeff7cc77d05effb12bf8f12cce012a5
:10bdd000229ce9cec39efe700302bf7a80d9c39431
:10bde00004504ce0701605929008b31224f97b01c0
:10bdf0007a0079081219ba740412221c900607e01e
:10be0000f87404c39812bfc2500ae0f87404c398cf
:10be1000f52180028e2112bfacab2112bf8f12cc54
:10be2000e012229ce9cec39efe900607e029f0e0d6
:10be3000c39404500302bda9e0640470189005c7c0
:10be4000e0600302bda3a3e0c3943d400890060751
:10be500074ff02bda8900607e0f89005c8e024042e
:10be6000c398f8c39e5004882480028e24e8601e84
:10be700090060712bfacab2412bf8f12cce0122287
:10be80009ce9f8e524687006900607e029f0e524af
:10be9000cec39efe900607e0fa9005c8e079002424
:10bea000045001096a49600302bda9900607e0f940
:10beb0007ac77b05121aa4900607e402bda88e2457
:10bec000e524c39e500302bf5a85242575260078b9
:10bed000251224e674c72afae43405fb121cd27436
:10bee0000212221c900607e02524f0e0c3940450bf
:10bef0000302bf7a9005c8e0fc900607e0faec2444
:10bf000004f8e43400f9ea98e499406e74042cf5de
:10bf100024f97ac77b05121aa4a824900607e0c367
:10bf200098f07c00900607e0f8ecc39850bd8c8236
:10bf3000a882852425e82525fae43400fb74c72a65
:10bf4000f58274053bf583e0c0e074c728f582e410
:10bf50003405f583d0e0f00c80ca7900801ee5c777
:10bf6000f525900368e0f5c790ff25e0f974ff69b7
:10bf700060057a00121ba68525c779018532828566
:10bf800033831224da740212221c7f060223767a8b
:10bf9000027900e52225e0f525e433f52674e7254e
:10bfa00025f58474083526f585059222e0f874c7d6
:10bfb00028fce43405fd22c39a12bfc2a2d265d088
:10bfc0003322f895e0f98e25c3e89525e9940022ff
:10bfd00074f612229e74fe1222371224d28a828ba9
:10bfe000837c007d00e0f8c3940340057c800d80d5
:10bff000548582848583850592a3a3e870150592f4
:10c00000a3e0f58f0592e0600553f7df803743f733
:10c0100020803274016870150592a3e0f5f6059250
:10c02000e0600553f7bf801d43f7408018e06004cf
:10c03000780080027880e5f75460fa0592a3e05416
:10c040001f484af5f712c34612c36d740502bc15aa
:10c0500074f612229e74fe1222371224d28a828b28
:10c06000837a007b00e0600814600f146016801e65
:10c0700012c09f558048f580801712c09f55904888
:10c08000f590800d12c09f55a048f5a080037a80de
:10c090000b90063eeaf0a3eb12c36d1402bc1585ab
:10c0a00082848583850592a3e0f90592a3a3e059d4
:10c0b000f8e9f42274f512229e74fe12223712243b
:10c0c000d28a218b228a828b83a3a3a3a3a3ac82cf
:10c0d000ad838a828b83a3a3a3a38a848b850592d5
:10c0e000a3a3a3a884a9858a848b85a3a3aa84abd0
:10c0f00085852184852285a3ae84af8585218485ad
:10c100002285e0701475864275c40212c132f5c5ed
:10c110008c828d83e0f5c2801275f84275fb0212a5
:10c12000c132f5fc8c828d83e0f5fa12db560402f5
:10c13000ba590592e0541ff52188828983e0c433ff
:10c1400054e0f88a828b83e0c4333354c0f98e8282
:10c150008f83e0a2e0e4331313494845212274f0b1
:10c1600012229e74fe1222371224d28a848b858575
:10c170008482858583a3aa82ab83e0c39441402255
:10c1800090063e748212d3e112c7baa3e412cf8a9a
:10c19000f0a3740412db597409f0e4f521f52202ce
:10c1a000c2457c00800c8df9a2f840fce5f90592af
:10c1b000f00c8a828b83e0f8ecc398502f8c82a815
:10c1c00082e58428f582e43585f583a3a3e0fd7438
:10c1d0008728f8e43405f9888289830592e070c6df
:10c1e0008dc1e586a2e040fae5c180c290063ee43a
:10c1f000f0a312c7ba8a828b83e0f525900641f03e
:10c20000752200240450020522e4c522f521e4f53c
:10c2100023f524f526f527f5289008b77825121f71
:10c220006474087825121f3278217925121fdc905a
:10c2300008bb7821121fef90063a782112204a7528
:10c24000218775220578211224e690064112ca1e24
:10c25000790812ccdb12229c740212221c853282d5
:10c260008533831224da740212221c7f080223769b
:10c2700074f612229e74fe1222371224d28a828b06
:10c28000837c007d008582848583850592a3a3a39a
:10c29000a884a985858284858385a30592e014609e
:10c2a0000a24fe604914606b02c3380592e0f52150
:10c2b000c39405400302c33812c355c0e074a025df
:10c2c00021f582e43462f583d0e0f088828983121c
:10c2d000ca180592e025e0f8e433f974a628f5823f
:10c2e000746239f583ea0592f0a3ebf0804d059274
:10c2f000e0f521c39402504012c34e700b8acc88e3
:10c30000828983e0f5cd80338ace88828983e0f507
:10c31000cf80280592e0f521c39402501b12c34e32
:10c32000700b8aec88828983e0f5ed800e8aee88b6
:10c33000828983e0f5ef80037c800d12c34612c32f
:10c340006d740d02bc1512db0eecf0a3ed2212c3ce
:10c3500055fae521220592a3a3e054073333335461
:10c36000f844042290063ee521f0a3e52212d45db4
:10c370007407f0a32274f012229e74fe1222371268
:10c3800024d274a5122206e9feeaffeec3941240fd
:10c390000302c785746512d3e6343d12d3eb500314
:10c3a00002c7858c848d850592a3a3a3a3ee059275
:10c3b000122510001185c7dbc3e9c30ac454c48f1a
:10c3c000c4c3c418c553c55dc5a0c5e1c50ac635fb
:10c3d000c640c6f0c6fac616c756c70592e0f9129f
:10c3e0001a027901745b02c25a12c7af0412cf73ea
:10c3f0001224e67c007d007a3a7b06790412ccdbbd
:10c4000012229c740212221c80d879067cea7dffdd
:10c41000741512228c1213fc7521067522007821e6
:10c420001224e674171222947a3e7b06121cd274f0
:10c430000212221c90063ae412d6ace412d40cf09c
:10c44000e4f52178211224e67c007d007a3a7b060f
:10c45000790a80a98584828585830592a3a3e0c09b
:10c46000e00592e0f584a3e0f585d0e00592f005c3
:10c470009212cf8412d44be4f0a3740312cf731240
:10c4800024e67c007d007a3a7b06790602c3fd85ae
:10c490008482858583e0f8a3e0f988848985900605
:10c4a0003ee8f0a3e912c7ba90063a12c7d3740463
:10c4b00012cf731224e67c007d007a3a7b0679075e
:10c4c00002c3fd740112228c12179e740112227095
:10c4d000e090063ef07402122270e090063ff07485
:10c4e00003122270e0900640f07404122270e09073
:10c4f0000641f01217d4e990064212cf4a12d42e08
:10c50000e4f0a3740512cf731224e67c007d007a58
:10c510003a7b06790902c3fd121390e912d4201266
:10c52000cf6e1224e67c007d007a3a7b06790512f4
:10c53000ccdb12229c740212221c121390e9f8e543
:10c5400021c398400302c3e27a00a921121b5e05b1
:10c550002180e7aa84ab85121a2602c3e279017c06
:10c56000e77dffaa32ab331213fc90063e74011232
:10c57000c7d1740212c7dc747a12c7d10412c7e99a
:10c5800090064912db40740c12c7dc740812cf739a
:10c590001224e67c007d007a3a7b06791002c3fd06
:10c5a000858482858583e0f8c394065028e582243b
:10c5b00002fce43583fda3e0fb7a017900e8281250
:10c5c000c78a12cce012229ce960067800790080cc
:10c5d00008788780027880790112ba7d740902c4d4
:10c5e0007caa84ab858a828b83a3a3a3a3a3a3e0a5
:10c5f000f9121648e990063e600512d40c8003e457
:10c60000f0a312ba84740a02c47c8584828585836f
:10c61000aa82ab83a3a3a3a3a3a3e0f912164ee9b6
:10c6200090063e600512d40c8003e4f0a312ba8495
:10c63000740b02c47c12165412c7af740c02c3ed03
:10c640008584828585837521007522007800e0f558
:10c6500023c39406502e741b122294a3e0fb7a028b
:10c660007900e52325e0f523e433f52474e7252359
:10c67000f58474083524f585059212cce012229ccd
:10c68000e9f8800675218075220190063ee521f0cb
:10c69000a3e522f0e812ca2750020522e4c522f5dc
:10c6a00021e4f523f524f526f527f5289008ab7845
:10c6b00025121f649008a37825121fc974087825d5
:10c6c000121f3278217925121fdc9008bf782112c1
:10c6d0001fef90063a782112204a741b1222848898
:10c6e00021892278211224e6900640e0fc02c4b899
:10c6f000aa84ab85121a2002c3e2858482858583d1
:10c70000e0f9a3ac82ad837a777b05121a0e12c7cb
:10c71000af740f02c3ed12c79f12228c121a0e744f
:10c72000051222848821892278211224e6740712b6
:10c7300022947a777b051212d6740212221c12c739
:10c74000c37410f078211224e67c107d007a3a7bc5
:10c7500006790502c3fd12c79f12228c121a0e74ad
:10c76000051222848821892278211224e674071276
:10c7700022947a777b051212dc740212221c12c7f3
:10c78000c3741180be790002c3e4f521e433f522bd
:10c7900074e72521f58474083522f58505922285f4
:10c7a0008482858583e0f9a3ac82ad8374052290f1
:10c7b000063ae4f0a3f0a3f0a322f00592e005927c
:10c7c000a3f02290063e741012db44741112c7dcf1
:10c7d00022f0a3e4f0a3740312c7dc22f0a3e4f078
:10c7e000a322e8f0a3e912d41912c7ed22f0853292
:10c7f00082853383e02274ef12229e74fe12223768
:10c800001224d274c0122206e9fec3940940030226
:10c81000ca0d749712d3e6343df583e493f8eac366
:10c8200098500302ca0d8c848d850592a3a3a3a3ff
:10c83000ee603014607014700302c8cf14700302ed
:10c84000c8da14700302c92114700302c9a214705b
:10c850000302c9b414700302c9f914700302ca03b5
:10c8600002ca0d12180412ca2ee4f0f521f522783e
:10c87000211224e67c007d007a3a7b06790412ccf2
:10c88000db12229c740212221c7901744012221cb9
:10c890008532828533835392fe1224da7402122287
:10c8a0001c7f09022376059212ca2e12cf7312241e
:10c8b000e67c007d007a3a7b06790412ccdb1222fa
:10c8c0009c740212221c7a327b1a12181c80ba1233
:10c8d000183a12ca2e04f0e48091858482858583fb
:10c8e000a3a3e0f9e5822403fce43583fd0592125d
:10c8f000ca18121816e96006780079008004788258
:10c90000790190063ee8f0a3e912ca3e740312cf03
:10c91000731224e67c007d007a3a7b06790602c811
:10c920007e7940ac32ad3312d68f12182ee9f874ee
:10c93000ff6870067a807b0180047a007b00900695
:10c940003eeaf0a3ebf074ff6870047f00800ce80f
:10c95000c394405004e8ff80027f40ef12ca275082
:10c96000020522e4c522f521e4f523f524f526f598
:10c9700027f5289008ab7825121f647408782512d3
:10c980001f3278217925121fdc9008c37821121fed
:10c99000ef12dcfc1224e690064012ca1e79070250
:10c9a000c87e7cff7dff12d68f12183412ca2e74f7
:10c9b0000502c8d6752100752200e5c7f52305924a
:10c9c000900368e0f5c70592e0f9059290f7e8e07a
:10c9d000f8e9c3985009743029f9121420800675bb
:10c9e00021807522018523c790063ee521f0a3e54d
:10c9f0002212ca3e740602c90eaa84ab85121a140a
:10ca000002c889aa84ab85121a1a02c88979000261
:10ca1000c88b858482858583e0faa3e0fb22e0fc55
:10ca20007d007a3a7b0622a312ccbd240322900615
:10ca30003ae4f0a312ca3822f0a304f0a32212d4dd
:10ca40005d14f0a32274f012229e74fe122237129b
:10ca500024d274df122206e9feeaffeec3940640f8
:10ca60000302ccb874af12d3e6343d12d3eb5003bb
:10ca700002ccb88c828d83a3a3a3a3ee601e1460a6
:10ca80007514700302cbaf14700302cc3c14700316
:10ca900002cc6c14700302cc7f02ccb8aa82ab83a8
:10caa0008a848b850592a3a3a3122501ea2404fca2
:10cab000e43bfd8a828b830592a3a3e0f98a828bf3
:10cac0008312ca1812155e740112221c12cceae4f9
:10cad000f0f521f52278211224e67c007d007a3ad7
:10cae0007b06790612ccdb12229c740212221c797e
:10caf00001742102c25a85828485838585328285ac
:10cb00003383742012d268a3858221858322a832c0
:10cb1000a9338823892478231224e67403122294eb
:10cb2000852182852283e0f912ca1212154c740203
:10cb300012221c12ccc4e8f0a3e9f08521828522e0
:10cb400083e0f8a3e0f990064012c7e29006441291
:10cb5000ccbd240750020522e4c522f521e4f523cb
:10cb6000f524f526f527f5289008c77825121f64c7
:10cb70009008a37825121fc974087825121f3278ef
:10cb8000217925121fdc9008cb7821121fef900627
:10cb90003a782112204a740112228488218922784d
:10cba000211224e690064412ca1e790b02cae485bb
:10cbb0008284858385853282853383742012dd0dde
:10cbc0001224e6740312229412ca1212155274022d
:10cbd00012221c12ccc412c7e290064212ccbd2411
:10cbe0000550020522e4c522f521e4f523f524f5dc
:10cbf00026f527f52890089f7825121f649008a332
:10cc00007825121fc974087825121f3278217925da
:10cc1000121fdc9008cf7821121fef90063a78217e
:10cc200012204a7401122284882189227821122438
:10cc3000e690064212ca1e790902cae485828485fa
:10cc40008385a3a3e0fbe5842403fce43585fd1282
:10cc5000d3fe12159a12d4450412cf731224e67c27
:10cc6000007d007a3a7b06790402cae485828485d5
:10cc7000838512d4041215a012d445740480daa856
:10cc800082a983888489850592a3a3a3122501e83c
:10cc90002404fce439fd888289830592a312ca1812
:10cca00088828983e0f9121558740112221c12cc73
:10ccb000ea7405f0e402cad1790002caf1f0f52560
:10ccc000752200220592e0f8a3e0f9059290063e55
:10ccd000227c007d007a3a7b067906059290064e0a
:10cce000e0f582a3e0f58305922212d456f0a32248
:10ccf00074f412229e74fe1222371224d274fb1294
:10cd00002206e9feeaffeec39409400302cf217434
:10cd10008e12d3e6343d12d3eb500302cf218c8226
:10cd20008d83a3a3a3a3ee6030146071147003027b
:10cd3000cded14700302ce3814700302ce58147077
:10cd40000302ce8514700302cea714700302ceca6c
:10cd500014700302cf0402cf218582848583857af3
:10cd6000130592e0f912145c0592e0059212d412b8
:10cd700012cf60e4f0f521f52278211224e67c0040
:10cd80007d007a3a7b06790712ccdb12229c740272
:10cd900012221c7901740512221c02cf8f85828415
:10cda000858385121390e9f80592e0f9c398400451
:10cdb000787f801512138ae970047800800b059241
:10cdc000e0f91217a4e92499f843920112cf28e858
:10cdd000a312cf4a12d44b0412d3e112cf73122400
:10cde000e67c007d007a3a7b067906809b8582216d
:10cdf0008583228521848522850592a3a3a3a3a3ed
:10ce0000a3a31224fd852184852285a3a3a3a3a324
:10ce10001224fd852182852283059212d25212149a
:10ce200056740412221c85218285228312d4111289
:10ce3000cf6014f0e402cd758582848583850592e8
:10ce4000e0f912173e12cf2d6005f87902800478c0
:10ce500000790012cf5b80db858284858385aa32ce
:10ce6000ab330592e0f912179812cf26a37405127e
:10ce7000cf4a12db597403f0a30412dd0d1224e62d
:10ce80007c0502cde385828485838512cf3c121711
:10ce900038e96005f8790280047800790012cf261d
:10cea00012cf5b7405808c8582848583850592e032
:10ceb000f912172012cf2d6005f87902800478004e
:10cec000790012cf5b740602ce33858221858322de
:10ced000e090063e12cf4f740712db371224e67c37
:10cee000007d007a3a7b06790512ccdb12229c7415
:10cef0000212221c7a00852182852283e0f9121b0e
:10cf00005e02cd9390063e748312cf4f740812cf09
:10cf1000731224e67c007d007a3a7b06790502cd07
:10cf200088790002cd95059212cf35f02212cf33c9
:10cf3000f0e9220592e0059290063e22e584240263
:10cf4000fae43585fb0592e0f92212cf8ae4221239
:10cf5000cf8ae412ca387403f0a322a3e8f0a3e94d
:10cf600012d43df0a32212d3e112cf7c740212c777
:10cf7000dc7406f0e4f521f52278212212cf8a74c0
:10cf800080f0a32290063ee4f0a3f090063a2285ba
:10cf900032828533831224da740212221c7f040247
:10cfa000237674f412229e74fe1222371224d2e9e0
:10cfb000feeaffeec3940c400302d208747712d34a
:10cfc000e6343d12d3eb500302d2088c828d83a34a
:10cfd000a3a3a3ee604514700302d088147003026b
:10cfe000d0b814700302d0e614700302d106147096
:10cff0000302d11714700302d13d14700302d164ef
:10d0000014700302d18514700302d19914700302c5
:10d01000d1c814700302d1e202d20885822185832f
:10d02000228521848522850592a3a3a3a3a3a3a37c
:10d03000122501e521240812d21a1224e685218442
:10d040008522850592a3a3a3a3a31224fd85218293
:10d05000852283059212d25212151c740512221ccd
:10d0600012d271e4f0f521f52278211224e67c0039
:10d070007d007a3a7b06790712ccdb12229c74027f
:10d0800012221c790102cf8f85822185832285217e
:10d09000848522850592a3a3a3a3a312250112d2fe
:10d0a000161224e612d24c121516740312221c1208
:10d0b000d2717401f0e480ad8582218583228521bf
:10d0c000848522850592a3a3a3a3a312250112d2ce
:10d0d000161224e612d24c121510740312221c12de
:10d0e000d271740280ce85828485838512d20d85ab
:10d0f000848285858312d24112150a0592e0059239
:10d1000012d2781480ae12d23b1215048584828527
:10d11000858312d277809d85822185832285218413
:10d120008522850592a3a3a312250112d2261214eb
:10d13000f8740112221c12d2710402d0b48582212b
:10d140008583228521848522850592a3a3a31225a8
:10d150000112d2261214e0740112221c12d2717430
:10d160000602d0b4e0f91214da12d4527404f0a317
:10d17000740712cf731224e67c007d007a3a7b0696
:10d18000790602d07812d23b1214fe8584828585fe
:10d190008312d277740802d0b485822185832285d8
:10d1a00021848522850592a3a3a3a3a3122501129e
:10d1b000d2161224e612d24c1214ec740312221c62
:10d1c00012d271740902d0b485828485838512d409
:10d1d000041214f285848285858312d277740a0240
:10d1e000d0b485828485838512cf3312d268e0fc67
:10d1f00012cf3c1214e690063feaf0a3eb12db508c
:10d2000012ca38740b02d0b4790002d085a3a3a34c
:10d21000e0fca3e0fd22e5212406f523e43522f518
:10d22000240592782322e5212404fce43522fd859f
:10d230002182852283059212d25f22858284858392
:10d2400085a3e0faa3e0fb0592e0f922852182851f
:10d25000228312d20d85218285228312d25f22a3de
:10d26000e0fa12db04e0f922f0858482858583a34d
:10d2700022852182852283e012d41612d43d04f047
:10d28000a32274f612229e74fe1222371224d2e9cf
:10d29000feeaffeec39408400302d3dc74a012d36d
:10d2a000e6343d12d3eb500302d3dc8c828d83a392
:10d2b000a3a3a3ee602714606114607a14700302c4
:10d2c000d36814700302d37514700302d3941470de
:10d2d0000302d3bd14700302d3d602d3dc8582844b
:10d2e00085838512d4041218fa8584828585831279
:10d2f000d41112d435e4f0f521f52278211224e678
:10d300007c007d007a3a7b06790712ccdb12229ce6
:10d31000740212221c790102bc26e0f91218ee12e6
:10d32000d428740112cf731224e67c007d007a3a6f
:10d330007b06790480d4e0f91218e8e990063e6093
:10d3400005e4f0a38005748012d3e112cf4a12d411
:10d350004b740512d40c12cf731224e67c007d00ae
:10d360007a3a7b06790680a212d3f41218f412d40a
:10d3700028740380af858284858385a31220598514
:10d380008482858583e0f912190612d4527405f05f
:10d39000a31480c212186ae9f5217b02fa790812f7
:10d3a000397de52112d42012d42e12cf731224e637
:10d3b0007c007d007a3a7b06790502d30a85828457
:10d3c0008583850592e0f9a3aa84ab8512187012b3
:10d3d000d4280402d324121a2c02d315790002d3c4
:10d3e00017f0a374012229f582e422f583e493f86f
:10d3f000efc39822858284858385a3a3e0fb85847f
:10d4000082858583a3e0fa0592e0f922f0a37402f5
:10d4100022e012d4162290063ef0a3eaf0a3eb22fb
:10d4200090063e12db44042290063ae4f0a3f0a3f7
:10d430007405f0a32212d43d7405f0a32212db4838
:10d440007403f0a32290063ae4f0a3f0a37402f070
:10d45000a32212d4562290063eeaf0a3eb12db4838
:10d460007402f0a32274f612229e74fe1222371266
:10d4700024d274ff122206e9feeaffeec3940b40a9
:10d480000302d68a748312d3e6343d12d3eb5003e1
:10d4900002d68a8c828d83a3a3a3a3ee603c146082
:10d4a0007514700302d53914700302d54514700346
:10d4b00002d5b414700302d5bf14700302d606144b
:10d4c000700302d61214700302d63214700302d60f
:10d4d0005114700302d67302d68a858284858385af
:10d4e00012d40412146e90063ae4f0a312d6ace4ff
:10d4f000f0f521f52278211224e67c007d007a3aad
:10d500007b06790412ccdb12229c740212221c7955
:10d5100001740102bc2385828485838512d40412a0
:10d52000148612d6c8740112cf731224e67c007dd3
:10d53000007a3a7b06790680cbe0f912146812d69d
:10d54000c8740280e2aa82ab83ea240df584e43b2e
:10d55000f58505921224fdea240bf584e43bf5855c
:10d560001224fd8a848b85a3a3a3a3a3a3a3a3a3af
:10d570001224fd8a848b85a3a3a3a3a3a3a31224af
:10d58000fd74081222948a828b830592a3a3a3a31d
:10d59000a3a3e0f9121450740812221c12d6b3741b
:10d5a0000312cf731224e67c007d007a3a7b067961
:10d5b0000702d50412146212d6c8740402d527a833
:10d5c00082a983888489850592a3a3a3a3a3a31218
:10d5d00024fd88848985a3a3a3a31224fd888489bc
:10d5e00085a3a31224fd888489851224fd74081262
:10d5f000229479007a007b00121450740812221cc5
:10d6000012d6b314809b12d3f412147412d6a5024e
:10d61000d527858284858385a3a3a312d69b12d2a6
:10d62000100592a3a312d68f12142c12d6c804028e
:10d63000d527858284858385a3a3a312d69512d28c
:10d6400010059212d68f12143812d6c8740802d55b
:10d650002785828485838512d6950592e0aa82abc0
:10d66000836005121690800312168a12d6a57409db
:10d6700002d527aa82ab83a3a3a3a3a3a3e0f91295
:10d68000148012d6c8740a02d527790002d511e099
:10d69000faa3e0fb2212d69ba3a322a3e0f9858480
:10d6a000828585832212db6012d6ac22f0a3740639
:10d6b000f0a32290063eeaf0a3eb12c7ed900640dd
:10d6c00012d43d7406f0a32212d4567406f0a3229d
:10d6d00074ee12229e74fe1222371224d274e012cb
:10d6e0002206e9fec39415400302daff745012d3f8
:10d6f000e6343df583e493f8eac398500302daff79
:10d700008c828d83a3a3a3a3aa82ab83ee122510e0
:10d710000014ffda3ed7acd7e2d72ed873d8b8d8ea
:10d72000bed8c4d81dd923d929d9b5d9f9d920da79
:10d7300026da3dda54da70daaddad8daefda8a844a
:10d740008b8575210075220012d3fe121b9ae960a9
:10d7500018858482858583a3a3e0fa8584828585e4
:10d7600083e0f9121ba0e970067521807522011271
:10d77000c364e4f0f521f52278211224e67c007dd3
:10d78000007a3a7b06790612ccdb12229c740212d4
:10d79000221c7901742012221c8532828533831267
:10d7a00024da740212221c7f0a022376eafcebfdc3
:10d7b0008c848d850592a3a3a3a3a31225018c823b
:10d7c0008d830592a3a3a3a3e0f98c828d831220fd
:10d7d00059121b88740112221c12db567401f0e4ea
:10d7e00080928a218b2212db56740212db371224bc
:10d7f000e67c007d007a3a7b06790690064ee0f5dd
:10d8000084a3e0f58585848285858312229c740239
:10d8100012221c852182852283a312db04a3e0fa55
:10d82000852182852283e0f9121b8202d7928a84a5
:10d830008b857a007b00858482858583a30592e0b1
:10d84000601c14601214701d0592e0541ff8e5ff6f
:10d8500054e048f5ff80110592e0f5fe800a05923c
:10d86000e0f5fd80037a800b12db1512c36d7403a3
:10d8700002d7de8a848b857a007b00858482858549
:10d8800083a30592e0601c14601214701d0592e0e1
:10d890005407f8e5ff54f848f5f580110592e0f5d6
:10d8a000f4800a0592e0f5f380037a800b12db1511
:10d8b00012c36d740402d7de121a4402d792121af0
:10d8c0004a02d7928a828b83780079007a00e060de
:10d8d0000e14600714700de5a08006e5908002e547
:10d8e00080fa8003788009059290063ee8f0a3e96b
:10d8f000f00592e00592900640f00592a3e05a9060
:10d90000064112db40740412db5912cf731224e675
:10d910007c007d007a3a7b06790802d787121a507c
:10d9200002d792121a5602d7928a848b85858482f6
:10d93000858583a3a3e0f8c394205004e8ff800208
:10d940007f20effcaa32ab330592e0f9121bb8e955
:10d95000f525f5290592a3e06003121bd012db0e1a
:10d96000e4f0a3f0e529a3f075220024035002059a
:10d9700022e4c522f521e4f523f524f526f527f563
:10d98000289008ab7825121f6474087825121f327e
:10d9900078217925121fdc9008d37821121fef120d
:10d9a000dcfc1224e6900640e0fc7d007a3a7b061f
:10d9b000790702d7878a848b85858482858583a3ae
:10d9c000a3e0fce584240312cf40121bbee9f5213d
:10d9d0000592a3e06003121bd0e5215392fe12d4fe
:10d9e0002012db59740b12cf731224e67c007d00e9
:10d9f0007a3a7b06790502d7878a828b83e0f9120f
:10da0000168490063ae4f0a312db59740c12cf731b
:10da10001224e67c007d007a3a7b06790402d787df
:10da2000121a5c02d79212db1d121b9ae97006755e
:10da3000218075220112c364740e02d7de12db1d31
:10da4000121ba0e9700675218075220112c364744f
:10da50000f02d7de8a828b83e06005121bd680031b
:10da6000121bdc90063ae4f0a312db597410809d7f
:10da7000752100752200752300121be2e96008126f
:10da80001be8e9f523800675218175220190063e89
:10da9000e521f0a3e522f0e523a312db5012db59c8
:10daa000741112cf731224e67c0002d9aa752100ea
:10dab0007522008a828b83e06013121be2e9600505
:10dac000121bee800b7521817522018003121bf45d
:10dad00012c364741202d7de8a828b83e0f91216b5
:10dae0007e90063ae4f0a312db59741302da0d902b
:10daf000063e748312d3e112c36d741402d7de792b
:10db00000002d794a3e0fb852182852283225392d1
:10db1000fe90063e2212db0eeaf0a3eb228a828bf5
:10db2000837521007522008582848583850592a3f3
:10db3000e0fa0592e0f922f0e4f523f524782322b7
:10db400012db442212db4822f090063ae4f0a322d2
:10db500012db4474032212db60f0a37407f0a322eb
:10db600012cf84f0a374022274f012229e74fe126b
:10db700022371224d274db122206e9feeaffeec33a
:10db80009407400302dcea74a812d3e6343d12d3b2
:10db9000eb500302dcea8c848d850592a3a3a3a33a
:10dba000ee602114606a14607514700302dc3b148b
:10dbb000700302dc4514700302dc7014700302dc95
:10dbc000dd02dcea858482858583a3a3e0fb858270
:10dbd0008485838512db2f1217c212dcefe4f0f587
:10dbe00021f52278211224e67c007d007a3a7b061a
:10dbf000790412ccdb12229c740212221c7901746b
:10dc00002512221c8532828533835392fe02c26321
:10dc1000e0f91217bc12dcef7401f0e480c11217b6
:10dc2000b612d452740812d40c12cf731224e67cac
:10dc3000007d007a3a7b06790680b71217b012dcb5
:10dc4000ef740380d5aa32ab3312179290063e745c
:10dc50002512db407426f0a37408f0a3740412ddcf
:10dc60000d1224e67c257d007a3a7b0679058082b8
:10dc70008584828585830592e0f525059290063e90
:10dc8000f0752200240150020522e4c522f521e4aa
:10dc9000f523f524f526f527f52890089778251221
:10dca0001f649008a37825121fc974087825121fd5
:10dcb0003278217925121fdc9008d77821121fefc6
:10dcc00090063a782112204a0592a3858221858305
:10dcd0002278211224e690063ee0fc8089e0f912c9
:10dce000177a12dcef740602dc1a790002dbff906f
:10dcf000063ae4f0a3f0a37408f0a32290063ae5f4
:10dd000021f0a3e522f0a3e523f0a3e524f0a83257
:10dd1000a9338821892278212274f612229e74fe6a
:10dd20001222371224d2e9feeaffeec394045052c5
:10dd300074b512d3e6343d12d3eb4046ee600b14bb
:10dd4000601a14602f14603380388c828d83a3a3f3
:10dd5000a3a3e0f9121a02790102bc2612dd86742f
:10dd60000112cf731224e612ccd112229c7402123b
:10dd7000221c80e312dd86740280e612dd867403c5
:10dd800080df790080d390063e748112d3e112d4f3
:10dd90005d7409f0a32274f712229eeafeebffe9fc
:10dda000601d14602314602914602f146035146002
:10ddb0003b14604114604714604d146053805aef67
:10ddc000faeef9121a628053effaeef9121a68802d
:10ddd0004aeffaeef9121a6e8041effaeef9121ad2
:10dde000748038effaeef9121a7a802feffaeef912
:10ddf000121a808026effaeef9121a86801deffac9
:10de0000eef9121a8c8014effaeef9121a92800bc6
:10de1000effaeef9121a98800279007f0102237658
:10de200074f612229e74fe1222371224d28a848b38
:10de300085e9fe7b017a0079081219aeac84ad85c4
:10de400074fc2efb858482858583a3a3a3e0fa0559
:10de500092a3a3e0f9121a9ee9701690063e74840c
:10de600012cf661224e612ccd112229c7402122226
:10de70001c02bc2674f712229ee9feea24fcfceb8d
:10de800034fffd7bffee75f01984aaf075f019eef2
:10de900084f9121a9e808474f012229e74fc12225d
:10dea00006e5c7fe12ec12501190f7e912208985a1
:10deb0003282853383122095802e7904aa32ab33c7
:10dec0001219e4853282853383782512203b90082d
:10ded00073782112203b78257921121e1785328212
:10dee000853383782112204a8ec785328285338319
:10def000122059740402eacd74f712229e9004dfb6
:10df0000e0f5217900800774ff2521522109e521e0
:10df100070f502fa4174f612229ee99004e170064f
:10df2000e054fbf08019e0440412f8871224e6ea7a
:10df3000fcebfd7ae37b04121cd2740212221c0259
:10df4000f87974f612229e7900752101752200e994
:10df500078211221f39004dfe05521600709e9c31d
:10df6000940840e5740869700279ff02f879c021cd
:10df7000e9faa2e050057521038003752100a2e1b2
:10df80005004780c80027800e84221eaa2e25004b2
:10df9000781080027800e84521f9d0215392fe02e2
:10dfa000112974f712229e74fe1222371224d2e92c
:10dfb000fe752100740b12227012ea67802a8521f7
:10dfc00082a882e58428f582e43585f583e0ffecbc
:10dfd00028f582e43df583e06fc0e0ea28f582e4ad
:10dfe0003bf583d0e0f00521e521c39e40d002fa45
:10dff0003374f712229e752100801c852182ae8227
:10e00000ec2ef582e43df583e0f8ea2ef582e43b60
:10e01000f583e068f00521e521c39940de02fa416d
:10e0200074f612229e74fe1222371224d28a848b36
:10e030008575210875220078211224e67af37b0485
:10e04000121cd2740212221c78211224e67c007d5c
:10e05000007afb7b04121cd8740212221c7521f377
:10e0600075220478211224e67cf37d04aa84ab8512
:10e070001212d6740212221c9004f3e0faa3e0fb01
:10e0800002f86b74f612229e74fe1222371224d20a
:10e09000eafeebff9004f3ecf0a3edf0740c122217
:10e0a0007012eb01f99004f512ede675210c752262
:10e0b0000078211224e67c007d007af77b04121c94
:10e0c000d8740212221c740e12227a05921224fdb8
:10e0d0007cf37d04eefaeffb1212d6740202fedf2f
:10e0e00074f412229e74fe1222371224d28a848b78
:10e0f00085740e122270e0f521a3e0f5228c238da9
:10e100002478231224e67910900361e0240212e4bb
:10e110007aaa21ab22121882740212221c782112d0
:10e1200024e6ac21ad22aa84ab851212d674021269
:10e13000221c900495e0a2e050067c9d7d048004a2
:10e140007c977d04900491e0a2e050047a00800264
:10e150007a067906e5212afae43522fb121888901e
:10e160000491e0a2e050047e0680027e00790690d1
:10e170000363e075f0e6a4faabf090045ee02afadf
:10e18000a3e03bfbea240bfce43bfde5212efae493
:10e190003522fb12188878211224e6ac21ad22aa80
:10e1a00084ab851212d6740212221c02fe6974f628
:10e1b00012229e74fe1222371224d28a848b857515
:10e1c000210375220078211224e67af37b04121cc5
:10e1d000d2740212221c75210d78211224e67c00d3
:10e1e0007d007af67b04121cd8740212221c752161
:10e1f000f375220478211224e67cf37d04aa84ab13
:10e20000851212d6740212221c7521037522007821
:10e21000211224e67cf37d04740e122270e0faa32e
:10e22000e0fb121cd202e0db74f612229e74fe1296
:10e2300022371224d212fa10640a752110752200b6
:10e240007821600302e2e61224e6900361e02442b2
:10e2500012ea5d121cd2740212221c7521f375227f
:10e260000478211224e612f2ae12189a74021222d5
:10e270001c75211075220078211224e612e71a7a03
:10e28000f37b04121ccc740212221c8b22ea45225e
:10e29000600302e33712f649aa84ab851219307580
:10e2a000210875220078211224e612e3b9121cd24b
:10e2b000740212221c12e7248a218b227821122454
:10e2c000e612e4701212d6740212221c12f66e12ba
:10e2d00024e612e3a2121cd8740212221c12e709cf
:10e2e000740bf002e39f1224e6900361e0243212e3
:10e2f000ea5d121cd2740212221c7521f3752204ed
:10e3000078211224e6900361e0243212f2b412184c
:10e310009a740212221c7521107522007821122491
:10e32000e612e4667af37b04121ccc740212221cff
:10e330008b22ea4522600b7904aa84ab851218c4ab
:10e34000805d75210875220078211224e612e3b958
:10e35000121cd2740212221c12edec12ea368582d3
:10e360002185832278211224e612e470aa21ab22af
:10e370001212d6740212221c12f66e1224e612e356
:10e38000a2121cd8740212221c12e7097406f07c37
:10e39000007d00900363e0f9aa84ab851217320276
:10e3a000f86b7c007d00900361e02af8a3e0340064
:10e3b000f9e82453fae439fb2212f64d900361e0a8
:10e3c000244afaa3e03400fb2274f612229e74fe63
:10e3d0001222371224d212fa106404752110752209
:10e3e00000782170251224e6900361e0242212eacd
:10e3f0005d121cd2740212221c12e470aa84ab8536
:10e4000012193012e7097405804c1224e69003615a
:10e41000e0241212ea5d121cd2740212221c12fabb
:10e420002764097034900361e02422f521a3e034cd
:10e4300000f52278211224e6900361e0243212f2e2
:10e44000b412189a740212221c12e466aa84ab85d4
:10e4500012192a12f297f0800a7408f0aa84ab8588
:10e460001217e002f86b900361e0242212e47a2292
:10e47000900361e0244212e47a22fca3e03400fd20
:10e480002274f012229e74fe1222371224d274fcdf
:10e490001222068a278b288a828b83a3a3a3a3a395
:10e4a000a3a3a3a3ae82af83a3a3a3a3e0f974f8ad
:10e4b0005970108e848f850592a3a3a3a3a3e05463
:10e4c000f86005790a02e60712187c12ea700592d4
:10e4d000e0f912187c12ea6bf07a0090618fe0c0cc
:10e4e000e012ea432442f582e439f583d0e0f00af1
:10e4f000eac3941040e575210675220078211224a4
:10e50000e6eefceffd900361e0240c12ea5d121cc4
:10e51000d2740212221c12edec240bf582e438f5c1
:10e5200083740212eab3c0e012ea89d0e0f09004ea
:10e5300095e05401c0e012e709a3d0e0f075211086
:10e540008e828f83a3a3a3e0f894105002882174d5
:10e55000f928c3940a400302e5f58e828f83a385d0
:10e560008225858326e0700d9004e1e05404600567
:10e57000790202e6038e828f83a3a385822385839b
:10e580002412fd9c82f0500f12eabd700a12187618
:10e5900012ea64e90592f012ea521219e49004e1d9
:10e5a000e0f85404600d852582852683e060047eb2
:10e5b000048037852382852483e0a2e24005e85465
:10e5c0000260259004dee0fc8e828f83e075f0050a
:10e5d000a4faabf0745a2afa74083bfbea2cf582d1
:10e5e000e43bf583e0fe80027e009004e0e0fae583
:10e5f00021c39a50047906800ae85402600fee7035
:10e600000c7903aa27ab281218c402e70112eaa367
:10e61000e521f0ee70047a0080027a0112edec241c
:10e6200068f584e438f58585848285858312ea76e9
:10e6300012e72474046e7523107524007823701279
:10e640001224e67ce37d04121cd2740212221c0206
:10e65000e6e21224e67c007d00121cd8740212222d
:10e660001cee607e14600c14602d14600614607241
:10e6700002e70112e7097403f0900363e0fef91268
:10e680001b0a900363e06e6005eef91213f0aa27ef
:10e69000ab281217e0806a121864eaf8ebf9ecfa7a
:10e6a000edfb853282853383122095752304782310
:10e6b0001224e6740212229412edf9121cd2740292
:10e6c00012221c900363e0fe853282853383122080
:10e6d00059eef9121b10900363e06e6005eef9121b
:10e6e00013f012f29d1224e612f2ae12189a74027e
:10e6f00012221c12e71aaa27ab2812192a12f29129
:10e70000f0740412221c02eac212e70d2212e71171
:10e710002212eafef5838882a322900361e024128c
:10e7200012e47a2212edf012ea3aaa82ab83227442
:10e73000f012229e74fe1222371224d274fc12228e
:10e74000068a278b288a828b83a3a3a3a3a3a3a3d0
:10e75000a3a3ae82af8312191e12f175601d05923c
:10e7600012f17d40168b237905aa27ab281218c415
:10e7700012ea64e5230592f002ea257522108e82e2
:10e780008f835392fea3a3a3e0f8c3941050028892
:10e790002274f928c3940a4004790680149004e195
:10e7a000e0f88e828f83a3e07011e85404600c7946
:10e7b00002aa27ab281218c402ea258e828f83a3ef
:10e7c000a3e0a2e092f0e8a2e082f0502e74ff6b8a
:10e7d000702912187612ef0f12eabd701e05929082
:10e7e0000363e0f5217a8b7b0179ff121b229003f2
:10e7f00063e065216005a9211213f012ea52121993
:10e80000e412eabd60258e828f830592a3a3a3a3a1
:10e81000e0f912187c12ea708e828f83a3a3a3a35f
:10e82000a3e0f912187c12ea6b800a059212eaf54d
:10e83000c812fb55e4f075250675260078251224cc
:10e84000e6eefceffd900361e0240512ea5d121c88
:10e85000d2740212221c12ea89a37401f09004956a
:10e86000e05401c0e012ea89d0e012eab3c0e0123d
:10e87000e709a3d0e0f07a0090618fe0c0e012eaef
:10e88000432432f582e439f583d0e0f00aeac394f8
:10e890001040e59004e1e0f85404600d8e828f830f
:10e8a000a3e0600575210480398e828f83a3a3e0e5
:10e8b000a2e24005e8540260268e828f83e0fa903f
:10e8c00004dee075f005a4f8a9f0745a28f874087d
:10e8d00039f9e82af582e439f583e0f521800375fa
:10e8e000210012eaa3e522f0e52170047a008002fb
:10e8f0007a0112edec2468f582e438f58385828490
:10e9000085838512ea768e828f83a3a3e0fa12eaca
:10e91000bd7004eac2e0fa05929004e1e05402609e
:10e9200004ead2e2fa8e828f83a3a3a3a3a3e0fd1d
:10e930008e828f83a3a3a3a3e0fceaf9aa27ab28c6
:10e940001219249004e0e0f8e522c39812eafe5080
:10e950000812ea8f740602ea24c812ea36aa82abc9
:10e9600083e52170139004e1e05402602212eafe74
:10e9700012ea8f740302ea2474046521701175256c
:10e980001078251224e67ce37d04121cd2800f75da
:10e99000251078251224e67c007d00121cd8740214
:10e9a00012221c900363e0fee521607314602714bb
:10e9b0006008146005146067806b12e7097407f043
:10e9c000900363e0f9121b0a900363e06e6056ee59
:10e9d000f91213f0804f121864eaf8ebf9ecfaed33
:10e9e000fb853282853383122095752504782512a4
:10e9f00024e6740212229412edf9121cd27402124f
:10ea0000221c853282853383122059900363e0f9fa
:10ea1000121b10900363e06e6005eef91213f01202
:10ea2000e7097409f0740412221c8532828533834d
:10ea30005392fe02eac812ea3a222453f582e438dd
:10ea4000f58322eaf8900361e028f8a3e03400f9a6
:10ea5000e82279025392fe900361e02465faa3e074
:10ea60003400fb2290036112ef1c2212eb06e92214
:10ea700012fb4ee9f022e054fef8a3e0f9e84a85e3
:10ea8000848285858312ede72212e70da3a322f588
:10ea9000838882a3740cf012edf02452f582e438de
:10eaa000f5832212eaa72212edf42467f582e438f6
:10eab000f58322f012f18c12f414e4332212fb627b
:10eac000f4228532828533831224da740212221ce6
:10ead0007f08022376c082c0835392fe12fb4ae471
:10eae000f012eaf5f5838882a3e4f0121918d083b6
:10eaf000d08202112912eb06e4f012eafe22900302
:10eb000061e0f8a3e02212edf412eb0d222463f58c
:10eb100082e438f5832274f412229e74fe122237a6
:10eb20001224d2eafeebff89211218be12fdbdf5b8
:10eb300022e5216005fa7b0380047a007b00e0f97e
:10eb4000121b22900363e065226005a9221213f0d4
:10eb50008e828f83a3a3a882a98312f7058584825e
:10eb600085858312f8e10592a3e521f002fe5e742b
:10eb7000f712229e74fe1222371224d274ea122255
:10eb8000069004e07407f09004dfe4f09004de7473
:10eb900003f0e5c7f812ec1250059004dee4f088ab
:10eba000c779017cdf7d047a027b0012182e853242
:10ebb0008485338590085474061220aef521a8216f
:10ebc000e828f8e433f9853282853383e58228f535
:10ebd00082e58339f583e0fea3e0ff79007c007dc8
:10ebe00000eefaeffb12182ee9f470187910740693
:10ebf00012228c12178c79107406122294eefaeffe
:10ec0000fb1218160521e521c3940340b1741602c6
:10ec1000fa30900368e0f5c790f7f4e0a2e62274ba
:10ec2000f212229e74fe1222371224d274f412229f
:10ec300006853282853383eaf0a3ebf0e9fe8c236c
:10ec40008d24900363f075f06fa4f8a9f09003652c
:10ec5000e028f8a3e039f990036112ede6f5838826
:10ec600082a3e0f8740b686005740668700b12edff
:10ec7000f9eef912172c02edc7ee75f0e6a4f521b6
:10ec8000e5f0f522900491e0a2e0400302eda975c1
:10ec9000250275260078251224e674021222947447
:10eca0000412228c121cd2740212221c75250878c0
:10ecb000251224e6ac23ad247406122270aa82ab7e
:10ecc00083121cd2740212221c7c0a740212228c3f
:10ecd00079861218288a828b83e582458370237a8d
:10ece00000eef91216f6900363e0ff7a087b03f951
:10ecf000121b22900363e06f6005eff91213f0021c
:10ed0000edcea3a3e0c0e012ea64d0e00592f07972
:10ed10001074021222947a067b0012182eac23add6
:10ed200024740212228c12188e8a238b24a823a901
:10ed30002485328285338312f65a12f64012ede6ac
:10ed4000791074021222947a057b0012182e12f4a4
:10ed50004f2480f523e439f52478231224e6e4f5e2
:10ed600023f52478231224e612edec12f839740608
:10ed700012228c121894740412221c12eaa312f6a6
:10ed80007df52395e0f52478231224e67c007d00b0
:10ed900012f44f2af8e439f9e82480fae439fb1236
:10eda0001cd8740212221c801e791090045ee0258b
:10edb00021faa3e03522fbea2480fce43bfd12fbb0
:10edc0005efb7a8012182e7a01eef91216f6740c98
:10edd00012221c8532828533831224da74021222b5
:10ede0001c7f06022376e8f0a3e9f02212edf02260
:10edf00012edf42212eafec82212f2bb2274f412bf
:10ee0000229e74ed122206eafeebff7521007523a7
:10ee100001752400e52178231221f39004dfe055e9
:10ee200023605a79107403122294ab217a8312184a
:10ee30002ee9f46048a832a9338823892478231264
:10ee400024e6ee2403fce43ffd740512228c121824
:10ee5000a0740212221c7523037524007823122447
:10ee6000e6eefceffd740212228c121ccc7402122e
:10ee7000221c8b24ea45247004a921800b0521e57e
:10ee800021c39408408879ff741302fe7474f6124b
:10ee9000229ee9701579817c061218288a828b835c
:10eea000e5824583702179ff80218a828b83a3a329
:10eeb000a3a3a3e054c024c06008248070e8798232
:10eec00080d51218d68004a3a3e0f902f87974f76c
:10eed00012229e74fe1222371224d212f196f58469
:10eee000a3e03912f42012f16ee584240bfae43524
:10eef00085fb1218dc12ef0f12f717600612fb38b1
:10ef000012182e8532828533835392fe02fa39120b
:10ef1000ef19e90592f0059222900361e0f584a3d0
:10ef2000e0f5852274f612229ee9fe74ff6e7015dc
:10ef30007c807df07a807b001218349004dfe4122c
:10ef4000f434fb802f752101752200ee7821122107
:10ef5000f3af219004dfe05f70047900801b7c80b8
:10ef60007dff7a80e9fb121834eff4f89004dfe0bb
:10ef70005812f42e121816790102f879c082c08353
:10ef8000e960047c0180027c005392fe9004e1e081
:10ef900054fefaa3e0fbea4c9004e1f0a3ebf0028c
:10efa000eaee74f712229ee960047c0180027c0084
:10efb0009004e1e054fdfea3e0ffec25e0fce43327
:10efc000fdee4cfcef4dfd9004e1ecf0a3edf0ea1a
:10efd000940750047a078008eac3941140027a101b
:10efe000ea9004e0f0ebc3940540027b03eb90044d
:10eff000def002fa4174f612229eeaff600b9004e2
:10f00000dfe0f470047a8b80131213f0e970047a55
:10f010008680091217daea4b70067a827b01801328
:10f020007c01eff9121900e96005fa7b0380047a8c
:10f03000007b0002f87974f312229e74fe122237cc
:10f040001224d274f61222068a238b2489228c2160
:10f0500012fa2760071217e0790580747c0012f11c
:10f060007d40010c12f1757006e52260027c0105fd
:10f07000929004e1e0f812f6652468f582e43af52e
:10f0800083e0a2e04009e854026004e52170159095
:10f0900004e0e0fd12f6652467f582e43af583e0ca
:10f0a000c39d50027c01e8a2e0e433fa900491e0b1
:10f0b000a2e0ec5033a2e05015e5226004eaff80a4
:10f0c000027f00ac21eff9aa23ab24121954790076
:10f0d000740a12221c8532828533831224da740268
:10f0e00012221c7f05022376a2e0503374ff6b705e
:10f0f0002ee5226004eafe80027e00752510782548
:10f100001224ea75250778251224ea7d07ac21ee42
:10f11000f9aa23ab24121960740212221c80b1795f
:10f120000aac32ad337a8412182ee9640a6024e501
:10f130002260089004e112f16e80027900752510ba
:10f1400078251224ea75250778251224ea7d07ac74
:10f150002180beac32ad33900363e0f9aa23ab2427
:10f16000121732e9700302f0ce790802f0d0e0a263
:10f17000e0e433f92212fb62fb74ff6b2212f18c84
:10f180002411f582e439f583e0a2e72212f196f822
:10f19000a3e039f9e822900363e075f0e6a4f8a94a
:10f1a000f090045ee0282274f412229e74fc122275
:10f1b00006853282853383eaf0a3ebf0a3ecf0a35b
:10f1c000edf01213f0e970057a8602f25212fb3369
:10f1d000740368600e740768600974086860047ad4
:10f1e00081806f75230475240078231224e674024d
:10f1f00012229412edf9121cd2740212221c12fa7d
:10f200002724fd600924fc6034146035807a1217cd
:10f21000da8a238b24ae23af24ee4f603312f29da3
:10f220001224e612f2ae12189a740212221c12e78d
:10f230001aeefaeffb12192a12f291804a74098031
:10f24000461217da8a238b24ae23af24ee4f7006c2
:10f250007a827b018036900361e02422f523a3e0cb
:10f260003400f52478231224e6900361e02432125e
:10f27000f2b412189a740212221c12e466eefaef2b
:10f28000fb12192a12f297f07a007b00740402fe36
:10f290007412e70d74042212e70d740a22900361c0
:10f2a000e02412f523a3e03400f524782322900310
:10f2b00061e0244212e47a12f2bb22900361e0245e
:10f2c00053faa3e03400fb2274f712229ee97b0775
:10f2d000fa79021219ae02fa4174f212229e74fef9
:10f2e0001222371224d28923e9900363f0fe75f0cd
:10f2f0006fa4f521e5f0f52212f43e900361e5825a
:10f30000f0a3e583f00592a3ea24fe601024fd60db
:10f310003214700302f40614600902f41112190c7d
:10f3200002f4117401f07a0512171aa923121b1c9a
:10f33000900363e06523700302f411a9231213f014
:10f3400002f41112f717700302f40e7525017526e9
:10f3500000e878251221f305929004dfe04525129c
:10f36000f42e12181612f43eaa82ab83ea2463f834
:10f37000e43bf9888489850592900491e0a2e00538
:10f3800092e0400b54096401600302f40e8014a261
:10f39000e0507bea2464f582e43bf5830592e0a229
:10f3a000e3406bee75f0e6a4feaff08e218f2253a2
:10f3b00092fe90045ee02ef584a3e0352212f42044
:10f3c000e0a2e050047e0280027e017906e58424fa
:10f3d0000bfce43585fd8a828b83e0fbee4480faea
:10f3e00012181612f44f12f41450047804800278a4
:10f3f00002900361e0f9a3e0c9246af582e439f5db
:10f4000083e048f08008e024f3c3940a5003121903
:10f410006c02edd32412f582e439f583e0a2e022f8
:10f42000f585e5842412f582e43585f5832212f40e
:10f43000347b0022f079017cdf7d047a0222059280
:10f44000900365e02521f582a3e03522f583229023
:10f45000045ee02521f8a3e03522f9e822c082c04d
:10f46000837b075392fe900363e0fa79021219ae90
:10f4700002eaee74f712229e74fe1222371224d290
:10f4800005929007e51224f97b070592900363e04b
:10f49000fa79021219ba740402fa3074f012229e38
:10f4a00074fe1222371224d28a278b2889218c25b8
:10f4b0008d2212f523740212f9b185848285858329
:10f4c000a3a3f074055521858482858583a3a3a316
:10f4d00012f8117410f0e9a2e05004ae2580027e0b
:10f4e00000ee858482858583a3a3a3a3a3f0e9a26c
:10f4f000e05004af2280027f00ef12f99b1224e655
:10f50000ac84ad85900361e0240b12ea5d121cd23d
:10f51000740212221c7c067d00aa27ab281215d685
:10f5200002eac28a828b83a3a37405f08a848b8546
:10f530000592a3a3a3a3a3a3a3a32274f612229ebe
:10f5400074fe1222371224d212f564740302f847b3
:10f5500074f612229e74fe1222371224d212f5641f
:10f560001402f8478a848b85858482858583a3a3ca
:10f57000a882a983740512f815a3a3a3a3aa82ab3a
:10f58000832274f612229e74fe1222371224d27441
:10f59000f0122206eafeebff7908900361e02432c4
:10f5a00012ea5d1219e47910ac32ad337a067b00b1
:10f5b00012182e12f649aa32ab3312188e8a218bfa
:10f5c00022a821a92212f66512f64012f65a244208
:10f5d000f582e43af58312ede612f6ff04f00592a7
:10f5e00012f8257a057b0012182e85848285858382
:10f5f000a385822185832278211224e6e4f521f572
:10f600002278211224e612f83012228c12189474f7
:10f610000412221c12f66e1224e67c007d00e584a2
:10f620002af582e43585f583a3aa82ab83121cd820
:10f63000740212221c7c067d00eefaeffb02feda59
:10f640002465f582e43af5832212f64d2290036197
:10f65000e02432fca3e03400fd22e068f8a3e06976
:10f66000f912f66522900361e0faa3e0ca2212ead9
:10f67000a712f67df52195e0f522782122e0f888a1
:10f6800082aa827410c39a2274f412229e74fe120b
:10f6900022371224d212f6fb7407f00592e0240af6
:10f6a00012f81c85822185832212edec2442f5821a
:10f6b000e438f58312eb01f985218285228312ed6e
:10f6c000e675230875240078231224e612f649e52e
:10f6d000842403fae43585fb121cd2740212221c26
:10f6e00012f717600d790aac21ad22e8fb7a861279
:10f6f000181612fdadd2e6f002fe5eeafeebff8eba
:10f70000828f83a3a37405f08e848f850592a3a3b3
:10f71000a3a3a3a3a3a32212fb62f874ff6822741d
:10f72000f712229e74fe1222371224d212f564744c
:10f730000812f87ef079108a828b83a3ac82ad83a5
:10f740007a077b0012182e7c067d00aa84ab8512f6
:10f7500015d602fa3374f612229e74fe1222371264
:10f7600024d212f6fb7409f00592e02407f075210b
:10f770000675220078211224e67c977d04e5842416
:10f7800002fae43585fb121cd2740212221c059287
:10f79000a3e4f07c06fdeefaeffb02f86874f612c3
:10f7a000229e74fe1222371224d274f01222068a8c
:10f7b000848b85858482858583a3a3a882a983748d
:10f7c0000512f811a3a3a3a3ae82af83740af08835
:10f7d00082898312f8257a077b0012182e8e828f79
:10f7e00083a385822185832278211224e675210155
:10f7f00075220078211224e612f83012228c121899
:10f8000094740412221c7c067d00aa84ab8502fe3f
:10f81000da12f8152212f81ca3a3a322f085848221
:10f82000858583a322e02410f07910ac32ad332219
:10f8300012edf012f8397404222465f582e438f5eb
:10f8400083e0fca3e0fd2212f87e12f8871224e682
:10f850008a828b83a30aab83121cd2740212221ced
:10f860007c067d00aa84ab851215d685328285334d
:10f87000831224da740212221c7f02022376f0889b
:10f88000828983e0241022f07521107522007821ee
:10f890002274f712229e74fe1222371224d2e9fe3d
:10f8a000ecff8a828b83a3a3a882a98312f5298502
:10f8b0008482858583740b12f8e1ee60047c0180fc
:10f8c000027c009004e1e054026007ef60047804d9
:10f8d00080027800ec480592a3f07c067d0002f7d8
:10f8e0004f0592f088828983e004f02274f212229c
:10f8f0009e74fe1222371224d28a258b26e9fe8db1
:10f900002112f523740112f9b1fa85848285858369
:10f91000a3a3f0ee60047b0180027b0085848285d6
:10f920008583a3a3a3a882a983ebf0ec6013ea70fc
:10f93000089004dee06403600888828983e0d2e2f4
:10f94000f0741112227012f9caa3a3a3f0ee60049e
:10f95000af2180027f00ef858482858583a3a3a3e6
:10f96000a3a3f0ee60087410122270e08001e4128c
:10f97000f99b1224e6ac84ad85900361e024041267
:10f98000ea5d121cd2740212221c7c067d00aa259c
:10f99000ab261215d612191e02edd38584828585f9
:10f9a00083a3a3a3a3a3a3f075230775240078233f
:10f9b00022f00592e02406f09004de12f9caf090dd
:10f9c00004e1e01313543f540122e08584828585cd
:10f9d00083a32274f712229e74fe1222371224d2bd
:10f9e00012fa2760071217e079058022740c1222a0
:10f9f0007a0592122501740c12227a12250112192d
:10fa00005a740212221c12e7097402f07900802352
:10fa10008a848b85858482858583a3a3a3a3a3a3de
:10fa2000a3a3a3ac82ad8312fa2b2212e711e0222a
:10fa300012221c8532828533831224da7402122248
:10fa40001c7f0102237674f612229ee9fe1217da59
:10fa5000ea4b70047901802fee600e146010146080
:10fa600012146014146016801912193680171219b6
:10fa70003c8012121942800d121948800812194e4a
:10fa800080031217e0790002f87974f612229e744e
:10fa9000fe1222371224d212fa27c3940d50087492
:10faa0000d800312fda8f012fb337417686059e84b
:10fab000c39412502a74f328f97521017522007835
:10fac000211221f312edec12eb0de0552160d490e0
:10fad0000491e0a2e05059121966e960c6805174a1
:10fae000ee28fa75210175220078211221f312fb0c
:10faf0004ae0552160ad900491e0a2e04032eaf97d
:10fb0000121966e9609d802812f717602012fb38f1
:10fb1000121816900363e0fe12fb5efaeef9121b58
:10fb200016900363e06e6005eef91213f01218be32
:10fb300002f86b12fa2bf82279040592900361e027
:10fb4000246712e47ae8fb7a872212fb4e2212ed38
:10fb5000f412fb55222464f582e438f5832212fb6b
:10fb60006222900361e0f584a3e0f5850592e0222e
:10fb700074f112229e74fe1222371224d2eafeeb96
:10fb8000ff8e828f83a3a3a3a3a3a3a3a3aa82ab65
:10fb90008312fa27fc74016c700302fc358a828b95
:10fba00083a38582238583248a828b83e0f8146073
:10fbb0003b14700302fc5214700302fc68147003bf
:10fbc00002fc9714604014700302fcaa1470030234
:10fbd000fcaa14700302fcaa14700302fcaa14709d
:10fbe0000302fcaa14700302fd598049ec60030271
:10fbf000fc8c900491e0a2e0400302fc8ceefaef52
:10fc0000fb1218b880361218be12fdbdf5218523ef
:10fc100082852483e06005fa7b0380047a007b0000
:10fc2000900363e0f9121b22900363e065216005f5
:10fc3000a9211213f0eefaeffb1217e0853282854c
:10fc400033835392fe1224da740212221c7f0702bd
:10fc5000237674026c7035900491e0a2e0402deea2
:10fc6000faeffb1218b280d474096c600a74076c46
:10fc7000600574046c7009eefaeffb1218ac80bcde
:10fc8000740c6c700712ea97e0f980027908eefaba
:10fc9000effb1218c480a5740a6c600574056c70c3
:10fca000ebeefaeffb1218a68092ecc3940d4085a0
:10fcb00012fb5ef974ff69700302fd488927790021
:10fcc000e527f522e824fa600e14601c1460611424
:10fcd000602714606c806c7910ac23ad247a80ab03
:10fce000221218167901805b790aac23ad247a843c
:10fcf000ab221218167910804a8523828524830549
:10fd000092e0700575250180037525027906ea24c5
:10fd100002fce43bfdab22e5254480fa121816856f
:10fd20002382852483e0700479028017790480138c
:10fd30007910ac23ad247a83ab221218167908808f
:10fd400002792012fdad49f0eefaeffb1217e01236
:10fd5000fda8f012196c02fc3c900491e0a2e05066
:10fd60000302fc3585238285248312fd9cb382f037
:10fd7000500a12eabd7005790502fc8eec600302a0
:10fd8000fc3c8523828524835392fee05404fc12bc
:10fd9000f16eeefaeffb12190002fc3ce0a2e092d9
:10fda000f09004e1e0a2e02212fa2b04225392fe2a
:10fdb00012edf0246af582e438f583e02212ef199f
:10fdc00074ff0592f00592900363e02274f612220c
:10fdd0009ee9fe75210175220078211221f390041d
:10fde000dfe0552170047900800f7904eafcebfd17
:10fdf000eefb7a8712182e790102f87974f4122238
:10fe00009e74fe1222371224d274fc12220689211b
:10fe1000eafeebff8c848d85aa32ab33121978e9a8
:10fe200060317403122270e0a2e15006752301e4f0
:10fe30008009a2e2501d75230274010592f0790633
:10fe4000eefceffdab21e5234480fa12182ee964a5
:10fe5000066004790080027901740402e1a87c063e
:10fe60007d00eefaeffb1215d685328285338312c0
:10fe700024da740212221c7f0402237674f6122202
:10fe80009e74fe1222371224d274f01222068a21a6
:10fe90008b228a848b850592a3a3a37903aa84abc2
:10fea000851219e4852182852283a3a3a3a3a3e05d
:10feb000543f4440f07910ac32ad337a077b0012e6
:10fec000182e78211224e6ac84ad85740212228c9f
:10fed0001218a0740212221c80031215d67410127c
:10fee000221c02f86b74f712229e74fe1222371243
:10fef00024d28a848b85a2afe433fcc2af8584828e
:10ff0000858583e0faa3e0fbea4b601a8a828b8343
:10ff1000e0f8a3e0f9e80592f0a3e9f08a828b8388
:10ff2000e40592f0a3f0eca2e092af853282853333
:10ff3000831224da740212221c7f0102237674f7e2
:10ff400012229e74fe1222371224d28a848b85ecf0
:10ff5000f8edf9a2afe433fcc2af858482858583d6
:10ff6000e0faa3e0fbea4b7009e80592f0a3e9f0a0
:10ff7000801d8a828b83858284858385439201e0fc
:10ff8000faa3e0fbea4b70eae80592f0a3e9f0ec93
:10ff9000a2e092af8532828533835392fe809274c1
:10ffa000f712229e74fe1222371224d2a2afe4333b
:10ffb000f521c2af8a828b83e0f8a3e0f9e84960bb
:10ffc000248c848d8580048e848f858584828585ac
:10ffd00083e0fea3e0ffee4f70ed8584828585838c
:10ffe000e8f0a3e9f0ecf8edf98a828b83e8f0a35e
:10fff000e9f0e52102ff27ffffffffffffffffff03
:020000040001f9
:1000000074f412229e74fe1222371224d274fc124f
:1000100022068a828b83853284853385e40592f0bb
:10002000a3f0a3f0a3f07404c399f5230592e0852f
:1000300032848533850592f00592a3740112227ae9
:10004000800d5392fee00592f00592a30592a3194c
:10005000e970efec602de58224fff582e58334ff43
:10006000f5835392fee0a2e75019e5236015fa7b71
:100070000078ffe8439201f0a3ea281aeb34fffb73
:100080004a70f08532828533835392fe1220597470
:100090000412221c8532828533831224da74021200
:1000a000221c7f0402237674f712229e74fe122211
:1000b000371224d21280dac824fcf582e834fff526
:1000c000831280e51220598532828533831224da27
:1000d000740212221c7f01022376900929e0f8a302
:1000e000e0221280ee0592900929128ce7229009f5
:1000f000291280f522e0f8a3e0f5838882a3227418
:10010000f412229e74fe1222371224d28a218b22ec
:100110008c238d24128f300592782112204a05926b
:10012000900929128c6c12813485328285338305c3
:100130009202809aa30592900929e582f0a3e583b3
:10014000f02274e812229e74fe1222371224d27416
:10015000fa1222067404122270eaf0a3ebf0801265
:10016000128c92858482858583e0fae4fbfcfd1283
:100170001c1274041222705392fe128d42e84960e0
:10018000317404122270e024fff018a3e034fff071
:10019000f9e849701d79ff740612221c85328285a8
:1001a00033835392fe1224da740212221c7f10024f
:1001b0002376128cabf805929006b6128c4a059203
:1001c0009006b612813a74176805929006b6700fc1
:1001d000128c7f05929006b612813a790080b8128f
:1001e0008c4aae82af837436687003028160741be0
:1001f00068702005929006b6128ef2122059121cd9
:10020000129006b6128c6ca305929006b612813a33
:100210000281727401687028128cabc0e0128f2ebc
:10022000d0e0128cc41280e2128cabc0e0128f2e90
:10023000d0e0128cf1128c03a3059290092980cd95
:10024000741068700f128cabc0e0128f2ed0e012c9
:100250008cc480e1741968700f1280dac824fdf52f
:1002600082e834fff58380d1741a6870081280da4e
:10027000c824fe80ea742468701d121c0c8a298b25
:100280002a740c78291221f3121c0ceb540ff9e597
:100290002a49fbe402816d7425687037121c0c8ab0
:1002a000298b2a8c2b8d2c74187829121f32121c42
:1002b0000c8a218b228c238d2490092c7821121feb
:1002c000c978297921121fdcaa29ab2aac2bad2cc5
:1002d00002816f742168702c121c0c8a298b2a8c65
:1002e0002b8d2c121c0c8a218b228c238d24aa2965
:1002f000ab2aac2bad2c121c12aa21ab22ac23ad25
:100300002402816f743468600302838c121c0c8a8f
:10031000258b268c278d28121c0c8a218b228c235e
:100320008d24121c0c8b2a8a2d8b2e8c2f8d3090b5
:100330000930782d121fc9128bd260059006b88043
:10034000039006b4128bdd121fc9128bc960059091
:1003500006b880039006b4128c608525218526227c
:100360008527238528249009347825121f64128b51
:10037000ba70030281720592e08a828b830592f043
:100380000592a30592a3aa82ab8380ce74356870d0
:1003900062121c0c8a258b268c278d28121c0c8a35
:1003a00021121c0c8b2a8a2d8b2e8c2f8d309009bc
:1003b00030782d121fc9128bd260059006b88003c9
:1003c0009006b4128bf8aa82ab8385252985262a4c
:1003d00085272b85282c5392fe9009347825121fef
:1003e00064128bc970030281728a828b83e521f0cb
:1003f000a380d374466860030284d085328285333b
:1004000083e4f0a3f0a3f0a3f0121c0c8a258b2642
:100410008c278d28121c0c8a218b228c238d241270
:100420001c0c8b2a8a2d8b2e8c2f8d3090093078c6
:100430002d121fc9128bd260059006b8800390065a
:10044000b4128bdd121fc9128bc960059006b880eb
:10045000039006b4128c60801ac2f0a2f0e433f567
:1004600021e4f522f523f524853282853383782132
:100470001220028525218526228527238528249080
:1004800009347825121f64128bba6028eafcebfd50
:100490008c828d83a3aa82ab83a884a9850592a3ad
:1004a0008c828d830592e0fc88828983e06c60a950
:1004b000d2f080a7853282853383122089e8494aa9
:1004c0004b7004d2f08002c2f0a2f0e43302816ae1
:1004d000740e687035121c0c752500752600752782
:1004e00000752800128cd2c0e0128c29d0e0059251
:1004f000f005929008977825121f649008b7782528
:10050000121d32500302817280da740c6870451239
:100510001c0c752503752600752700752800852598
:1005200021852622ea2521f8eb3522128f3fc0e0f3
:10053000128f2ed0e00592f005921280e2900934dd
:100540007825121f649009387825121d3240030265
:10055000817280ca741c687021121c0c8b2a128c48
:10056000a5858482858583e0f99006b8e02afaa300
:10057000e0352afb121c0602816f741e68700c1293
:100580001c0c8b2a128c927c0180d6740d687057db
:10059000121c0c8a218b228c238d24121c0c752595
:1005a00000752600752700752800801d85252d857e
:1005b000262eea252df8eb352e128f3fc0e0128f44
:1005c0002ed0e0128d04121f6478217925121d08a7
:1005d00040da9008b77825121d325003028172125a
:1005e0008d00121f6480eb741d68705b121c0c8af6
:1005f000218b228c238d24121c0c7525007526005e
:10060000752700752800802185252d85262eea2551
:100610002df8eb352ef99006b8128f43c0e0128ffb
:100620002ed0e0128d04121f6478217925121d0846
:1006300040d69008b77825121d32500302817212fd
:100640008d00121f6480eb740f6860030287011233
:100650001c0c8a218b228c238d24121c0c9008b731
:100660007821121d3240607525047526007527001b
:1006700075280078257921121f8a85328285338377
:10068000782512204a8009900929128c7f12813521
:100690008532828533835392fe782512203b85254f
:1006a0002d85262e85272f852830900934782d1208
:1006b0001f64853282853383782d12204ae52545d3
:1006c000264527452870c09009347821121f64857b
:1006d00021258522268523278524289009387825f9
:1006e000121d324003028172128cd2c0e0128c299a
:1006f000d0e00592f005929009347825121f6480ad
:10070000da742068600302879c121c0c8a218b22f9
:100710008c238d24121c0c8a298b2a121c0c8532e6
:1007200082853383122065121c0c8a258b26853224
:10073000828533837821121d1d500b8532828533cb
:1007400083782112203be52124fff8e52234fff9cc
:10075000c3e99400a2d265d033500302817285258b
:1007600021852622e52128fae52239fb5392fe90c5
:1007700006b8128c1f0592e0c0e0852921852a2247
:10078000e52128fae52239fb05929006b4128c1f68
:10079000d0e00592f0e824ff18e980b17402687097
:1007a00020121c0c8a298b2a8c2b8d2c121c0c8a53
:1007b000218b228c238d2478297921121f510282ca
:1007c000c87403687020121c0c8a298b2a8c2b8d0c
:1007d0002c121c0c8a218b228c238d2478217929c0
:1007e000121f8a0282f97404687020121c0c8a2974
:1007f0008b2a8c2b8d2c121c0c8a218b228c238d06
:100800002478297921121fb60282c87406687020e4
:10081000121c0c8a298b2a8c2b8d2c121c0c8a21e1
:100820008b228c238d24782979211220150282c8ed
:100830007405687019121c0c8a298b2a8c2b8d2c3c
:10084000121c0c8a218b228c238d240282c17407f6
:10085000687020121c0c8a298b2a8c2b8d2c121c60
:100860000c8a218b228c238d2478297921121d97c3
:100870000282c8740868702d121c0c8a298b2a8c7d
:100880002b8d2c121c0c8a21128bc36009782179c4
:1008900029121eb0800c7521007522007523007589
:1008a00024000282f97432687028121c0c8a218b91
:1008b000228c238d24121c0c8a258b268c278d28b4
:1008c00078257921121d085004d2f08002c2f0026e
:1008d00084c9740a687028121c0c8a218b228c230c
:1008e0008d24121c0c8a258b268c278d2878217943
:1008f00025121d085004d2f08002c2f00284c9748f
:1009000033687028121c0c8a218b228c238d2412b0
:100910001c0c8a258b268c278d2878257921121c82
:10092000de6004d2f08002c2f00284c974096870eb
:1009300028121c0c8a218b228c238d24121c0c8ad9
:10094000258b268c278d2878257921121cde7004b2
:10095000d2f08002c2f00284c9740b687061121c6c
:100960000c8b2a8c2b8d2c128cabf521e4f522f507
:1009700023f52405929006b6eef0a3eff0128cabaf
:10098000f525e4c525f526e4f527f5287821792510
:10099000121fdc05929006b6128c7212813aea128e
:1009a0008bcb6003028172059290f790e02521f8cd
:1009b000a3e03522f99006b6e8f0a3e902815d7460
:1009c0001868704a128cabf529e4f52af52bf52c42
:1009d00005929006b6eef0a3eff0852921852a2234
:1009e000852b23852c245392fe9009347829121fdd
:1009f00064128bba7003028172128cabc0e0128f4a
:100a00002ed0e0128cf1128c0312813480cc744011
:100a1000687022121c0c8a298b2a8c2b8d2c121c9c
:100a20000c128bc3600aea128bbc6004d2f0800205
:100a3000c2f00284c97441687022121c0c8a298b8e
:100a40002a8c2b8d2c121c0c128bc37006ea128b75
:100a5000bc6004d2f08002c2f00284c974426870a3
:100a60001a121c0c8a29121c0c8a218b228c238db1
:100a700024e5297821121f320282f9744368701a22
:100a8000121c0c8a29121c0c8a218b228c238d2487
:100a9000e5297821121eff0282f974456870281238
:100aa0001c0c8a218b228c238d24121c0c8a258bf2
:100ab000268c278d2878217925121d084004d2f034
:100ac0008002c2f00284c97444687028121c0c8a27
:100ad000218b228c238d24121c0c8a258b268c279b
:100ae0008d2878257921121d084004d2f08002c299
:100af000f00284c9741568701b9006ba128c5412e7
:100b00001c129006b8128c54121c12900929128cd7
:100b10000b0289b8741668701d9006bc7401f0123f
:100b20008ca59006ba128f14858482858583e0f99e
:100b3000121aaa028172745068702d128efce82479
:100b400002fae439fb3395e0fcfd121c129006ba60
:100b5000128f1a128cb9128c721280ea128cabf9b5
:100b6000a821128c130289b4741468700a128cb90b
:100b7000eef0a3eff080e574516870169006b8129d
:100b80008c0b128f28121c0c8b2290f790e02a02fb
:100b900089af742f6860030281729006ba128d4289
:100ba000900929128f28121c0c9006b8eaf0a3ebca
:100bb000f0121c0c9006ba028159e521452245230a
:100bc0004524228b228c238d24e529452a452b455b
:100bd0002c22e52d452e452f4530059222128bf80b
:100be000aa82ab8385212985222a85232b85242c63
:100bf0000592900930782922e02af582a3e0352a6f
:100c0000f583221280daf5838882221280ddf99042
:100c100006ba22059290f790e028f8a3e03922e086
:100c20002af584a3e03bf58522852521852622ea45
:100c30002521f8eb3522f905929006b4128c40225a
:100c4000e028f584a3e039f58522e0f9a3e0f583f7
:100c50008982a322e0f521a3e0aa21fbe4fcfd2286
:100c6000e02521f584a3e03522f585221280f1a349
:100c7000a322128c76221280f505929006b62212db
:100c80008c8322e0f8a3e0c824fff582e834fff566
:100c90008322128c96229006b6128f379006b6eefb
:100ca000f0a3eff022128c967c0022128caf2290df
:100cb00006b6128f370592e022128caff52105920d
:100cc0009006b6220592f005929006b6eef0a3efdc
:100cd000f022900929128c83128ce2900929128c3f
:100ce000b2220592900929e582f0a3e583f00592ee
:100cf000220592f005929006b6128c76128ce722ad
:100d0000128f34e40592f005921280ee128ce2907c
:100d1000089778252274f712229ee5c7fe90036893
:100d2000e0f5c790f790128d42128f2590f7e612ea
:100d30008f1412130c9006b4eaf0a3ebf08ec702e6
:100d400080d51280ddf92274f212229e74fe1222e6
:100d5000371224d2e9fee5c7f521900368e0f5c714
:100d60008a828b83e0f525a3a3e0f5268a828b8314
:100d7000a3a3a3e0f522e525a2e7400b9006bce083
:100d80007003028edfe4f0900929128f1a9006b8e2
:100d9000e0f523a3e0f5248a828b83a3a3a3a3aa6f
:100da00082ab8374fc2efe80308a828b83e0c0e0ad
:100db000128f30d0e00592f08a828b830592a3aa2d
:100dc00082ab831280daf58588840592a305929020
:100dd0000929e584f0a3e585f0eeff74ff2f1e04da
:100de00070c77410122270128d42803488828983f9
:100df000e0c0e0128f30d0e00592f0888289830550
:100e000092a3a882a983900929e0faa3e0f5858a34
:100e1000840592a30592900929e584f0a3e585f065
:100e2000ecfaedfbea24ff1ceb34fffdea4b70bc4f
:100e3000e525a2e74003028edca826e828f8e43383
:100e4000f990f790128f43f8a3e0f974ff687003ec
:100e500074ff69607aaa22ea2afae433fb128c133f
:100e6000f9e82af582e93bf583128d4274ff687038
:100e70000374ff696059128c15f9128f2590f7edf4
:100e8000128f14121c18e96046128efc90063e1256
:100e90008f28a37485f0a37401f090063a7480f053
:100ea000a37404f0a3e4f0a37404f0e4f525f5269c
:100eb00078251224e67c007d007a3a7b06790805c5
:100ec0009290064e128ef212229c740212221c5331
:100ed00092fe900929e523f0a3e524f08521c7853a
:100ee00032828533831224da740212221c7f0602b6
:100ef0002376e0f582a3e0f5830592229006b605fd
:100f00009290f790e0f8a3e0f90592e0c398f8a377
:100f1000e099f922e0faa3e0fb221280ddf99006c5
:100f2000b8128f28229006b6e8f0a3e9f0220592c5
:100f3000128f3422900929e0f584a3e0f58522f987
:100f40009006b4128c400592e02274f712229e742f
:100f5000fe1222371224d2eafeebffee6005146087
:100f60000c805c128fc490092be4f0804e90092b0a
:100f7000e06401700f128fc49006c0e4f09006c1c7
:100f8000f0a3800cef9006c0f09006c1ecf0a3ed4a
:100f9000f090092b7401f005929006c11224fd0512
:100fa000929006c0e0fc7d009006be128f14900661
:100fb000bde0f9121c24740212221c79018002790e
:100fc000000280c7ef9006bdf09006beecf0a3ede6
:100fd000f02274f412229e89237524007409782368
:100fe0001221f38a218b22740278211221e4aa2192
:100ff000e5225401fbe42ae5243bfb02908e74f7c2
:1010000012229e74fe1222371224d274fc1222067f
:10101000e9fe85328485338590084474041220ae3d
:10102000eef4853282853383129093121426740471
:1010300012221c8532828533831224da7402122232
:101040001c7f0102237674f412229e74fc12220685
:101050008921ebfe7403122270eaf0eef4853282ed
:10106000853383f0740212227074fff0740112222f
:101070007074ff12909385212375240074097823de
:101080001221f3faab24121426740412221c7f04da
:10109000022376f07904ac32ad332274f712229e2b
:1010a00074fc122206eafeebff8921853282853329
:1010b0008374fff07403122270e9f074011222703d
:1010c000ecf0a3ed1290931214267980eefaeffb68
:1010d0001217f27403252154fcf9740d122270e0ea
:1010e000fca3e0fdee2401fae43ffb121426794054
:1010f000eefaeffb1217f2740402903e74f0122223
:101100009e74fe1222371224d27582fa7583fe1263
:101110002252e5c7c0e07403122270d0e0f09004c0
:10112000d1e0f89004cee068700d9004cde0f89026
:1011300004cee02814800374ff28feeef912142078
:101140007402122270e4f0fbfaeef91217f8752718
:10115000047528007401122270e40292080e7402d1
:10116000122270e004f0752704752800852382851b
:101170002483e0f52175220078211224e6e58424f9
:1011800004fce43585fd740812228c121cd2740212
:1011900012221caa27ab28eef91217ec74061222b1
:1011a000848821892278211224e68523828524835c
:1011b000e0f90592a3e0fca3e0fd1217fe74021211
:1011c000221c852382852483e024fff8e434fff980
:1011d000e854fc2408f8500109e52728f527e528fc
:1011e00039f52812977a1221d412973ec3e5269436
:1011f00002407a8532828533835392fee0f91214dd
:10120000207401122270e004f09004d3e0f874011d
:10121000122270e0c3984003029327e0f89004d1b3
:10122000e028853282853383f01298cc40041297ef
:101230006ef0853282853383e01297387b107aff17
:10124000e0f91217f8853282853383e0f5217522a3
:1012500000740b78211221f3e5224480f974041202
:101260002270e4f0a3e9f07525017526008525219b
:10127000852622740278211221f37404122270123e
:101280009b5412203b8584828585837821121cf330
:1012900070030291f30592e0a2e7500b0525e525c6
:1012a000700205260291ec8584828585830592a3d0
:1012b000a3a3858223858324a2e540030291e3e072
:1012c000f8e52728f8e43528f9e82404500109c393
:1012d0009401e99408500302916c74012eff8f2150
:1012e00012934a65214970059004cee0ffeff91290
:1012f00014207b007402122270e004faeff9121736
:10130000f87b207affeef91217f88e2112934a2407
:10131000ff18e934fff9e8652149600302915d9007
:1013200004cee0fe02915e7b207affeef91217f800
:101330007403122270e0f5c712180a7582067583cd
:1013400001122252853282029b049004cee0f89072
:1013500004cde0fae82af8e43400f9e82274f51242
:10136000229e74fe1222371224d2e5c7fe90036833
:10137000e0f5c790f7efe09004cdf090f7e8e024b7
:10138000309004cef0f8743ec398f9900368e0649e
:10139000077005747ec398f99004cde0f8e9c3980e
:1013a00050057901121a028ec7e5c7fe9004cf746a
:1013b000fff0a3e4f0a3f0a3f0a3f07ffff52390e8
:1013c00004cee0fc80368582848583850592a3e087
:1013d000f4704d858284858385a3a3e0f4704185f4
:1013e0008284858385a3a3a3e0f4703405929004de
:1013f000cfe0f47002ecf0a3e004f00c8c82858264
:1014000021752200129781505fec129738740b7887
:10141000211221f3f582e5224480f583e0f460a6f1
:101420004392019004d3e004f0858284858385a3f0
:10143000a3a37803a985e0fac39f5007eaffec90c5
:1014400004d1f088848985e0f8c395234007882378
:10145000ec9004d2f00592e054306410609d1218b4
:101460003a9004d1e4f080069004d1e0700c90042e
:10147000cee09004d1f09004d2f08ec78532828500
:1014800033831224da740212221c7f03022376743f
:10149000f012229e74fe1222371224d274f212220b
:1014a000067408122270eaf0a3ebf0740a1222709c
:1014b000ecf0a3edf07403122270e9f01298b4126c
:1014c00021d4e52104c0e07407122270d0e0f0e5d9
:1014d000c7c0e07406122270d0e0f07404122270cb
:1014e000e4f0a3f0f528853282853383800b8532c2
:1014f000828533835392fee004f09004d312976efa
:10150000e0f89004d1e0400302967428f527129782
:101510007f4008e0c527c39527f527129736852712
:1015200021752200740b78211221f3e5224480f901
:10153000740c122270e4f0a3e9f07407122270e038
:10154000f87401c398fe74029400ff752501752696
:101550000080080525e52570020526c3e5259ee5e2
:10156000269f508a85252185262274027821122102
:10157000f3740c1222705392fee02521f8a3e0359b
:1015800022f97401122270e8f0a3e9f0900934788e
:101590002112203b74011222701297647821121cd0
:1015a000f37041740a12227a1224fd74051222701b
:1015b0000592e0f9740a12227012975bc0e074037e
:1015c0001222701298c6a9271217ecd0e0f9eefc8f
:1015d000effd1217fe740212221ce5287003029719
:1015e0002702971174011222700592129764e0a2eb
:1015f000e75003029553740112227005921297521c
:10160000129ce97408122270e0687003a3e069700c
:10161000490592e0a2e5504274041222700592122c
:101620009ceae849601fe5281297387420c0e074ee
:10163000041222701298c6a9281217ecd0e0f912f1
:1016400017f21297367401122270129cea74041277
:101650002270e8f0a3e9f085272874011222705364
:1016600092fe129752a3a3a312977a1221d4129733
:101670003e02955b28f521f52312978ae5231298ff
:10168000e34008e0c521c39521f521e521129738f3
:101690009004d0e0c39402500d7406122270e0f55d
:1016a000c77900029731e014f09004d3e0fa740196
:1016b0002af07b20a9211217f8740a12227a0592c7
:1016c0001224fd74051222700592e0f9740a1222a8
:1016d0007012975bc0e0852123752400740b78237a
:1016e0001221f3e5244480f9e42404fae439fba947
:1016f000211217ecd0e0f9eefceffd1217fe740298
:1017000012221c7404122270129ceae8496018e547
:101710002812973874041222701298c6a92812173a
:10172000ec7420f91217f27406122270e0f5c779f2
:1017300001740e029afbe527c4540ff5c722e52178
:101740002401f8e43522f9e52528f525e52639f5c3
:101750002622e0f8a3e0f583888222e0fca3e0ffe4
:10176000ecfee922e0f584a3e0f585059222e0f89d
:10177000853282853383e0c39822e01298b822f53f
:101780002112978ae5211298e3229004cee0fa9084
:1017900004cde0f8ea28f8e43400f92274f61222c5
:1017a0009e74fe1222371224d28a218b228c848dc1
:1017b00085e9fe121810e97012121804eef9ac84d3
:1017c000ad85aa21ab2212181080027901853282e0
:1017d0008533831224da740212221c7f02022376dc
:1017e00074f012229e74fe1222371224d274fe125a
:1017f00022068a278b28752500803d858284858373
:10180000850592a3a3a3a2e5501ae5822404fce473
:101810003583fde0f90592a31298c68527828528b5
:101820008312229c4392011298b31221d4129b2955
:10183000c3ef940240200525129b11505e9004d105
:10184000e025251298cc4005e0cac39afa129b19ec
:101850001221f3129b398e218f22740278211221da
:10186000f3853284853385439201e02521f582a3f7
:10187000e03522f583900934782112203b8582845b
:101880008583857821121cf360ac0592e0a2e740c5
:10189000030297fb0eee70980f80957c007d007917
:1018a000007aff7bff85278285288312229c7402a1
:1018b000029afbe01298b8222403f521e43400f5e3
:1018c000227402782122e0faa3e0fb22fa9004ceef
:1018d000e0f89004cde0fce82c1298dd22f8e43426
:1018e00000f9ea98e499c365d0332274f412229e79
:1018f00074fe1222371224d2eafcebfd790080320a
:101900005392fea3a3a3e07522002403f521500205
:101910000522740278211221d4e5212401f52150f9
:10192000020522ea2521faeb3522fbc3eb940240a3
:101930004b09129cdce9c39840030299db9004d167
:10194000e029f89004cee0fe9004cde0faee2afa09
:10195000e43400fbe89ae49bc365d0334005e0c85b
:10196000c398f8e81297388821752200740b782103
:101970001221f3e5224480ff7a017b008a218b2229
:10198000740278211221f32521f582ef3522f583a7
:101990000592900934782112203b858284858385c5
:1019a0007821121cf3608a0592e0a2e750080aea47
:1019b00070010b02992b8582848583850592a3e0b3
:1019c0006c7003a3e06d60030299000592e0a2e54c
:1019d0004003029900aa82ab8380047a007b0085d1
:1019e00032828533831224da740202908b74f012ef
:1019f000229e74fe1222371224d274fc1222067424
:101a000002122270eaf0a3ebf089288c26e5c7f5d4
:101a100027752500801785238285248312977a12e3
:101a200021d4129b29c3ef940240300525129b114b
:101a30004003029af29004d1e02525fa9004cee00a
:101a4000fc9004cde0f8ec281298dd4005e0cac314
:101a50009afa129b191221f3129b398e218f22744c
:101a60000278211221f3129b4e12203b858482853d
:101a700085837821121cf360b20592e0a2e750073b
:101a80000eee70a10f809e8584828585830592a3ca
:101a9000a3a3858223858324a2e54003029a1685a9
:101aa0008482858583a3e065286003029a168523d6
:101ab00082852483e065266003029a1685262175b7
:101ac000220078211224e67404122270e0fca3e0c4
:101ad000fde5842404fae43585fb121ccc74021263
:101ae000221c8b22ea45226003029a16aa84ab8547
:101af00080078527c77a007b00740412221c853278
:101b0000828533831224da740212221c7f08022396
:101b100076129ce0e525c39822eac4540ff5c78ae3
:101b200021752200740b782122e5212401f8e43587
:101b300022f9ee28feef39ff22e5224480f98532b2
:101b400082853383e4f0a3e9f07e017f00228532b1
:101b5000828533835392fee02521f584a3e035226c
:101b6000f58590093478212274f212229e74fe12b7
:101b700022371224d28c258d26e9fee5c7ff1218e4
:101b800022ea4b603e8a848b850592a3a3a3e0f8ea
:101b9000eec39850048e218002882185212375246c
:101ba00000059278231224e6ea2404fce43bfdaa13
:101bb00025ab26121cd2740212221c0592e08fc79c
:101bc000f980048fc779ff8532828533835392fe73
:101bd0001224da740212221c7f0602237674f11298
:101be000229e74fe1222371224d274fa1222067434
:101bf00004122270eaf0a3ebf07402122270ecf0ef
:101c0000a3edf0e5c7f5277526008053a2e550380f
:101c10008584828585830592129ce9740212227064
:101c2000e058f8a3e059f97404122270e0687003d8
:101c3000a3e06970137420c0e0aa84ab85a92512c3
:101c400017ecd0e0f91217f2439201a3a3a3129864
:101c5000b31221d4129b29c3ef94024035052612fa
:101c60009cdce526c39850599004d1e02526f52543
:101c700012977f4008e0c525c39525f525e5251277
:101c80009738852521752200740b78211221f312d3
:101c90009b398e218f22740278211221f3129b4ee0
:101ca00012203b8584828585837821121cf360ade8
:101cb0000592e0a2e74003029c0c0eee70990f80a3
:101cc000968527c7740612221c85328285338312bb
:101cd00024da740212221c7f07022376129ce0226f
:101ce0005392fe9004d3e0f822a3e0f8a3e0f92297
:101cf00074f612229e9004cee0fe8006eef91214d5
:101d0000200e8e2112978140f312180a0297db747d
:101d1000f612229eea24fcfeeb129d5e500aec2491
:101d2000fcfeed129d5e40067a127b02802e90032f
:101d300097129dba900394e054bffaa3e0fbe9a286
:101d4000e0e433f521752200740678211221f3ac0a
:101d500021ea4c900394f0a3eb12a091801334ff7e
:101d6000ffc3ee94fdef943f221224da7402122294
:101d70001c7f02022376c082c0835392fe9003949c
:101d8000e033335401f9d083d08202112974f71261
:101d9000229eea24e0feeb129dc6500aec24e0feef
:101da000ed129dc640067a127b02800b90039b12b7
:101db0009dbae9a312a091029e66eaf0a3ebf0a3fc
:101dc000ecf0a3edf02234ffffc3ee94e1ef943f7b
:101dd0002274f712229ee9feea24fc602b24fd7097
:101de00034ee900363f075f06fa4f8a9f0900365ea
:101df000e028f8a3e039f9900361e8f0a3e9f07a6c
:101e0000007900121486800d900392e4f090039103
:101e1000f0900393f0804f74f712229e74ff122209
:101e200006900393e4f0f52178211224ea7c327db8
:101e3000007a4b7b00900394e0c4131354035401c5
:101e4000f9121714740112221c7901ac32ad337ae5
:101e5000047b0012182ee9f46007900394e044809c
:101e6000f0740112221c7f0102237674f212229e6a
:101e700074fe1222371224d28a218b228a828b830b
:101e8000a3a3ae82af83e4f08a848b850592a3a3db
:101e9000a3a37402129fa314f0858482858583a373
:101ea000a3e91460051460068008740580067406b2
:101eb00080027404129faef8ea28f584e43bf585ad
:101ec0000592a3a3a3a37901129f977a077b2a12f5
:101ed00015b2e9600a7402129fa1740a129fae8eb5
:101ee000828f83e0f8e52128f584e43522f5850525
:101ef00092a3a3a3a37904129f977a047b2a1215b5
:101f0000b2e9600a7405129fa17412129faeaa2151
:101f1000ab22121522852182852283a3a3a3a38548
:101f200082258583268e828f83e0f9aa25ab26122f
:101f3000168a8e828f83e4f085218485228505921e
:101f4000a3a3a3a3791d129f977a007b2a1215b22f
:101f5000e9858482858583a3c3941d500a74012971
:101f60000592f074098007741e0592f074080592ba
:101f7000129faef96007aa25ab26121690aa21abd4
:101f8000221217e08532828533831224da7402121a
:101f9000221c7f06022376e5842402fce43585fdbd
:101fa000220592f08584828585830592a322f0051f
:101fb00092e004f88e828f830592e028f02274f478
:101fc00012229e74fe1222371224d274fa122206b2
:101fd000eafeebff89218c238d24121a08e9700494
:101fe0007a89800c900393e0f8c3940440077a81c7
:101ff0007b0102a079e86003121462900394e0a2ce
:10200000e0500eaa32ab33121984aa32ab33121647
:102010009cee4f6006eefaeffb80047a007b0074c2
:102020001a12227a05921224fd741a12227a1224ac
:10203000fd741a12227a1224fd741a12227a1224c2
:10204000fd0592900394e05401f52278221224eacf
:10205000ac23ad24a921121660740912221ce96078
:1020600005fa7b028013852382852483e090039602
:10207000f0900393740712a091740612221c85320b
:10208000828533831224da740212221c7f04022315
:1020900076f07a007b002274f012229e74ff1222e6
:1020a00006e9853282853383f08a278b288c238d3d
:1020b000241213f0e970047a86805274111222708f
:1020c000e0f521a3e0f5227413122270e0fea3e0f4
:1020d000ff900491e0a2e0402b8e258f26782512f8
:1020e00024e678211224e6ac23ad24aa27ab28905d
:1020f0000363e0f9121726740412221ce96031fa16
:102100007b0280301217daea4b70067a827b0180fc
:10211000238e258f2678251224e678211224e6784e
:10212000231224e6ac27ad281215e8740612221cef
:102130007a007b00740112221c7f0802237674f758
:1021400012229eeafe1213f0e970067a867b018065
:102150000eeefa900363e0f912171a7a007b000280
:102160009e6674f612229e900393e014600a146037
:102170000714600424fc70267b00a3e0c313540101
:10218000fa7900121678e9600ffa7b0244027005b2
:10219000900393e4f0029d717a007b0080f27a81d3
:1021a0007b0180f174f412229e74fa1222068921b6
:1021b000121a08e970047a898008900393e0600697
:1021c0007a817b018074a3e0a2e0500eaa32ab3387
:1021d000121984aa32ab3312169c900394e0fe5479
:1021e00001f52278221224ea900397e0fca3e0fd97
